Archive member included to satisfy reference by file (symbol)

c:/program files (x86)/atollic/truestudio for stm32 9.3.0/armtools/bin/../lib/gcc/arm-atollic-eabi/6.3.1/../../../../arm-atollic-eabi/lib/armv7-m\libc_nano.a(lib_a-errno.o)
                              Src\syscalls.o (__errno)
c:/program files (x86)/atollic/truestudio for stm32 9.3.0/armtools/bin/../lib/gcc/arm-atollic-eabi/6.3.1/../../../../arm-atollic-eabi/lib/armv7-m\libc_nano.a(lib_a-impure.o)
                              Src\main.o (_impure_ptr)
c:/program files (x86)/atollic/truestudio for stm32 9.3.0/armtools/bin/../lib/gcc/arm-atollic-eabi/6.3.1/../../../../arm-atollic-eabi/lib/armv7-m\libc_nano.a(lib_a-init.o)
                              startup\startup_stm32f207xx.o (__libc_init_array)
c:/program files (x86)/atollic/truestudio for stm32 9.3.0/armtools/bin/../lib/gcc/arm-atollic-eabi/6.3.1/../../../../arm-atollic-eabi/lib/armv7-m\libc_nano.a(lib_a-memcpy-stub.o)
                              Src\atten_ctrl.o (memcpy)
c:/program files (x86)/atollic/truestudio for stm32 9.3.0/armtools/bin/../lib/gcc/arm-atollic-eabi/6.3.1/../../../../arm-atollic-eabi/lib/armv7-m\libc_nano.a(lib_a-memset.o)
                              Src\Character_lcd.o (memset)
c:/program files (x86)/atollic/truestudio for stm32 9.3.0/armtools/bin/../lib/gcc/arm-atollic-eabi/6.3.1/../../../../arm-atollic-eabi/lib/armv7-m\libc_nano.a(lib_a-nano-vfprintf_float.o)
                              (_printf_float)
c:/program files (x86)/atollic/truestudio for stm32 9.3.0/armtools/bin/../lib/gcc/arm-atollic-eabi/6.3.1/../../../../arm-atollic-eabi/lib/armv7-m\libc_nano.a(lib_a-nano-vfprintf_i.o)
                              c:/program files (x86)/atollic/truestudio for stm32 9.3.0/armtools/bin/../lib/gcc/arm-atollic-eabi/6.3.1/../../../../arm-atollic-eabi/lib/armv7-m\libc_nano.a(lib_a-nano-vfprintf_float.o) (_printf_common)
c:/program files (x86)/atollic/truestudio for stm32 9.3.0/armtools/bin/../lib/gcc/arm-atollic-eabi/6.3.1/../../../../arm-atollic-eabi/lib/armv7-m\libc_nano.a(lib_a-printf.o)
                              Src\atten_ctrl.o (printf)
c:/program files (x86)/atollic/truestudio for stm32 9.3.0/armtools/bin/../lib/gcc/arm-atollic-eabi/6.3.1/../../../../arm-atollic-eabi/lib/armv7-m\libc_nano.a(lib_a-puts.o)
                              Src\atten_ctrl.o (puts)
c:/program files (x86)/atollic/truestudio for stm32 9.3.0/armtools/bin/../lib/gcc/arm-atollic-eabi/6.3.1/../../../../arm-atollic-eabi/lib/armv7-m\libc_nano.a(lib_a-setbuf.o)
                              Src\main.o (setbuf)
c:/program files (x86)/atollic/truestudio for stm32 9.3.0/armtools/bin/../lib/gcc/arm-atollic-eabi/6.3.1/../../../../arm-atollic-eabi/lib/armv7-m\libc_nano.a(lib_a-setvbuf.o)
                              c:/program files (x86)/atollic/truestudio for stm32 9.3.0/armtools/bin/../lib/gcc/arm-atollic-eabi/6.3.1/../../../../arm-atollic-eabi/lib/armv7-m\libc_nano.a(lib_a-setbuf.o) (setvbuf)
c:/program files (x86)/atollic/truestudio for stm32 9.3.0/armtools/bin/../lib/gcc/arm-atollic-eabi/6.3.1/../../../../arm-atollic-eabi/lib/armv7-m\libc_nano.a(lib_a-sprintf.o)
                              Src\Character_lcd.o (sprintf)
c:/program files (x86)/atollic/truestudio for stm32 9.3.0/armtools/bin/../lib/gcc/arm-atollic-eabi/6.3.1/../../../../arm-atollic-eabi/lib/armv7-m\libc_nano.a(lib_a-strcpy.o)
                              Src\Character_lcd.o (strcpy)
c:/program files (x86)/atollic/truestudio for stm32 9.3.0/armtools/bin/../lib/gcc/arm-atollic-eabi/6.3.1/../../../../arm-atollic-eabi/lib/armv7-m\libc_nano.a(lib_a-strlen.o)
                              c:/program files (x86)/atollic/truestudio for stm32 9.3.0/armtools/bin/../lib/gcc/arm-atollic-eabi/6.3.1/../../../../arm-atollic-eabi/lib/armv7-m\libc_nano.a(lib_a-nano-vfprintf_float.o) (strlen)
c:/program files (x86)/atollic/truestudio for stm32 9.3.0/armtools/bin/../lib/gcc/arm-atollic-eabi/6.3.1/../../../../arm-atollic-eabi/lib/armv7-m\libc_nano.a(lib_a-wbuf.o)
                              c:/program files (x86)/atollic/truestudio for stm32 9.3.0/armtools/bin/../lib/gcc/arm-atollic-eabi/6.3.1/../../../../arm-atollic-eabi/lib/armv7-m\libc_nano.a(lib_a-puts.o) (__swbuf_r)
c:/program files (x86)/atollic/truestudio for stm32 9.3.0/armtools/bin/../lib/gcc/arm-atollic-eabi/6.3.1/../../../../arm-atollic-eabi/lib/armv7-m\libc_nano.a(lib_a-wsetup.o)
                              c:/program files (x86)/atollic/truestudio for stm32 9.3.0/armtools/bin/../lib/gcc/arm-atollic-eabi/6.3.1/../../../../arm-atollic-eabi/lib/armv7-m\libc_nano.a(lib_a-puts.o) (__swsetup_r)
c:/program files (x86)/atollic/truestudio for stm32 9.3.0/armtools/bin/../lib/gcc/arm-atollic-eabi/6.3.1/../../../../arm-atollic-eabi/lib/armv7-m\libc_nano.a(lib_a-dtoa.o)
                              c:/program files (x86)/atollic/truestudio for stm32 9.3.0/armtools/bin/../lib/gcc/arm-atollic-eabi/6.3.1/../../../../arm-atollic-eabi/lib/armv7-m\libc_nano.a(lib_a-nano-vfprintf_float.o) (_dtoa_r)
c:/program files (x86)/atollic/truestudio for stm32 9.3.0/armtools/bin/../lib/gcc/arm-atollic-eabi/6.3.1/../../../../arm-atollic-eabi/lib/armv7-m\libc_nano.a(lib_a-fflush.o)
                              c:/program files (x86)/atollic/truestudio for stm32 9.3.0/armtools/bin/../lib/gcc/arm-atollic-eabi/6.3.1/../../../../arm-atollic-eabi/lib/armv7-m\libc_nano.a(lib_a-setvbuf.o) (_fflush_r)
c:/program files (x86)/atollic/truestudio for stm32 9.3.0/armtools/bin/../lib/gcc/arm-atollic-eabi/6.3.1/../../../../arm-atollic-eabi/lib/armv7-m\libc_nano.a(lib_a-findfp.o)
                              c:/program files (x86)/atollic/truestudio for stm32 9.3.0/armtools/bin/../lib/gcc/arm-atollic-eabi/6.3.1/../../../../arm-atollic-eabi/lib/armv7-m\libc_nano.a(lib_a-printf.o) (__sinit)
c:/program files (x86)/atollic/truestudio for stm32 9.3.0/armtools/bin/../lib/gcc/arm-atollic-eabi/6.3.1/../../../../arm-atollic-eabi/lib/armv7-m\libc_nano.a(lib_a-fwalk.o)
                              c:/program files (x86)/atollic/truestudio for stm32 9.3.0/armtools/bin/../lib/gcc/arm-atollic-eabi/6.3.1/../../../../arm-atollic-eabi/lib/armv7-m\libc_nano.a(lib_a-findfp.o) (_fwalk)
c:/program files (x86)/atollic/truestudio for stm32 9.3.0/armtools/bin/../lib/gcc/arm-atollic-eabi/6.3.1/../../../../arm-atollic-eabi/lib/armv7-m\libc_nano.a(lib_a-localeconv.o)
                              c:/program files (x86)/atollic/truestudio for stm32 9.3.0/armtools/bin/../lib/gcc/arm-atollic-eabi/6.3.1/../../../../arm-atollic-eabi/lib/armv7-m\libc_nano.a(lib_a-nano-vfprintf_float.o) (_localeconv_r)
c:/program files (x86)/atollic/truestudio for stm32 9.3.0/armtools/bin/../lib/gcc/arm-atollic-eabi/6.3.1/../../../../arm-atollic-eabi/lib/armv7-m\libc_nano.a(lib_a-makebuf.o)
                              c:/program files (x86)/atollic/truestudio for stm32 9.3.0/armtools/bin/../lib/gcc/arm-atollic-eabi/6.3.1/../../../../arm-atollic-eabi/lib/armv7-m\libc_nano.a(lib_a-setvbuf.o) (__swhatbuf_r)
c:/program files (x86)/atollic/truestudio for stm32 9.3.0/armtools/bin/../lib/gcc/arm-atollic-eabi/6.3.1/../../../../arm-atollic-eabi/lib/armv7-m\libc_nano.a(lib_a-malloc.o)
                              c:/program files (x86)/atollic/truestudio for stm32 9.3.0/armtools/bin/../lib/gcc/arm-atollic-eabi/6.3.1/../../../../arm-atollic-eabi/lib/armv7-m\libc_nano.a(lib_a-setvbuf.o) (malloc)
c:/program files (x86)/atollic/truestudio for stm32 9.3.0/armtools/bin/../lib/gcc/arm-atollic-eabi/6.3.1/../../../../arm-atollic-eabi/lib/armv7-m\libc_nano.a(lib_a-memchr-stub.o)
                              c:/program files (x86)/atollic/truestudio for stm32 9.3.0/armtools/bin/../lib/gcc/arm-atollic-eabi/6.3.1/../../../../arm-atollic-eabi/lib/armv7-m\libc_nano.a(lib_a-nano-vfprintf_i.o) (memchr)
c:/program files (x86)/atollic/truestudio for stm32 9.3.0/armtools/bin/../lib/gcc/arm-atollic-eabi/6.3.1/../../../../arm-atollic-eabi/lib/armv7-m\libc_nano.a(lib_a-mprec.o)
                              c:/program files (x86)/atollic/truestudio for stm32 9.3.0/armtools/bin/../lib/gcc/arm-atollic-eabi/6.3.1/../../../../arm-atollic-eabi/lib/armv7-m\libc_nano.a(lib_a-dtoa.o) (_Balloc)
c:/program files (x86)/atollic/truestudio for stm32 9.3.0/armtools/bin/../lib/gcc/arm-atollic-eabi/6.3.1/../../../../arm-atollic-eabi/lib/armv7-m\libc_nano.a(lib_a-nano-callocr.o)
                              c:/program files (x86)/atollic/truestudio for stm32 9.3.0/armtools/bin/../lib/gcc/arm-atollic-eabi/6.3.1/../../../../arm-atollic-eabi/lib/armv7-m\libc_nano.a(lib_a-mprec.o) (_calloc_r)
c:/program files (x86)/atollic/truestudio for stm32 9.3.0/armtools/bin/../lib/gcc/arm-atollic-eabi/6.3.1/../../../../arm-atollic-eabi/lib/armv7-m\libc_nano.a(lib_a-nano-freer.o)
                              c:/program files (x86)/atollic/truestudio for stm32 9.3.0/armtools/bin/../lib/gcc/arm-atollic-eabi/6.3.1/../../../../arm-atollic-eabi/lib/armv7-m\libc_nano.a(lib_a-setvbuf.o) (_free_r)
c:/program files (x86)/atollic/truestudio for stm32 9.3.0/armtools/bin/../lib/gcc/arm-atollic-eabi/6.3.1/../../../../arm-atollic-eabi/lib/armv7-m\libc_nano.a(lib_a-nano-mallocr.o)
                              c:/program files (x86)/atollic/truestudio for stm32 9.3.0/armtools/bin/../lib/gcc/arm-atollic-eabi/6.3.1/../../../../arm-atollic-eabi/lib/armv7-m\libc_nano.a(lib_a-findfp.o) (_malloc_r)
c:/program files (x86)/atollic/truestudio for stm32 9.3.0/armtools/bin/../lib/gcc/arm-atollic-eabi/6.3.1/../../../../arm-atollic-eabi/lib/armv7-m\libc_nano.a(lib_a-nano-svfprintf.o)
                              c:/program files (x86)/atollic/truestudio for stm32 9.3.0/armtools/bin/../lib/gcc/arm-atollic-eabi/6.3.1/../../../../arm-atollic-eabi/lib/armv7-m\libc_nano.a(lib_a-sprintf.o) (_svfprintf_r)
c:/program files (x86)/atollic/truestudio for stm32 9.3.0/armtools/bin/../lib/gcc/arm-atollic-eabi/6.3.1/../../../../arm-atollic-eabi/lib/armv7-m\libc_nano.a(lib_a-nano-vfprintf.o)
                              c:/program files (x86)/atollic/truestudio for stm32 9.3.0/armtools/bin/../lib/gcc/arm-atollic-eabi/6.3.1/../../../../arm-atollic-eabi/lib/armv7-m\libc_nano.a(lib_a-printf.o) (_vfprintf_r)
c:/program files (x86)/atollic/truestudio for stm32 9.3.0/armtools/bin/../lib/gcc/arm-atollic-eabi/6.3.1/../../../../arm-atollic-eabi/lib/armv7-m\libc_nano.a(lib_a-sbrkr.o)
                              c:/program files (x86)/atollic/truestudio for stm32 9.3.0/armtools/bin/../lib/gcc/arm-atollic-eabi/6.3.1/../../../../arm-atollic-eabi/lib/armv7-m\libc_nano.a(lib_a-nano-mallocr.o) (_sbrk_r)
c:/program files (x86)/atollic/truestudio for stm32 9.3.0/armtools/bin/../lib/gcc/arm-atollic-eabi/6.3.1/../../../../arm-atollic-eabi/lib/armv7-m\libc_nano.a(lib_a-stdio.o)
                              c:/program files (x86)/atollic/truestudio for stm32 9.3.0/armtools/bin/../lib/gcc/arm-atollic-eabi/6.3.1/../../../../arm-atollic-eabi/lib/armv7-m\libc_nano.a(lib_a-findfp.o) (__sread)
c:/program files (x86)/atollic/truestudio for stm32 9.3.0/armtools/bin/../lib/gcc/arm-atollic-eabi/6.3.1/../../../../arm-atollic-eabi/lib/armv7-m\libc_nano.a(lib_a-writer.o)
                              c:/program files (x86)/atollic/truestudio for stm32 9.3.0/armtools/bin/../lib/gcc/arm-atollic-eabi/6.3.1/../../../../arm-atollic-eabi/lib/armv7-m\libc_nano.a(lib_a-stdio.o) (_write_r)
c:/program files (x86)/atollic/truestudio for stm32 9.3.0/armtools/bin/../lib/gcc/arm-atollic-eabi/6.3.1/../../../../arm-atollic-eabi/lib/armv7-m\libc_nano.a(lib_a-closer.o)
                              c:/program files (x86)/atollic/truestudio for stm32 9.3.0/armtools/bin/../lib/gcc/arm-atollic-eabi/6.3.1/../../../../arm-atollic-eabi/lib/armv7-m\libc_nano.a(lib_a-stdio.o) (_close_r)
c:/program files (x86)/atollic/truestudio for stm32 9.3.0/armtools/bin/../lib/gcc/arm-atollic-eabi/6.3.1/../../../../arm-atollic-eabi/lib/armv7-m\libc_nano.a(lib_a-fstatr.o)
                              c:/program files (x86)/atollic/truestudio for stm32 9.3.0/armtools/bin/../lib/gcc/arm-atollic-eabi/6.3.1/../../../../arm-atollic-eabi/lib/armv7-m\libc_nano.a(lib_a-makebuf.o) (_fstat_r)
c:/program files (x86)/atollic/truestudio for stm32 9.3.0/armtools/bin/../lib/gcc/arm-atollic-eabi/6.3.1/../../../../arm-atollic-eabi/lib/armv7-m\libc_nano.a(lib_a-fvwrite.o)
                              c:/program files (x86)/atollic/truestudio for stm32 9.3.0/armtools/bin/../lib/gcc/arm-atollic-eabi/6.3.1/../../../../arm-atollic-eabi/lib/armv7-m\libc_nano.a(lib_a-nano-vfprintf.o) (__sfvwrite_r)
c:/program files (x86)/atollic/truestudio for stm32 9.3.0/armtools/bin/../lib/gcc/arm-atollic-eabi/6.3.1/../../../../arm-atollic-eabi/lib/armv7-m\libc_nano.a(lib_a-isattyr.o)
                              c:/program files (x86)/atollic/truestudio for stm32 9.3.0/armtools/bin/../lib/gcc/arm-atollic-eabi/6.3.1/../../../../arm-atollic-eabi/lib/armv7-m\libc_nano.a(lib_a-makebuf.o) (_isatty_r)
c:/program files (x86)/atollic/truestudio for stm32 9.3.0/armtools/bin/../lib/gcc/arm-atollic-eabi/6.3.1/../../../../arm-atollic-eabi/lib/armv7-m\libc_nano.a(lib_a-locale.o)
                              c:/program files (x86)/atollic/truestudio for stm32 9.3.0/armtools/bin/../lib/gcc/arm-atollic-eabi/6.3.1/../../../../arm-atollic-eabi/lib/armv7-m\libc_nano.a(lib_a-localeconv.o) (__global_locale)
c:/program files (x86)/atollic/truestudio for stm32 9.3.0/armtools/bin/../lib/gcc/arm-atollic-eabi/6.3.1/../../../../arm-atollic-eabi/lib/armv7-m\libc_nano.a(lib_a-lseekr.o)
                              c:/program files (x86)/atollic/truestudio for stm32 9.3.0/armtools/bin/../lib/gcc/arm-atollic-eabi/6.3.1/../../../../arm-atollic-eabi/lib/armv7-m\libc_nano.a(lib_a-stdio.o) (_lseek_r)
c:/program files (x86)/atollic/truestudio for stm32 9.3.0/armtools/bin/../lib/gcc/arm-atollic-eabi/6.3.1/../../../../arm-atollic-eabi/lib/armv7-m\libc_nano.a(lib_a-mbtowc_r.o)
                              c:/program files (x86)/atollic/truestudio for stm32 9.3.0/armtools/bin/../lib/gcc/arm-atollic-eabi/6.3.1/../../../../arm-atollic-eabi/lib/armv7-m\libc_nano.a(lib_a-locale.o) (__ascii_mbtowc)
c:/program files (x86)/atollic/truestudio for stm32 9.3.0/armtools/bin/../lib/gcc/arm-atollic-eabi/6.3.1/../../../../arm-atollic-eabi/lib/armv7-m\libc_nano.a(lib_a-memmove.o)
                              c:/program files (x86)/atollic/truestudio for stm32 9.3.0/armtools/bin/../lib/gcc/arm-atollic-eabi/6.3.1/../../../../arm-atollic-eabi/lib/armv7-m\libc_nano.a(lib_a-nano-svfprintf.o) (memmove)
c:/program files (x86)/atollic/truestudio for stm32 9.3.0/armtools/bin/../lib/gcc/arm-atollic-eabi/6.3.1/../../../../arm-atollic-eabi/lib/armv7-m\libc_nano.a(lib_a-mlock.o)
                              c:/program files (x86)/atollic/truestudio for stm32 9.3.0/armtools/bin/../lib/gcc/arm-atollic-eabi/6.3.1/../../../../arm-atollic-eabi/lib/armv7-m\libc_nano.a(lib_a-nano-freer.o) (__malloc_lock)
c:/program files (x86)/atollic/truestudio for stm32 9.3.0/armtools/bin/../lib/gcc/arm-atollic-eabi/6.3.1/../../../../arm-atollic-eabi/lib/armv7-m\libc_nano.a(lib_a-nano-reallocr.o)
                              c:/program files (x86)/atollic/truestudio for stm32 9.3.0/armtools/bin/../lib/gcc/arm-atollic-eabi/6.3.1/../../../../arm-atollic-eabi/lib/armv7-m\libc_nano.a(lib_a-nano-svfprintf.o) (_realloc_r)
c:/program files (x86)/atollic/truestudio for stm32 9.3.0/armtools/bin/../lib/gcc/arm-atollic-eabi/6.3.1/../../../../arm-atollic-eabi/lib/armv7-m\libc_nano.a(lib_a-readr.o)
                              c:/program files (x86)/atollic/truestudio for stm32 9.3.0/armtools/bin/../lib/gcc/arm-atollic-eabi/6.3.1/../../../../arm-atollic-eabi/lib/armv7-m\libc_nano.a(lib_a-stdio.o) (_read_r)
c:/program files (x86)/atollic/truestudio for stm32 9.3.0/armtools/bin/../lib/gcc/arm-atollic-eabi/6.3.1/../../../../arm-atollic-eabi/lib/armv7-m\libc_nano.a(lib_a-reent.o)
                              c:/program files (x86)/atollic/truestudio for stm32 9.3.0/armtools/bin/../lib/gcc/arm-atollic-eabi/6.3.1/../../../../arm-atollic-eabi/lib/armv7-m\libc_nano.a(lib_a-sbrkr.o) (errno)
c:/program files (x86)/atollic/truestudio for stm32 9.3.0/armtools/bin/../lib/gcc/arm-atollic-eabi/6.3.1/../../../../arm-atollic-eabi/lib/armv7-m\libc_nano.a(lib_a-strcmp.o)
                              c:/program files (x86)/atollic/truestudio for stm32 9.3.0/armtools/bin/../lib/gcc/arm-atollic-eabi/6.3.1/../../../../arm-atollic-eabi/lib/armv7-m\libc_nano.a(lib_a-locale.o) (strcmp)
c:/program files (x86)/atollic/truestudio for stm32 9.3.0/armtools/bin/../lib/gcc/arm-atollic-eabi/6.3.1/../../../../arm-atollic-eabi/lib/armv7-m\libc_nano.a(lib_a-wctomb_r.o)
                              c:/program files (x86)/atollic/truestudio for stm32 9.3.0/armtools/bin/../lib/gcc/arm-atollic-eabi/6.3.1/../../../../arm-atollic-eabi/lib/armv7-m\libc_nano.a(lib_a-locale.o) (__ascii_wctomb)
c:/program files (x86)/atollic/truestudio for stm32 9.3.0/armtools/bin/../lib/gcc/arm-atollic-eabi/6.3.1/../../../../arm-atollic-eabi/lib/armv7-m\libc_nano.a(lib_a-ctype_.o)
                              c:/program files (x86)/atollic/truestudio for stm32 9.3.0/armtools/bin/../lib/gcc/arm-atollic-eabi/6.3.1/../../../../arm-atollic-eabi/lib/armv7-m\libc_nano.a(lib_a-locale.o) (_ctype_)
c:/program files (x86)/atollic/truestudio for stm32 9.3.0/armtools/bin/../lib/gcc/arm-atollic-eabi/6.3.1/../../../../arm-atollic-eabi/lib/armv7-m\libc_nano.a(lib_a-nano-msizer.o)
                              c:/program files (x86)/atollic/truestudio for stm32 9.3.0/armtools/bin/../lib/gcc/arm-atollic-eabi/6.3.1/../../../../arm-atollic-eabi/lib/armv7-m\libc_nano.a(lib_a-nano-reallocr.o) (_malloc_usable_size_r)
c:/program files (x86)/atollic/truestudio for stm32 9.3.0/armtools/bin/../lib/gcc/arm-atollic-eabi/6.3.1/armv7-m\libgcc.a(_arm_addsubdf3.o)
                              c:/program files (x86)/atollic/truestudio for stm32 9.3.0/armtools/bin/../lib/gcc/arm-atollic-eabi/6.3.1/../../../../arm-atollic-eabi/lib/armv7-m\libc_nano.a(lib_a-dtoa.o) (__aeabi_dsub)
c:/program files (x86)/atollic/truestudio for stm32 9.3.0/armtools/bin/../lib/gcc/arm-atollic-eabi/6.3.1/armv7-m\libgcc.a(_arm_muldivdf3.o)
                              c:/program files (x86)/atollic/truestudio for stm32 9.3.0/armtools/bin/../lib/gcc/arm-atollic-eabi/6.3.1/../../../../arm-atollic-eabi/lib/armv7-m\libc_nano.a(lib_a-dtoa.o) (__aeabi_dmul)
c:/program files (x86)/atollic/truestudio for stm32 9.3.0/armtools/bin/../lib/gcc/arm-atollic-eabi/6.3.1/armv7-m\libgcc.a(_arm_cmpdf2.o)
                              c:/program files (x86)/atollic/truestudio for stm32 9.3.0/armtools/bin/../lib/gcc/arm-atollic-eabi/6.3.1/../../../../arm-atollic-eabi/lib/armv7-m\libc_nano.a(lib_a-nano-vfprintf_float.o) (__aeabi_dcmpeq)
c:/program files (x86)/atollic/truestudio for stm32 9.3.0/armtools/bin/../lib/gcc/arm-atollic-eabi/6.3.1/armv7-m\libgcc.a(_arm_unorddf2.o)
                              c:/program files (x86)/atollic/truestudio for stm32 9.3.0/armtools/bin/../lib/gcc/arm-atollic-eabi/6.3.1/../../../../arm-atollic-eabi/lib/armv7-m\libc_nano.a(lib_a-nano-vfprintf_float.o) (__aeabi_dcmpun)
c:/program files (x86)/atollic/truestudio for stm32 9.3.0/armtools/bin/../lib/gcc/arm-atollic-eabi/6.3.1/armv7-m\libgcc.a(_arm_fixdfsi.o)
                              c:/program files (x86)/atollic/truestudio for stm32 9.3.0/armtools/bin/../lib/gcc/arm-atollic-eabi/6.3.1/../../../../arm-atollic-eabi/lib/armv7-m\libc_nano.a(lib_a-dtoa.o) (__aeabi_d2iz)
c:/program files (x86)/atollic/truestudio for stm32 9.3.0/armtools/bin/../lib/gcc/arm-atollic-eabi/6.3.1/armv7-m\libgcc.a(_arm_addsubsf3.o)
                              Src\atten_ctrl.o (__aeabi_fsub)
c:/program files (x86)/atollic/truestudio for stm32 9.3.0/armtools/bin/../lib/gcc/arm-atollic-eabi/6.3.1/armv7-m\libgcc.a(_arm_cmpsf2.o)
                              Src\atten_ctrl.o (__aeabi_fcmpeq)
c:/program files (x86)/atollic/truestudio for stm32 9.3.0/armtools/bin/../lib/gcc/arm-atollic-eabi/6.3.1/armv7-m\libgcc.a(_arm_fixunssfsi.o)
                              Src\atten_ctrl.o (__aeabi_f2uiz)
c:/program files (x86)/atollic/truestudio for stm32 9.3.0/armtools/bin/../lib/gcc/arm-atollic-eabi/6.3.1/armv7-m\libgcc.a(_aeabi_uldivmod.o)
                              Drivers\STM32F2xx_HAL_Driver\Src\stm32f2xx_hal_rcc.o (__aeabi_uldivmod)
c:/program files (x86)/atollic/truestudio for stm32 9.3.0/armtools/bin/../lib/gcc/arm-atollic-eabi/6.3.1/armv7-m\libgcc.a(_udivmoddi4.o)
                              c:/program files (x86)/atollic/truestudio for stm32 9.3.0/armtools/bin/../lib/gcc/arm-atollic-eabi/6.3.1/armv7-m\libgcc.a(_aeabi_uldivmod.o) (__udivmoddi4)
c:/program files (x86)/atollic/truestudio for stm32 9.3.0/armtools/bin/../lib/gcc/arm-atollic-eabi/6.3.1/armv7-m\libgcc.a(_dvmd_tls.o)
                              c:/program files (x86)/atollic/truestudio for stm32 9.3.0/armtools/bin/../lib/gcc/arm-atollic-eabi/6.3.1/armv7-m\libgcc.a(_aeabi_uldivmod.o) (__aeabi_ldiv0)

Allocating common symbols
Common symbol       size              file

ATT_B_EN_WIFI4_2_4Ghz_Table
                    0x40              Src\atten_ctrl.o
hi2c3               0x54              Src\main.o
ATT_A_EN_30G3_29_29_5Ghz_Table
                    0x40              Src\atten_ctrl.o
ATT_B_EN_30G1_28_28_5Ghz_Table
                    0x40              Src\atten_ctrl.o
ATT_A_EN_WIFI4_2_4Ghz_Table
                    0x40              Src\atten_ctrl.o
ATT_A_EN_30G3_29_5_30Ghz_Table
                    0x40              Src\atten_ctrl.o
errno               0x4               c:/program files (x86)/atollic/truestudio for stm32 9.3.0/armtools/bin/../lib/gcc/arm-atollic-eabi/6.3.1/../../../../arm-atollic-eabi/lib/armv7-m\libc_nano.a(lib_a-reent.o)
hdma_usart3_rx      0x60              Src\main.o
UartDataisReved     0x1               Src\main.o
huart3              0x40              Src\main.o
ATT_B_EN_WIFI3_5_8Ghz_Table
                    0x40              Src\atten_ctrl.o
ATT_B_EN_30G3_28_5_29Ghz_Table
                    0x40              Src\atten_ctrl.o
ATT_A_EN_WIFI1_2_4Ghz_Table
                    0x40              Src\atten_ctrl.o
rx2_data            0x2               Src\main.o
ATT_B_EN_30G2_28_28_5Ghz_Table
                    0x40              Src\atten_ctrl.o
ATT_B_EN_WIFI4_5_8Ghz_Table
                    0x40              Src\atten_ctrl.o
ATT_A_EN_WIFI3_2_4Ghz_Table
                    0x40              Src\atten_ctrl.o
ATT_B_EN_WIFI2_2_4Ghz_Table
                    0x40              Src\atten_ctrl.o
ATT_B_EN_30G1_28_5_29Ghz_Table
                    0x40              Src\atten_ctrl.o
ATT_A_EN_30G2_28_5_29Ghz_Table
                    0x40              Src\atten_ctrl.o
ATT_B_EN_WIFI1_2_4Ghz_Table
                    0x40              Src\atten_ctrl.o
uwTick              0x4               Drivers\STM32F2xx_HAL_Driver\Src\stm32f2xx_hal.o
ATT_A_EN_30G2_29_29_5Ghz_Table
                    0x40              Src\atten_ctrl.o
ATT_B_EN_30G3_29_29_5Ghz_Table
                    0x40              Src\atten_ctrl.o
hdma_usart3_tx      0x60              Src\main.o
pFlash              0x20              Drivers\STM32F2xx_HAL_Driver\Src\stm32f2xx_hal_flash.o
count_out           0x1               Src\main.o
ATT_B_EN_30G2_28_5_29Ghz_Table
                    0x40              Src\atten_ctrl.o
ATT_A_EN_30G3_28_5_29Ghz_Table
                    0x40              Src\atten_ctrl.o
count_in            0x1               Src\main.o
ATT_B_EN_WIFI2_5_8Ghz_Table
                    0x40              Src\atten_ctrl.o
ATT_A_EN_30G1_28_28_5Ghz_Table
                    0x40              Src\atten_ctrl.o
ATT_B_EN_30G1_29_29_5Ghz_Table
                    0x40              Src\atten_ctrl.o
ATT_B_EN_30G2_29_29_5Ghz_Table
                    0x40              Src\atten_ctrl.o
ATT_A_EN_WIFI3_5_8Ghz_Table
                    0x40              Src\atten_ctrl.o
ATT_A_EN_30G3_28_28_5Ghz_Table
                    0x40              Src\atten_ctrl.o
ATT_A_EN_WIFI4_5_8Ghz_Table
                    0x40              Src\atten_ctrl.o
Atten_Setting       0x30              Src\atten_ctrl.o
ATT_A_EN_150M_Table
                    0x40              Src\atten_ctrl.o
ATT_B_EN_WIFI3_2_4Ghz_Table
                    0x40              Src\atten_ctrl.o
ATT_A_EN_30G2_29_5_30Ghz_Table
                    0x40              Src\atten_ctrl.o
ring_buf            0x64              Src\main.o
ATT_A_EN_30G1_29_5_30Ghz_Table
                    0x40              Src\atten_ctrl.o
ATT_B_EN_30G3_29_5_30Ghz_Table
                    0x40              Src\atten_ctrl.o
ATT_A_EN_30G1_28_5_29Ghz_Table
                    0x40              Src\atten_ctrl.o
ATT_B_EN_30G1_29_5_30Ghz_Table
                    0x40              Src\atten_ctrl.o
ATT_B_EN_150M_Table
                    0x40              Src\atten_ctrl.o
htim6               0x40              Src\main.o
ATT_B_EN_30G3_28_28_5Ghz_Table
                    0x40              Src\atten_ctrl.o
Timer10ms           0x4               Src\main.o
ATT_A_EN_WIFI1_5_8Ghz_Table
                    0x40              Src\atten_ctrl.o
ATT_B_EN_WIFI1_5_8Ghz_Table
                    0x40              Src\atten_ctrl.o
TerminalQueue       0x40c             Src\uart.o
ATT_B_EN_30G2_29_5_30Ghz_Table
                    0x40              Src\atten_ctrl.o
ATT_A_EN_30G2_28_28_5Ghz_Table
                    0x40              Src\atten_ctrl.o
ATT_A_EN_WIFI2_2_4Ghz_Table
                    0x40              Src\atten_ctrl.o
ATT_Curr_Value      0x10              Src\atten_ctrl.o
ATT_A_EN_30G1_29_29_5Ghz_Table
                    0x40              Src\atten_ctrl.o
WifiQueue           0x40c             Src\uart.o
ATT_A_EN_WIFI2_5_8Ghz_Table
                    0x40              Src\atten_ctrl.o

Discarded input sections

 .text          0x00000000        0x0 c:/program files (x86)/atollic/truestudio for stm32 9.3.0/armtools/bin/../lib/gcc/arm-atollic-eabi/6.3.1/armv7-m/crti.o
 .data          0x00000000        0x0 c:/program files (x86)/atollic/truestudio for stm32 9.3.0/armtools/bin/../lib/gcc/arm-atollic-eabi/6.3.1/armv7-m/crti.o
 .bss           0x00000000        0x0 c:/program files (x86)/atollic/truestudio for stm32 9.3.0/armtools/bin/../lib/gcc/arm-atollic-eabi/6.3.1/armv7-m/crti.o
 .data          0x00000000        0x4 c:/program files (x86)/atollic/truestudio for stm32 9.3.0/armtools/bin/../lib/gcc/arm-atollic-eabi/6.3.1/armv7-m/crtbegin.o
 .text          0x00000000        0x0 Drivers\STM32F2xx_HAL_Driver\Src\stm32f2xx_hal.o
 .data          0x00000000        0x0 Drivers\STM32F2xx_HAL_Driver\Src\stm32f2xx_hal.o
 .bss           0x00000000        0x0 Drivers\STM32F2xx_HAL_Driver\Src\stm32f2xx_hal.o
 .text.HAL_MspInit
                0x00000000        0x2 Drivers\STM32F2xx_HAL_Driver\Src\stm32f2xx_hal.o
 .text.HAL_MspDeInit
                0x00000000        0x2 Drivers\STM32F2xx_HAL_Driver\Src\stm32f2xx_hal.o
 .text.HAL_DeInit
                0x00000000       0x2c Drivers\STM32F2xx_HAL_Driver\Src\stm32f2xx_hal.o
 .text.HAL_GetTickPrio
                0x00000000        0xc Drivers\STM32F2xx_HAL_Driver\Src\stm32f2xx_hal.o
 .text.HAL_SetTickFreq
                0x00000000       0x28 Drivers\STM32F2xx_HAL_Driver\Src\stm32f2xx_hal.o
 .text.HAL_GetTickFreq
                0x00000000        0xc Drivers\STM32F2xx_HAL_Driver\Src\stm32f2xx_hal.o
 .text.HAL_SuspendTick
                0x00000000       0x10 Drivers\STM32F2xx_HAL_Driver\Src\stm32f2xx_hal.o
 .text.HAL_ResumeTick
                0x00000000       0x10 Drivers\STM32F2xx_HAL_Driver\Src\stm32f2xx_hal.o
 .text.HAL_GetHalVersion
                0x00000000        0x8 Drivers\STM32F2xx_HAL_Driver\Src\stm32f2xx_hal.o
 .text.HAL_GetREVID
                0x00000000        0xc Drivers\STM32F2xx_HAL_Driver\Src\stm32f2xx_hal.o
 .text.HAL_GetDEVID
                0x00000000       0x10 Drivers\STM32F2xx_HAL_Driver\Src\stm32f2xx_hal.o
 .text.HAL_DBGMCU_EnableDBGSleepMode
                0x00000000       0x10 Drivers\STM32F2xx_HAL_Driver\Src\stm32f2xx_hal.o
 .text.HAL_DBGMCU_DisableDBGSleepMode
                0x00000000       0x10 Drivers\STM32F2xx_HAL_Driver\Src\stm32f2xx_hal.o
 .text.HAL_DBGMCU_EnableDBGStopMode
                0x00000000       0x10 Drivers\STM32F2xx_HAL_Driver\Src\stm32f2xx_hal.o
 .text.HAL_DBGMCU_DisableDBGStopMode
                0x00000000       0x10 Drivers\STM32F2xx_HAL_Driver\Src\stm32f2xx_hal.o
 .text.HAL_DBGMCU_EnableDBGStandbyMode
                0x00000000       0x10 Drivers\STM32F2xx_HAL_Driver\Src\stm32f2xx_hal.o
 .text.HAL_DBGMCU_DisableDBGStandbyMode
                0x00000000       0x10 Drivers\STM32F2xx_HAL_Driver\Src\stm32f2xx_hal.o
 .text.HAL_EnableCompensationCell
                0x00000000       0x18 Drivers\STM32F2xx_HAL_Driver\Src\stm32f2xx_hal.o
 .text.HAL_DisableCompensationCell
                0x00000000       0x1c Drivers\STM32F2xx_HAL_Driver\Src\stm32f2xx_hal.o
 .text.HAL_GetUIDw0
                0x00000000        0xc Drivers\STM32F2xx_HAL_Driver\Src\stm32f2xx_hal.o
 .text.HAL_GetUIDw1
                0x00000000        0xc Drivers\STM32F2xx_HAL_Driver\Src\stm32f2xx_hal.o
 .text.HAL_GetUIDw2
                0x00000000        0xc Drivers\STM32F2xx_HAL_Driver\Src\stm32f2xx_hal.o
 .text          0x00000000        0x0 Drivers\STM32F2xx_HAL_Driver\Src\stm32f2xx_hal_cortex.o
 .data          0x00000000        0x0 Drivers\STM32F2xx_HAL_Driver\Src\stm32f2xx_hal_cortex.o
 .bss           0x00000000        0x0 Drivers\STM32F2xx_HAL_Driver\Src\stm32f2xx_hal_cortex.o
 .text.HAL_NVIC_DisableIRQ
                0x00000000       0x28 Drivers\STM32F2xx_HAL_Driver\Src\stm32f2xx_hal_cortex.o
 .text.HAL_NVIC_SystemReset
                0x00000000       0x24 Drivers\STM32F2xx_HAL_Driver\Src\stm32f2xx_hal_cortex.o
 .text.HAL_MPU_Disable
                0x00000000       0x20 Drivers\STM32F2xx_HAL_Driver\Src\stm32f2xx_hal_cortex.o
 .text.HAL_MPU_Enable
                0x00000000       0x24 Drivers\STM32F2xx_HAL_Driver\Src\stm32f2xx_hal_cortex.o
 .text.HAL_MPU_ConfigRegion
                0x00000000       0x50 Drivers\STM32F2xx_HAL_Driver\Src\stm32f2xx_hal_cortex.o
 .text.HAL_NVIC_GetPriorityGrouping
                0x00000000       0x10 Drivers\STM32F2xx_HAL_Driver\Src\stm32f2xx_hal_cortex.o
 .text.HAL_NVIC_GetPriority
                0x00000000       0x5c Drivers\STM32F2xx_HAL_Driver\Src\stm32f2xx_hal_cortex.o
 .text.HAL_NVIC_SetPendingIRQ
                0x00000000       0x20 Drivers\STM32F2xx_HAL_Driver\Src\stm32f2xx_hal_cortex.o
 .text.HAL_NVIC_GetPendingIRQ
                0x00000000       0x24 Drivers\STM32F2xx_HAL_Driver\Src\stm32f2xx_hal_cortex.o
 .text.HAL_NVIC_ClearPendingIRQ
                0x00000000       0x20 Drivers\STM32F2xx_HAL_Driver\Src\stm32f2xx_hal_cortex.o
 .text.HAL_NVIC_GetActive
                0x00000000       0x24 Drivers\STM32F2xx_HAL_Driver\Src\stm32f2xx_hal_cortex.o
 .text.HAL_SYSTICK_CLKSourceConfig
                0x00000000       0x18 Drivers\STM32F2xx_HAL_Driver\Src\stm32f2xx_hal_cortex.o
 .text.HAL_SYSTICK_Callback
                0x00000000        0x2 Drivers\STM32F2xx_HAL_Driver\Src\stm32f2xx_hal_cortex.o
 .text.HAL_SYSTICK_IRQHandler
                0x00000000        0x8 Drivers\STM32F2xx_HAL_Driver\Src\stm32f2xx_hal_cortex.o
 .text          0x00000000        0x0 Drivers\STM32F2xx_HAL_Driver\Src\stm32f2xx_hal_dma.o
 .data          0x00000000        0x0 Drivers\STM32F2xx_HAL_Driver\Src\stm32f2xx_hal_dma.o
 .bss           0x00000000        0x0 Drivers\STM32F2xx_HAL_Driver\Src\stm32f2xx_hal_dma.o
 .text.HAL_DMA_DeInit
                0x00000000       0x54 Drivers\STM32F2xx_HAL_Driver\Src\stm32f2xx_hal_dma.o
 .text.HAL_DMA_Start
                0x00000000       0x52 Drivers\STM32F2xx_HAL_Driver\Src\stm32f2xx_hal_dma.o
 .text.HAL_DMA_Abort
                0x00000000       0x86 Drivers\STM32F2xx_HAL_Driver\Src\stm32f2xx_hal_dma.o
 .text.HAL_DMA_PollForTransfer
                0x00000000      0x112 Drivers\STM32F2xx_HAL_Driver\Src\stm32f2xx_hal_dma.o
 .text.HAL_DMA_RegisterCallback
                0x00000000       0x50 Drivers\STM32F2xx_HAL_Driver\Src\stm32f2xx_hal_dma.o
 .text.HAL_DMA_UnRegisterCallback
                0x00000000       0x5c Drivers\STM32F2xx_HAL_Driver\Src\stm32f2xx_hal_dma.o
 .text.HAL_DMA_GetState
                0x00000000        0x6 Drivers\STM32F2xx_HAL_Driver\Src\stm32f2xx_hal_dma.o
 .text.HAL_DMA_GetError
                0x00000000        0x4 Drivers\STM32F2xx_HAL_Driver\Src\stm32f2xx_hal_dma.o
 .text          0x00000000        0x0 Drivers\STM32F2xx_HAL_Driver\Src\stm32f2xx_hal_dma_ex.o
 .data          0x00000000        0x0 Drivers\STM32F2xx_HAL_Driver\Src\stm32f2xx_hal_dma_ex.o
 .bss           0x00000000        0x0 Drivers\STM32F2xx_HAL_Driver\Src\stm32f2xx_hal_dma_ex.o
 .text.HAL_DMAEx_MultiBufferStart
                0x00000000       0x5a Drivers\STM32F2xx_HAL_Driver\Src\stm32f2xx_hal_dma_ex.o
 .text.HAL_DMAEx_MultiBufferStart_IT
                0x00000000      0x3e8 Drivers\STM32F2xx_HAL_Driver\Src\stm32f2xx_hal_dma_ex.o
 .text.HAL_DMAEx_ChangeMemory
                0x00000000        0xe Drivers\STM32F2xx_HAL_Driver\Src\stm32f2xx_hal_dma_ex.o
 .debug_info    0x00000000      0x62b Drivers\STM32F2xx_HAL_Driver\Src\stm32f2xx_hal_dma_ex.o
 .debug_abbrev  0x00000000      0x1ad Drivers\STM32F2xx_HAL_Driver\Src\stm32f2xx_hal_dma_ex.o
 .debug_loc     0x00000000      0x452 Drivers\STM32F2xx_HAL_Driver\Src\stm32f2xx_hal_dma_ex.o
 .debug_aranges
                0x00000000       0x30 Drivers\STM32F2xx_HAL_Driver\Src\stm32f2xx_hal_dma_ex.o
 .debug_ranges  0x00000000       0x58 Drivers\STM32F2xx_HAL_Driver\Src\stm32f2xx_hal_dma_ex.o
 .debug_line    0x00000000      0x5a0 Drivers\STM32F2xx_HAL_Driver\Src\stm32f2xx_hal_dma_ex.o
 .debug_str     0x00000000      0x61d Drivers\STM32F2xx_HAL_Driver\Src\stm32f2xx_hal_dma_ex.o
 .comment       0x00000000       0x7d Drivers\STM32F2xx_HAL_Driver\Src\stm32f2xx_hal_dma_ex.o
 .debug_frame   0x00000000       0x58 Drivers\STM32F2xx_HAL_Driver\Src\stm32f2xx_hal_dma_ex.o
 .ARM.attributes
                0x00000000       0x33 Drivers\STM32F2xx_HAL_Driver\Src\stm32f2xx_hal_dma_ex.o
 .text          0x00000000        0x0 Drivers\STM32F2xx_HAL_Driver\Src\stm32f2xx_hal_exti.o
 .data          0x00000000        0x0 Drivers\STM32F2xx_HAL_Driver\Src\stm32f2xx_hal_exti.o
 .bss           0x00000000        0x0 Drivers\STM32F2xx_HAL_Driver\Src\stm32f2xx_hal_exti.o
 .text.HAL_EXTI_SetConfigLine
                0x00000000       0xa4 Drivers\STM32F2xx_HAL_Driver\Src\stm32f2xx_hal_exti.o
 .text.HAL_EXTI_GetConfigLine
                0x00000000       0x90 Drivers\STM32F2xx_HAL_Driver\Src\stm32f2xx_hal_exti.o
 .text.HAL_EXTI_ClearConfigLine
                0x00000000       0x68 Drivers\STM32F2xx_HAL_Driver\Src\stm32f2xx_hal_exti.o
 .text.HAL_EXTI_RegisterCallback
                0x00000000        0xc Drivers\STM32F2xx_HAL_Driver\Src\stm32f2xx_hal_exti.o
 .text.HAL_EXTI_GetHandle
                0x00000000        0xc Drivers\STM32F2xx_HAL_Driver\Src\stm32f2xx_hal_exti.o
 .text.HAL_EXTI_IRQHandler
                0x00000000       0x20 Drivers\STM32F2xx_HAL_Driver\Src\stm32f2xx_hal_exti.o
 .text.HAL_EXTI_GetPending
                0x00000000       0x1c Drivers\STM32F2xx_HAL_Driver\Src\stm32f2xx_hal_exti.o
 .text.HAL_EXTI_ClearPending
                0x00000000       0x14 Drivers\STM32F2xx_HAL_Driver\Src\stm32f2xx_hal_exti.o
 .text.HAL_EXTI_GenerateSWI
                0x00000000       0x14 Drivers\STM32F2xx_HAL_Driver\Src\stm32f2xx_hal_exti.o
 .debug_info    0x00000000      0x5f6 Drivers\STM32F2xx_HAL_Driver\Src\stm32f2xx_hal_exti.o
 .debug_abbrev  0x00000000      0x1e1 Drivers\STM32F2xx_HAL_Driver\Src\stm32f2xx_hal_exti.o
 .debug_loc     0x00000000      0x3d0 Drivers\STM32F2xx_HAL_Driver\Src\stm32f2xx_hal_exti.o
 .debug_aranges
                0x00000000       0x60 Drivers\STM32F2xx_HAL_Driver\Src\stm32f2xx_hal_exti.o
 .debug_ranges  0x00000000       0x50 Drivers\STM32F2xx_HAL_Driver\Src\stm32f2xx_hal_exti.o
 .debug_line    0x00000000      0x364 Drivers\STM32F2xx_HAL_Driver\Src\stm32f2xx_hal_exti.o
 .debug_str     0x00000000      0x4b5 Drivers\STM32F2xx_HAL_Driver\Src\stm32f2xx_hal_exti.o
 .comment       0x00000000       0x7d Drivers\STM32F2xx_HAL_Driver\Src\stm32f2xx_hal_exti.o
 .debug_frame   0x00000000       0xc0 Drivers\STM32F2xx_HAL_Driver\Src\stm32f2xx_hal_exti.o
 .ARM.attributes
                0x00000000       0x33 Drivers\STM32F2xx_HAL_Driver\Src\stm32f2xx_hal_exti.o
 .text          0x00000000        0x0 Drivers\STM32F2xx_HAL_Driver\Src\stm32f2xx_hal_flash.o
 .data          0x00000000        0x0 Drivers\STM32F2xx_HAL_Driver\Src\stm32f2xx_hal_flash.o
 .bss           0x00000000        0x0 Drivers\STM32F2xx_HAL_Driver\Src\stm32f2xx_hal_flash.o
 .text.FLASH_Program_DoubleWord
                0x00000000       0x2c Drivers\STM32F2xx_HAL_Driver\Src\stm32f2xx_hal_flash.o
 .text.FLASH_Program_Word
                0x00000000       0x24 Drivers\STM32F2xx_HAL_Driver\Src\stm32f2xx_hal_flash.o
 .text.FLASH_Program_HalfWord
                0x00000000       0x24 Drivers\STM32F2xx_HAL_Driver\Src\stm32f2xx_hal_flash.o
 .text.FLASH_SetErrorCode
                0x00000000       0x74 Drivers\STM32F2xx_HAL_Driver\Src\stm32f2xx_hal_flash.o
 .text.HAL_FLASH_Program_IT
                0x00000000       0x74 Drivers\STM32F2xx_HAL_Driver\Src\stm32f2xx_hal_flash.o
 .text.HAL_FLASH_EndOfOperationCallback
                0x00000000        0x2 Drivers\STM32F2xx_HAL_Driver\Src\stm32f2xx_hal_flash.o
 .text.HAL_FLASH_OperationErrorCallback
                0x00000000        0x2 Drivers\STM32F2xx_HAL_Driver\Src\stm32f2xx_hal_flash.o
 .text.HAL_FLASH_IRQHandler
                0x00000000       0xc4 Drivers\STM32F2xx_HAL_Driver\Src\stm32f2xx_hal_flash.o
 .text.HAL_FLASH_Unlock
                0x00000000       0x24 Drivers\STM32F2xx_HAL_Driver\Src\stm32f2xx_hal_flash.o
 .text.HAL_FLASH_Lock
                0x00000000       0x14 Drivers\STM32F2xx_HAL_Driver\Src\stm32f2xx_hal_flash.o
 .text.HAL_FLASH_OB_Unlock
                0x00000000       0x24 Drivers\STM32F2xx_HAL_Driver\Src\stm32f2xx_hal_flash.o
 .text.HAL_FLASH_OB_Lock
                0x00000000       0x14 Drivers\STM32F2xx_HAL_Driver\Src\stm32f2xx_hal_flash.o
 .text.HAL_FLASH_GetError
                0x00000000        0xc Drivers\STM32F2xx_HAL_Driver\Src\stm32f2xx_hal_flash.o
 .text.FLASH_WaitForLastOperation
                0x00000000       0x54 Drivers\STM32F2xx_HAL_Driver\Src\stm32f2xx_hal_flash.o
 .text.HAL_FLASH_Program
                0x00000000       0x90 Drivers\STM32F2xx_HAL_Driver\Src\stm32f2xx_hal_flash.o
 .text.HAL_FLASH_OB_Launch
                0x00000000       0x18 Drivers\STM32F2xx_HAL_Driver\Src\stm32f2xx_hal_flash.o
 .debug_info    0x00000000      0x7a5 Drivers\STM32F2xx_HAL_Driver\Src\stm32f2xx_hal_flash.o
 .debug_abbrev  0x00000000      0x2e1 Drivers\STM32F2xx_HAL_Driver\Src\stm32f2xx_hal_flash.o
 .debug_loc     0x00000000      0x2e4 Drivers\STM32F2xx_HAL_Driver\Src\stm32f2xx_hal_flash.o
 .debug_aranges
                0x00000000       0x90 Drivers\STM32F2xx_HAL_Driver\Src\stm32f2xx_hal_flash.o
 .debug_ranges  0x00000000       0xb0 Drivers\STM32F2xx_HAL_Driver\Src\stm32f2xx_hal_flash.o
 .debug_line    0x00000000      0x46d Drivers\STM32F2xx_HAL_Driver\Src\stm32f2xx_hal_flash.o
 .debug_str     0x00000000      0x605 Drivers\STM32F2xx_HAL_Driver\Src\stm32f2xx_hal_flash.o
 .comment       0x00000000       0x7d Drivers\STM32F2xx_HAL_Driver\Src\stm32f2xx_hal_flash.o
 .debug_frame   0x00000000      0x154 Drivers\STM32F2xx_HAL_Driver\Src\stm32f2xx_hal_flash.o
 .ARM.attributes
                0x00000000       0x33 Drivers\STM32F2xx_HAL_Driver\Src\stm32f2xx_hal_flash.o
 COMMON         0x00000000       0x20 Drivers\STM32F2xx_HAL_Driver\Src\stm32f2xx_hal_flash.o
 .text          0x00000000        0x0 Drivers\STM32F2xx_HAL_Driver\Src\stm32f2xx_hal_flash_ex.o
 .data          0x00000000        0x0 Drivers\STM32F2xx_HAL_Driver\Src\stm32f2xx_hal_flash_ex.o
 .bss           0x00000000        0x0 Drivers\STM32F2xx_HAL_Driver\Src\stm32f2xx_hal_flash_ex.o
 .text.FLASH_MassErase.isra.0
                0x00000000       0x24 Drivers\STM32F2xx_HAL_Driver\Src\stm32f2xx_hal_flash_ex.o
 .text.HAL_FLASHEx_OBProgram
                0x00000000       0xb8 Drivers\STM32F2xx_HAL_Driver\Src\stm32f2xx_hal_flash_ex.o
 .text.HAL_FLASHEx_OBGetConfig
                0x00000000       0x48 Drivers\STM32F2xx_HAL_Driver\Src\stm32f2xx_hal_flash_ex.o
 .text.FLASH_Erase_Sector
                0x00000000       0x54 Drivers\STM32F2xx_HAL_Driver\Src\stm32f2xx_hal_flash_ex.o
 .text.HAL_FLASHEx_Erase_IT
                0x00000000       0x60 Drivers\STM32F2xx_HAL_Driver\Src\stm32f2xx_hal_flash_ex.o
 .text.FLASH_FlushCaches
                0x00000000       0x58 Drivers\STM32F2xx_HAL_Driver\Src\stm32f2xx_hal_flash_ex.o
 .text.HAL_FLASHEx_Erase
                0x00000000       0x9c Drivers\STM32F2xx_HAL_Driver\Src\stm32f2xx_hal_flash_ex.o
 .debug_info    0x00000000      0x922 Drivers\STM32F2xx_HAL_Driver\Src\stm32f2xx_hal_flash_ex.o
 .debug_abbrev  0x00000000      0x2e4 Drivers\STM32F2xx_HAL_Driver\Src\stm32f2xx_hal_flash_ex.o
 .debug_loc     0x00000000      0x3fa Drivers\STM32F2xx_HAL_Driver\Src\stm32f2xx_hal_flash_ex.o
 .debug_aranges
                0x00000000       0x50 Drivers\STM32F2xx_HAL_Driver\Src\stm32f2xx_hal_flash_ex.o
 .debug_ranges  0x00000000       0xf0 Drivers\STM32F2xx_HAL_Driver\Src\stm32f2xx_hal_flash_ex.o
 .debug_line    0x00000000      0x432 Drivers\STM32F2xx_HAL_Driver\Src\stm32f2xx_hal_flash_ex.o
 .debug_str     0x00000000      0x669 Drivers\STM32F2xx_HAL_Driver\Src\stm32f2xx_hal_flash_ex.o
 .comment       0x00000000       0x7d Drivers\STM32F2xx_HAL_Driver\Src\stm32f2xx_hal_flash_ex.o
 .debug_frame   0x00000000       0xa8 Drivers\STM32F2xx_HAL_Driver\Src\stm32f2xx_hal_flash_ex.o
 .ARM.attributes
                0x00000000       0x33 Drivers\STM32F2xx_HAL_Driver\Src\stm32f2xx_hal_flash_ex.o
 .text          0x00000000        0x0 Drivers\STM32F2xx_HAL_Driver\Src\stm32f2xx_hal_gpio.o
 .data          0x00000000        0x0 Drivers\STM32F2xx_HAL_Driver\Src\stm32f2xx_hal_gpio.o
 .bss           0x00000000        0x0 Drivers\STM32F2xx_HAL_Driver\Src\stm32f2xx_hal_gpio.o
 .text.HAL_GPIO_DeInit
                0x00000000      0x12c Drivers\STM32F2xx_HAL_Driver\Src\stm32f2xx_hal_gpio.o
 .text.HAL_GPIO_LockPin
                0x00000000       0x2a Drivers\STM32F2xx_HAL_Driver\Src\stm32f2xx_hal_gpio.o
 .text.HAL_GPIO_EXTI_Callback
                0x00000000        0x2 Drivers\STM32F2xx_HAL_Driver\Src\stm32f2xx_hal_gpio.o
 .text          0x00000000        0x0 Drivers\STM32F2xx_HAL_Driver\Src\stm32f2xx_hal_i2c.o
 .data          0x00000000        0x0 Drivers\STM32F2xx_HAL_Driver\Src\stm32f2xx_hal_i2c.o
 .bss           0x00000000        0x0 Drivers\STM32F2xx_HAL_Driver\Src\stm32f2xx_hal_i2c.o
 .text.HAL_I2C_MspInit
                0x00000000        0x2 Drivers\STM32F2xx_HAL_Driver\Src\stm32f2xx_hal_i2c.o
 .text.HAL_I2C_MspDeInit
                0x00000000        0x2 Drivers\STM32F2xx_HAL_Driver\Src\stm32f2xx_hal_i2c.o
 .text.HAL_I2C_DeInit
                0x00000000       0x32 Drivers\STM32F2xx_HAL_Driver\Src\stm32f2xx_hal_i2c.o
 .text.HAL_I2C_Master_Transmit
                0x00000000      0x19c Drivers\STM32F2xx_HAL_Driver\Src\stm32f2xx_hal_i2c.o
 .text.HAL_I2C_Master_Receive
                0x00000000      0x2dc Drivers\STM32F2xx_HAL_Driver\Src\stm32f2xx_hal_i2c.o
 .text.HAL_I2C_Slave_Transmit
                0x00000000      0x158 Drivers\STM32F2xx_HAL_Driver\Src\stm32f2xx_hal_i2c.o
 .text.HAL_I2C_Slave_Receive
                0x00000000      0x178 Drivers\STM32F2xx_HAL_Driver\Src\stm32f2xx_hal_i2c.o
 .text.HAL_I2C_Master_Transmit_IT
                0x00000000       0xb8 Drivers\STM32F2xx_HAL_Driver\Src\stm32f2xx_hal_i2c.o
 .text.HAL_I2C_Master_Receive_IT
                0x00000000       0xc0 Drivers\STM32F2xx_HAL_Driver\Src\stm32f2xx_hal_i2c.o
 .text.HAL_I2C_Slave_Transmit_IT
                0x00000000       0x78 Drivers\STM32F2xx_HAL_Driver\Src\stm32f2xx_hal_i2c.o
 .text.HAL_I2C_Slave_Receive_IT
                0x00000000       0x78 Drivers\STM32F2xx_HAL_Driver\Src\stm32f2xx_hal_i2c.o
 .text.HAL_I2C_Master_Transmit_DMA
                0x00000000      0x12c Drivers\STM32F2xx_HAL_Driver\Src\stm32f2xx_hal_i2c.o
 .text.HAL_I2C_Master_Receive_DMA
                0x00000000      0x12c Drivers\STM32F2xx_HAL_Driver\Src\stm32f2xx_hal_i2c.o
 .text.HAL_I2C_Slave_Transmit_DMA
                0x00000000       0xc0 Drivers\STM32F2xx_HAL_Driver\Src\stm32f2xx_hal_i2c.o
 .text.HAL_I2C_Slave_Receive_DMA
                0x00000000       0xc0 Drivers\STM32F2xx_HAL_Driver\Src\stm32f2xx_hal_i2c.o
 .text.HAL_I2C_Mem_Write_IT
                0x00000000       0xc4 Drivers\STM32F2xx_HAL_Driver\Src\stm32f2xx_hal_i2c.o
 .text.HAL_I2C_Mem_Read_IT
                0x00000000       0xd4 Drivers\STM32F2xx_HAL_Driver\Src\stm32f2xx_hal_i2c.o
 .text.HAL_I2C_Mem_Write_DMA
                0x00000000      0x144 Drivers\STM32F2xx_HAL_Driver\Src\stm32f2xx_hal_i2c.o
 .text.HAL_I2C_Mem_Read_DMA
                0x00000000      0x190 Drivers\STM32F2xx_HAL_Driver\Src\stm32f2xx_hal_i2c.o
 .text.HAL_I2C_IsDeviceReady
                0x00000000      0x154 Drivers\STM32F2xx_HAL_Driver\Src\stm32f2xx_hal_i2c.o
 .text.HAL_I2C_Master_Seq_Transmit_IT
                0x00000000       0xd8 Drivers\STM32F2xx_HAL_Driver\Src\stm32f2xx_hal_i2c.o
 .text.HAL_I2C_Master_Seq_Transmit_DMA
                0x00000000      0x174 Drivers\STM32F2xx_HAL_Driver\Src\stm32f2xx_hal_i2c.o
 .text.HAL_I2C_Master_Seq_Receive_IT
                0x00000000      0x110 Drivers\STM32F2xx_HAL_Driver\Src\stm32f2xx_hal_i2c.o
 .text.HAL_I2C_Master_Seq_Receive_DMA
                0x00000000      0x1cc Drivers\STM32F2xx_HAL_Driver\Src\stm32f2xx_hal_i2c.o
 .text.HAL_I2C_Slave_Seq_Transmit_IT
                0x00000000       0x7c Drivers\STM32F2xx_HAL_Driver\Src\stm32f2xx_hal_i2c.o
 .text.HAL_I2C_Slave_Seq_Transmit_DMA
                0x00000000      0x144 Drivers\STM32F2xx_HAL_Driver\Src\stm32f2xx_hal_i2c.o
 .text.HAL_I2C_Slave_Seq_Receive_IT
                0x00000000       0x7c Drivers\STM32F2xx_HAL_Driver\Src\stm32f2xx_hal_i2c.o
 .text.HAL_I2C_Slave_Seq_Receive_DMA
                0x00000000      0x144 Drivers\STM32F2xx_HAL_Driver\Src\stm32f2xx_hal_i2c.o
 .text.HAL_I2C_EnableListen_IT
                0x00000000       0x36 Drivers\STM32F2xx_HAL_Driver\Src\stm32f2xx_hal_i2c.o
 .text.HAL_I2C_DisableListen_IT
                0x00000000       0x3e Drivers\STM32F2xx_HAL_Driver\Src\stm32f2xx_hal_i2c.o
 .text.HAL_I2C_MasterTxCpltCallback
                0x00000000        0x2 Drivers\STM32F2xx_HAL_Driver\Src\stm32f2xx_hal_i2c.o
 .text.HAL_I2C_MasterRxCpltCallback
                0x00000000        0x2 Drivers\STM32F2xx_HAL_Driver\Src\stm32f2xx_hal_i2c.o
 .text.HAL_I2C_SlaveTxCpltCallback
                0x00000000        0x2 Drivers\STM32F2xx_HAL_Driver\Src\stm32f2xx_hal_i2c.o
 .text.HAL_I2C_SlaveRxCpltCallback
                0x00000000        0x2 Drivers\STM32F2xx_HAL_Driver\Src\stm32f2xx_hal_i2c.o
 .text.HAL_I2C_AddrCallback
                0x00000000        0x2 Drivers\STM32F2xx_HAL_Driver\Src\stm32f2xx_hal_i2c.o
 .text.HAL_I2C_ListenCpltCallback
                0x00000000        0x2 Drivers\STM32F2xx_HAL_Driver\Src\stm32f2xx_hal_i2c.o
 .text.HAL_I2C_MemTxCpltCallback
                0x00000000        0x2 Drivers\STM32F2xx_HAL_Driver\Src\stm32f2xx_hal_i2c.o
 .text.HAL_I2C_MemRxCpltCallback
                0x00000000        0x2 Drivers\STM32F2xx_HAL_Driver\Src\stm32f2xx_hal_i2c.o
 .text.HAL_I2C_ErrorCallback
                0x00000000        0x2 Drivers\STM32F2xx_HAL_Driver\Src\stm32f2xx_hal_i2c.o
 .text.I2C_DMAError
                0x00000000       0x3c Drivers\STM32F2xx_HAL_Driver\Src\stm32f2xx_hal_i2c.o
 .text.I2C_DMAXferCplt
                0x00000000      0x102 Drivers\STM32F2xx_HAL_Driver\Src\stm32f2xx_hal_i2c.o
 .text.HAL_I2C_AbortCpltCallback
                0x00000000        0x2 Drivers\STM32F2xx_HAL_Driver\Src\stm32f2xx_hal_i2c.o
 .text.I2C_DMAAbort
                0x00000000       0x76 Drivers\STM32F2xx_HAL_Driver\Src\stm32f2xx_hal_i2c.o
 .text.I2C_ITError
                0x00000000      0x144 Drivers\STM32F2xx_HAL_Driver\Src\stm32f2xx_hal_i2c.o
 .text.HAL_I2C_Master_Abort_IT
                0x00000000       0x4c Drivers\STM32F2xx_HAL_Driver\Src\stm32f2xx_hal_i2c.o
 .text.HAL_I2C_EV_IRQHandler
                0x00000000      0x848 Drivers\STM32F2xx_HAL_Driver\Src\stm32f2xx_hal_i2c.o
 .text.HAL_I2C_ER_IRQHandler
                0x00000000      0x12c Drivers\STM32F2xx_HAL_Driver\Src\stm32f2xx_hal_i2c.o
 .text.HAL_I2C_GetState
                0x00000000        0x6 Drivers\STM32F2xx_HAL_Driver\Src\stm32f2xx_hal_i2c.o
 .text.HAL_I2C_GetMode
                0x00000000        0x6 Drivers\STM32F2xx_HAL_Driver\Src\stm32f2xx_hal_i2c.o
 .text.HAL_I2C_GetError
                0x00000000        0x4 Drivers\STM32F2xx_HAL_Driver\Src\stm32f2xx_hal_i2c.o
 .text          0x00000000        0x0 Drivers\STM32F2xx_HAL_Driver\Src\stm32f2xx_hal_pwr.o
 .data          0x00000000        0x0 Drivers\STM32F2xx_HAL_Driver\Src\stm32f2xx_hal_pwr.o
 .bss           0x00000000        0x0 Drivers\STM32F2xx_HAL_Driver\Src\stm32f2xx_hal_pwr.o
 .text.HAL_PWR_DeInit
                0x00000000       0x18 Drivers\STM32F2xx_HAL_Driver\Src\stm32f2xx_hal_pwr.o
 .text.HAL_PWR_EnableBkUpAccess
                0x00000000       0x1c Drivers\STM32F2xx_HAL_Driver\Src\stm32f2xx_hal_pwr.o
 .text.HAL_PWR_DisableBkUpAccess
                0x00000000       0x1c Drivers\STM32F2xx_HAL_Driver\Src\stm32f2xx_hal_pwr.o
 .text.HAL_PWR_ConfigPVD
                0x00000000       0x70 Drivers\STM32F2xx_HAL_Driver\Src\stm32f2xx_hal_pwr.o
 .text.HAL_PWR_EnablePVD
                0x00000000       0x1a Drivers\STM32F2xx_HAL_Driver\Src\stm32f2xx_hal_pwr.o
 .text.HAL_PWR_DisablePVD
                0x00000000       0x1a Drivers\STM32F2xx_HAL_Driver\Src\stm32f2xx_hal_pwr.o
 .text.HAL_PWR_EnableWakeUpPin
                0x00000000       0x10 Drivers\STM32F2xx_HAL_Driver\Src\stm32f2xx_hal_pwr.o
 .text.HAL_PWR_DisableWakeUpPin
                0x00000000       0x10 Drivers\STM32F2xx_HAL_Driver\Src\stm32f2xx_hal_pwr.o
 .text.HAL_PWR_EnterSLEEPMode
                0x00000000       0x20 Drivers\STM32F2xx_HAL_Driver\Src\stm32f2xx_hal_pwr.o
 .text.HAL_PWR_EnterSTOPMode
                0x00000000       0x38 Drivers\STM32F2xx_HAL_Driver\Src\stm32f2xx_hal_pwr.o
 .text.HAL_PWR_EnterSTANDBYMode
                0x00000000       0x20 Drivers\STM32F2xx_HAL_Driver\Src\stm32f2xx_hal_pwr.o
 .text.HAL_PWR_PVDCallback
                0x00000000        0x2 Drivers\STM32F2xx_HAL_Driver\Src\stm32f2xx_hal_pwr.o
 .text.HAL_PWR_PVD_IRQHandler
                0x00000000       0x1c Drivers\STM32F2xx_HAL_Driver\Src\stm32f2xx_hal_pwr.o
 .text.HAL_PWR_EnableSleepOnExit
                0x00000000       0x10 Drivers\STM32F2xx_HAL_Driver\Src\stm32f2xx_hal_pwr.o
 .text.HAL_PWR_DisableSleepOnExit
                0x00000000       0x10 Drivers\STM32F2xx_HAL_Driver\Src\stm32f2xx_hal_pwr.o
 .text.HAL_PWR_EnableSEVOnPend
                0x00000000       0x10 Drivers\STM32F2xx_HAL_Driver\Src\stm32f2xx_hal_pwr.o
 .text.HAL_PWR_DisableSEVOnPend
                0x00000000       0x10 Drivers\STM32F2xx_HAL_Driver\Src\stm32f2xx_hal_pwr.o
 .debug_info    0x00000000      0x852 Drivers\STM32F2xx_HAL_Driver\Src\stm32f2xx_hal_pwr.o
 .debug_abbrev  0x00000000      0x1f5 Drivers\STM32F2xx_HAL_Driver\Src\stm32f2xx_hal_pwr.o
 .debug_loc     0x00000000       0xd8 Drivers\STM32F2xx_HAL_Driver\Src\stm32f2xx_hal_pwr.o
 .debug_aranges
                0x00000000       0xa0 Drivers\STM32F2xx_HAL_Driver\Src\stm32f2xx_hal_pwr.o
 .debug_ranges  0x00000000       0x90 Drivers\STM32F2xx_HAL_Driver\Src\stm32f2xx_hal_pwr.o
 .debug_line    0x00000000      0x39a Drivers\STM32F2xx_HAL_Driver\Src\stm32f2xx_hal_pwr.o
 .debug_str     0x00000000      0x60d Drivers\STM32F2xx_HAL_Driver\Src\stm32f2xx_hal_pwr.o
 .comment       0x00000000       0x7d Drivers\STM32F2xx_HAL_Driver\Src\stm32f2xx_hal_pwr.o
 .debug_frame   0x00000000      0x128 Drivers\STM32F2xx_HAL_Driver\Src\stm32f2xx_hal_pwr.o
 .ARM.attributes
                0x00000000       0x33 Drivers\STM32F2xx_HAL_Driver\Src\stm32f2xx_hal_pwr.o
 .text          0x00000000        0x0 Drivers\STM32F2xx_HAL_Driver\Src\stm32f2xx_hal_pwr_ex.o
 .data          0x00000000        0x0 Drivers\STM32F2xx_HAL_Driver\Src\stm32f2xx_hal_pwr_ex.o
 .bss           0x00000000        0x0 Drivers\STM32F2xx_HAL_Driver\Src\stm32f2xx_hal_pwr_ex.o
 .text.HAL_PWREx_EnableBkUpReg
                0x00000000       0x44 Drivers\STM32F2xx_HAL_Driver\Src\stm32f2xx_hal_pwr_ex.o
 .text.HAL_PWREx_DisableBkUpReg
                0x00000000       0x44 Drivers\STM32F2xx_HAL_Driver\Src\stm32f2xx_hal_pwr_ex.o
 .text.HAL_PWREx_EnableFlashPowerDown
                0x00000000       0x1c Drivers\STM32F2xx_HAL_Driver\Src\stm32f2xx_hal_pwr_ex.o
 .text.HAL_PWREx_DisableFlashPowerDown
                0x00000000       0x1c Drivers\STM32F2xx_HAL_Driver\Src\stm32f2xx_hal_pwr_ex.o
 .debug_info    0x00000000      0x383 Drivers\STM32F2xx_HAL_Driver\Src\stm32f2xx_hal_pwr_ex.o
 .debug_abbrev  0x00000000      0x18a Drivers\STM32F2xx_HAL_Driver\Src\stm32f2xx_hal_pwr_ex.o
 .debug_loc     0x00000000       0x96 Drivers\STM32F2xx_HAL_Driver\Src\stm32f2xx_hal_pwr_ex.o
 .debug_aranges
                0x00000000       0x38 Drivers\STM32F2xx_HAL_Driver\Src\stm32f2xx_hal_pwr_ex.o
 .debug_ranges  0x00000000       0x28 Drivers\STM32F2xx_HAL_Driver\Src\stm32f2xx_hal_pwr_ex.o
 .debug_line    0x00000000      0x2aa Drivers\STM32F2xx_HAL_Driver\Src\stm32f2xx_hal_pwr_ex.o
 .debug_str     0x00000000      0x38e Drivers\STM32F2xx_HAL_Driver\Src\stm32f2xx_hal_pwr_ex.o
 .comment       0x00000000       0x7d Drivers\STM32F2xx_HAL_Driver\Src\stm32f2xx_hal_pwr_ex.o
 .debug_frame   0x00000000       0x68 Drivers\STM32F2xx_HAL_Driver\Src\stm32f2xx_hal_pwr_ex.o
 .ARM.attributes
                0x00000000       0x33 Drivers\STM32F2xx_HAL_Driver\Src\stm32f2xx_hal_pwr_ex.o
 .text          0x00000000        0x0 Drivers\STM32F2xx_HAL_Driver\Src\stm32f2xx_hal_rcc.o
 .data          0x00000000        0x0 Drivers\STM32F2xx_HAL_Driver\Src\stm32f2xx_hal_rcc.o
 .bss           0x00000000        0x0 Drivers\STM32F2xx_HAL_Driver\Src\stm32f2xx_hal_rcc.o
 .text.HAL_RCC_DeInit
                0x00000000       0xfc Drivers\STM32F2xx_HAL_Driver\Src\stm32f2xx_hal_rcc.o
 .text.HAL_RCC_MCOConfig
                0x00000000       0x98 Drivers\STM32F2xx_HAL_Driver\Src\stm32f2xx_hal_rcc.o
 .text.HAL_RCC_EnableCSS
                0x00000000        0xc Drivers\STM32F2xx_HAL_Driver\Src\stm32f2xx_hal_rcc.o
 .text.HAL_RCC_DisableCSS
                0x00000000        0xc Drivers\STM32F2xx_HAL_Driver\Src\stm32f2xx_hal_rcc.o
 .text.HAL_RCC_GetHCLKFreq
                0x00000000        0xc Drivers\STM32F2xx_HAL_Driver\Src\stm32f2xx_hal_rcc.o
 .text.HAL_RCC_GetOscConfig
                0x00000000       0xcc Drivers\STM32F2xx_HAL_Driver\Src\stm32f2xx_hal_rcc.o
 .text.HAL_RCC_GetClockConfig
                0x00000000       0x3c Drivers\STM32F2xx_HAL_Driver\Src\stm32f2xx_hal_rcc.o
 .text.HAL_RCC_CSSCallback
                0x00000000        0x2 Drivers\STM32F2xx_HAL_Driver\Src\stm32f2xx_hal_rcc.o
 .text.HAL_RCC_NMI_IRQHandler
                0x00000000       0x20 Drivers\STM32F2xx_HAL_Driver\Src\stm32f2xx_hal_rcc.o
 .text          0x00000000        0x0 Drivers\STM32F2xx_HAL_Driver\Src\stm32f2xx_hal_rcc_ex.o
 .data          0x00000000        0x0 Drivers\STM32F2xx_HAL_Driver\Src\stm32f2xx_hal_rcc_ex.o
 .bss           0x00000000        0x0 Drivers\STM32F2xx_HAL_Driver\Src\stm32f2xx_hal_rcc_ex.o
 .text.HAL_RCCEx_PeriphCLKConfig
                0x00000000      0x14c Drivers\STM32F2xx_HAL_Driver\Src\stm32f2xx_hal_rcc_ex.o
 .text.HAL_RCCEx_GetPeriphCLKConfig
                0x00000000       0x4c Drivers\STM32F2xx_HAL_Driver\Src\stm32f2xx_hal_rcc_ex.o
 .debug_info    0x00000000      0x5db Drivers\STM32F2xx_HAL_Driver\Src\stm32f2xx_hal_rcc_ex.o
 .debug_abbrev  0x00000000      0x20c Drivers\STM32F2xx_HAL_Driver\Src\stm32f2xx_hal_rcc_ex.o
 .debug_loc     0x00000000      0x17e Drivers\STM32F2xx_HAL_Driver\Src\stm32f2xx_hal_rcc_ex.o
 .debug_aranges
                0x00000000       0x28 Drivers\STM32F2xx_HAL_Driver\Src\stm32f2xx_hal_rcc_ex.o
 .debug_ranges  0x00000000       0x48 Drivers\STM32F2xx_HAL_Driver\Src\stm32f2xx_hal_rcc_ex.o
 .debug_line    0x00000000      0x2f9 Drivers\STM32F2xx_HAL_Driver\Src\stm32f2xx_hal_rcc_ex.o
 .debug_str     0x00000000      0x4f4 Drivers\STM32F2xx_HAL_Driver\Src\stm32f2xx_hal_rcc_ex.o
 .comment       0x00000000       0x7d Drivers\STM32F2xx_HAL_Driver\Src\stm32f2xx_hal_rcc_ex.o
 .debug_frame   0x00000000       0x4c Drivers\STM32F2xx_HAL_Driver\Src\stm32f2xx_hal_rcc_ex.o
 .ARM.attributes
                0x00000000       0x33 Drivers\STM32F2xx_HAL_Driver\Src\stm32f2xx_hal_rcc_ex.o
 .text          0x00000000        0x0 Drivers\STM32F2xx_HAL_Driver\Src\stm32f2xx_hal_tim.o
 .data          0x00000000        0x0 Drivers\STM32F2xx_HAL_Driver\Src\stm32f2xx_hal_tim.o
 .bss           0x00000000        0x0 Drivers\STM32F2xx_HAL_Driver\Src\stm32f2xx_hal_tim.o
 .text.TIM_OC1_SetConfig
                0x00000000       0x64 Drivers\STM32F2xx_HAL_Driver\Src\stm32f2xx_hal_tim.o
 .text.TIM_OC3_SetConfig
                0x00000000       0x6c Drivers\STM32F2xx_HAL_Driver\Src\stm32f2xx_hal_tim.o
 .text.TIM_OC4_SetConfig
                0x00000000       0x4c Drivers\STM32F2xx_HAL_Driver\Src\stm32f2xx_hal_tim.o
 .text.HAL_TIM_Base_MspInit
                0x00000000        0x2 Drivers\STM32F2xx_HAL_Driver\Src\stm32f2xx_hal_tim.o
 .text.HAL_TIM_Base_MspDeInit
                0x00000000        0x2 Drivers\STM32F2xx_HAL_Driver\Src\stm32f2xx_hal_tim.o
 .text.HAL_TIM_Base_DeInit
                0x00000000       0x3a Drivers\STM32F2xx_HAL_Driver\Src\stm32f2xx_hal_tim.o
 .text.HAL_TIM_Base_Start
                0x00000000       0x24 Drivers\STM32F2xx_HAL_Driver\Src\stm32f2xx_hal_tim.o
 .text.HAL_TIM_Base_Stop
                0x00000000       0x2e Drivers\STM32F2xx_HAL_Driver\Src\stm32f2xx_hal_tim.o
 .text.HAL_TIM_Base_Stop_IT
                0x00000000       0x2a Drivers\STM32F2xx_HAL_Driver\Src\stm32f2xx_hal_tim.o
 .text.HAL_TIM_Base_Start_DMA
                0x00000000       0x6c Drivers\STM32F2xx_HAL_Driver\Src\stm32f2xx_hal_tim.o
 .text.HAL_TIM_Base_Stop_DMA
                0x00000000       0x3c Drivers\STM32F2xx_HAL_Driver\Src\stm32f2xx_hal_tim.o
 .text.HAL_TIM_OC_MspInit
                0x00000000        0x2 Drivers\STM32F2xx_HAL_Driver\Src\stm32f2xx_hal_tim.o
 .text.HAL_TIM_OC_MspDeInit
                0x00000000        0x2 Drivers\STM32F2xx_HAL_Driver\Src\stm32f2xx_hal_tim.o
 .text.HAL_TIM_OC_DeInit
                0x00000000       0x3a Drivers\STM32F2xx_HAL_Driver\Src\stm32f2xx_hal_tim.o
 .text.HAL_TIM_PWM_MspInit
                0x00000000        0x2 Drivers\STM32F2xx_HAL_Driver\Src\stm32f2xx_hal_tim.o
 .text.HAL_TIM_PWM_MspDeInit
                0x00000000        0x2 Drivers\STM32F2xx_HAL_Driver\Src\stm32f2xx_hal_tim.o
 .text.HAL_TIM_PWM_DeInit
                0x00000000       0x3a Drivers\STM32F2xx_HAL_Driver\Src\stm32f2xx_hal_tim.o
 .text.HAL_TIM_IC_MspInit
                0x00000000        0x2 Drivers\STM32F2xx_HAL_Driver\Src\stm32f2xx_hal_tim.o
 .text.HAL_TIM_IC_MspDeInit
                0x00000000        0x2 Drivers\STM32F2xx_HAL_Driver\Src\stm32f2xx_hal_tim.o
 .text.HAL_TIM_IC_DeInit
                0x00000000       0x3a Drivers\STM32F2xx_HAL_Driver\Src\stm32f2xx_hal_tim.o
 .text.HAL_TIM_OnePulse_MspInit
                0x00000000        0x2 Drivers\STM32F2xx_HAL_Driver\Src\stm32f2xx_hal_tim.o
 .text.HAL_TIM_OnePulse_MspDeInit
                0x00000000        0x2 Drivers\STM32F2xx_HAL_Driver\Src\stm32f2xx_hal_tim.o
 .text.HAL_TIM_OnePulse_DeInit
                0x00000000       0x3a Drivers\STM32F2xx_HAL_Driver\Src\stm32f2xx_hal_tim.o
 .text.HAL_TIM_OnePulse_Start
                0x00000000       0x40 Drivers\STM32F2xx_HAL_Driver\Src\stm32f2xx_hal_tim.o
 .text.HAL_TIM_OnePulse_Stop
                0x00000000       0x68 Drivers\STM32F2xx_HAL_Driver\Src\stm32f2xx_hal_tim.o
 .text.HAL_TIM_OnePulse_Start_IT
                0x00000000       0x50 Drivers\STM32F2xx_HAL_Driver\Src\stm32f2xx_hal_tim.o
 .text.HAL_TIM_OnePulse_Stop_IT
                0x00000000       0x78 Drivers\STM32F2xx_HAL_Driver\Src\stm32f2xx_hal_tim.o
 .text.HAL_TIM_Encoder_MspInit
                0x00000000        0x2 Drivers\STM32F2xx_HAL_Driver\Src\stm32f2xx_hal_tim.o
 .text.HAL_TIM_Encoder_MspDeInit
                0x00000000        0x2 Drivers\STM32F2xx_HAL_Driver\Src\stm32f2xx_hal_tim.o
 .text.HAL_TIM_Encoder_DeInit
                0x00000000       0x3a Drivers\STM32F2xx_HAL_Driver\Src\stm32f2xx_hal_tim.o
 .text.HAL_TIM_Encoder_Start
                0x00000000       0x44 Drivers\STM32F2xx_HAL_Driver\Src\stm32f2xx_hal_tim.o
 .text.HAL_TIM_Encoder_Stop
                0x00000000       0x48 Drivers\STM32F2xx_HAL_Driver\Src\stm32f2xx_hal_tim.o
 .text.HAL_TIM_Encoder_Start_IT
                0x00000000       0x6e Drivers\STM32F2xx_HAL_Driver\Src\stm32f2xx_hal_tim.o
 .text.HAL_TIM_Encoder_Stop_IT
                0x00000000       0x74 Drivers\STM32F2xx_HAL_Driver\Src\stm32f2xx_hal_tim.o
 .text.HAL_TIM_Encoder_Start_DMA
                0x00000000      0x150 Drivers\STM32F2xx_HAL_Driver\Src\stm32f2xx_hal_tim.o
 .text.HAL_TIM_Encoder_Stop_DMA
                0x00000000       0x92 Drivers\STM32F2xx_HAL_Driver\Src\stm32f2xx_hal_tim.o
 .text.HAL_TIM_DMABurst_WriteStart
                0x00000000       0xdc Drivers\STM32F2xx_HAL_Driver\Src\stm32f2xx_hal_tim.o
 .text.HAL_TIM_DMABurst_ReadStart
                0x00000000       0xdc Drivers\STM32F2xx_HAL_Driver\Src\stm32f2xx_hal_tim.o
 .text.HAL_TIM_DMABurst_ReadStop
                0x00000000       0x60 Drivers\STM32F2xx_HAL_Driver\Src\stm32f2xx_hal_tim.o
 .text.HAL_TIM_DMABurst_WriteStop
                0x00000000        0x4 Drivers\STM32F2xx_HAL_Driver\Src\stm32f2xx_hal_tim.o
 .text.HAL_TIM_GenerateEvent
                0x00000000       0x24 Drivers\STM32F2xx_HAL_Driver\Src\stm32f2xx_hal_tim.o
 .text.HAL_TIM_ConfigTI1Input
                0x00000000       0x10 Drivers\STM32F2xx_HAL_Driver\Src\stm32f2xx_hal_tim.o
 .text.HAL_TIM_ReadCapturedValue
                0x00000000       0x32 Drivers\STM32F2xx_HAL_Driver\Src\stm32f2xx_hal_tim.o
 .text.HAL_TIM_PeriodElapsedCallback
                0x00000000        0x2 Drivers\STM32F2xx_HAL_Driver\Src\stm32f2xx_hal_tim.o
 .text.TIM_DMAPeriodElapsedCplt
                0x00000000       0x10 Drivers\STM32F2xx_HAL_Driver\Src\stm32f2xx_hal_tim.o
 .text.HAL_TIM_PeriodElapsedHalfCpltCallback
                0x00000000        0x2 Drivers\STM32F2xx_HAL_Driver\Src\stm32f2xx_hal_tim.o
 .text.TIM_DMAPeriodElapsedHalfCplt
                0x00000000       0x10 Drivers\STM32F2xx_HAL_Driver\Src\stm32f2xx_hal_tim.o
 .text.TIM_DMACaptureCplt
                0x00000000       0x3c Drivers\STM32F2xx_HAL_Driver\Src\stm32f2xx_hal_tim.o
 .text.HAL_TIM_IC_CaptureHalfCpltCallback
                0x00000000        0x2 Drivers\STM32F2xx_HAL_Driver\Src\stm32f2xx_hal_tim.o
 .text.TIM_DMACaptureHalfCplt
                0x00000000       0x3c Drivers\STM32F2xx_HAL_Driver\Src\stm32f2xx_hal_tim.o
 .text.TIM_DMADelayPulseCplt
                0x00000000       0x3c Drivers\STM32F2xx_HAL_Driver\Src\stm32f2xx_hal_tim.o
 .text.HAL_TIM_PWM_PulseFinishedHalfCpltCallback
                0x00000000        0x2 Drivers\STM32F2xx_HAL_Driver\Src\stm32f2xx_hal_tim.o
 .text.TIM_DMADelayPulseHalfCplt
                0x00000000       0x3c Drivers\STM32F2xx_HAL_Driver\Src\stm32f2xx_hal_tim.o
 .text.TIM_DMATriggerCplt
                0x00000000       0x10 Drivers\STM32F2xx_HAL_Driver\Src\stm32f2xx_hal_tim.o
 .text.HAL_TIM_TriggerHalfCpltCallback
                0x00000000        0x2 Drivers\STM32F2xx_HAL_Driver\Src\stm32f2xx_hal_tim.o
 .text.TIM_DMATriggerHalfCplt
                0x00000000       0x10 Drivers\STM32F2xx_HAL_Driver\Src\stm32f2xx_hal_tim.o
 .text.HAL_TIM_ErrorCallback
                0x00000000        0x2 Drivers\STM32F2xx_HAL_Driver\Src\stm32f2xx_hal_tim.o
 .text.TIM_DMAError
                0x00000000       0x10 Drivers\STM32F2xx_HAL_Driver\Src\stm32f2xx_hal_tim.o
 .text.HAL_TIM_Base_GetState
                0x00000000        0x6 Drivers\STM32F2xx_HAL_Driver\Src\stm32f2xx_hal_tim.o
 .text.HAL_TIM_OC_GetState
                0x00000000        0x6 Drivers\STM32F2xx_HAL_Driver\Src\stm32f2xx_hal_tim.o
 .text.HAL_TIM_PWM_GetState
                0x00000000        0x6 Drivers\STM32F2xx_HAL_Driver\Src\stm32f2xx_hal_tim.o
 .text.HAL_TIM_IC_GetState
                0x00000000        0x6 Drivers\STM32F2xx_HAL_Driver\Src\stm32f2xx_hal_tim.o
 .text.HAL_TIM_OnePulse_GetState
                0x00000000        0x6 Drivers\STM32F2xx_HAL_Driver\Src\stm32f2xx_hal_tim.o
 .text.HAL_TIM_Encoder_GetState
                0x00000000        0x6 Drivers\STM32F2xx_HAL_Driver\Src\stm32f2xx_hal_tim.o
 .text.HAL_TIM_OC_Init
                0x00000000       0x34 Drivers\STM32F2xx_HAL_Driver\Src\stm32f2xx_hal_tim.o
 .text.HAL_TIM_PWM_Init
                0x00000000       0x34 Drivers\STM32F2xx_HAL_Driver\Src\stm32f2xx_hal_tim.o
 .text.HAL_TIM_IC_Init
                0x00000000       0x34 Drivers\STM32F2xx_HAL_Driver\Src\stm32f2xx_hal_tim.o
 .text.HAL_TIM_OnePulse_Init
                0x00000000       0x46 Drivers\STM32F2xx_HAL_Driver\Src\stm32f2xx_hal_tim.o
 .text.HAL_TIM_Encoder_Init
                0x00000000       0x96 Drivers\STM32F2xx_HAL_Driver\Src\stm32f2xx_hal_tim.o
 .text.TIM_OC2_SetConfig
                0x00000000       0x6c Drivers\STM32F2xx_HAL_Driver\Src\stm32f2xx_hal_tim.o
 .text.HAL_TIM_OC_ConfigChannel
                0x00000000       0x5c Drivers\STM32F2xx_HAL_Driver\Src\stm32f2xx_hal_tim.o
 .text.HAL_TIM_PWM_ConfigChannel
                0x00000000       0xc4 Drivers\STM32F2xx_HAL_Driver\Src\stm32f2xx_hal_tim.o
 .text.TIM_TI1_SetConfig
                0x00000000       0x74 Drivers\STM32F2xx_HAL_Driver\Src\stm32f2xx_hal_tim.o
 .text.HAL_TIM_IC_ConfigChannel
                0x00000000      0x110 Drivers\STM32F2xx_HAL_Driver\Src\stm32f2xx_hal_tim.o
 .text.HAL_TIM_OnePulse_ConfigChannel
                0x00000000       0xf4 Drivers\STM32F2xx_HAL_Driver\Src\stm32f2xx_hal_tim.o
 .text.TIM_ETR_SetConfig
                0x00000000       0x14 Drivers\STM32F2xx_HAL_Driver\Src\stm32f2xx_hal_tim.o
 .text.HAL_TIM_ConfigOCrefClear
                0x00000000       0xcc Drivers\STM32F2xx_HAL_Driver\Src\stm32f2xx_hal_tim.o
 .text.HAL_TIM_ConfigClockSource
                0x00000000      0x128 Drivers\STM32F2xx_HAL_Driver\Src\stm32f2xx_hal_tim.o
 .text.TIM_SlaveTimer_SetConfig
                0x00000000       0xa4 Drivers\STM32F2xx_HAL_Driver\Src\stm32f2xx_hal_tim.o
 .text.HAL_TIM_SlaveConfigSynchro
                0x00000000       0x4e Drivers\STM32F2xx_HAL_Driver\Src\stm32f2xx_hal_tim.o
 .text.HAL_TIM_SlaveConfigSynchro_IT
                0x00000000       0x4e Drivers\STM32F2xx_HAL_Driver\Src\stm32f2xx_hal_tim.o
 .text.TIM_CCxChannelCmd
                0x00000000       0x1c Drivers\STM32F2xx_HAL_Driver\Src\stm32f2xx_hal_tim.o
 .text.HAL_TIM_OC_Stop
                0x00000000       0x5c Drivers\STM32F2xx_HAL_Driver\Src\stm32f2xx_hal_tim.o
 .text.HAL_TIM_PWM_Start
                0x00000000       0x40 Drivers\STM32F2xx_HAL_Driver\Src\stm32f2xx_hal_tim.o
 .text.HAL_TIM_OC_Start
                0x00000000        0x4 Drivers\STM32F2xx_HAL_Driver\Src\stm32f2xx_hal_tim.o
 .text.HAL_TIM_PWM_Stop
                0x00000000       0x64 Drivers\STM32F2xx_HAL_Driver\Src\stm32f2xx_hal_tim.o
 .text.HAL_TIM_PWM_Start_IT
                0x00000000       0x80 Drivers\STM32F2xx_HAL_Driver\Src\stm32f2xx_hal_tim.o
 .text.HAL_TIM_OC_Start_IT
                0x00000000        0x4 Drivers\STM32F2xx_HAL_Driver\Src\stm32f2xx_hal_tim.o
 .text.HAL_TIM_PWM_Stop_IT
                0x00000000       0x9c Drivers\STM32F2xx_HAL_Driver\Src\stm32f2xx_hal_tim.o
 .text.HAL_TIM_OC_Stop_IT
                0x00000000        0x4 Drivers\STM32F2xx_HAL_Driver\Src\stm32f2xx_hal_tim.o
 .text.HAL_TIM_PWM_Start_DMA
                0x00000000      0x11c Drivers\STM32F2xx_HAL_Driver\Src\stm32f2xx_hal_tim.o
 .text.HAL_TIM_OC_Start_DMA
                0x00000000        0x4 Drivers\STM32F2xx_HAL_Driver\Src\stm32f2xx_hal_tim.o
 .text.HAL_TIM_PWM_Stop_DMA
                0x00000000       0xb8 Drivers\STM32F2xx_HAL_Driver\Src\stm32f2xx_hal_tim.o
 .text.HAL_TIM_OC_Stop_DMA
                0x00000000        0x4 Drivers\STM32F2xx_HAL_Driver\Src\stm32f2xx_hal_tim.o
 .text.HAL_TIM_IC_Start
                0x00000000       0x24 Drivers\STM32F2xx_HAL_Driver\Src\stm32f2xx_hal_tim.o
 .text.HAL_TIM_IC_Stop
                0x00000000       0x2e Drivers\STM32F2xx_HAL_Driver\Src\stm32f2xx_hal_tim.o
 .text.HAL_TIM_IC_Start_IT
                0x00000000       0x62 Drivers\STM32F2xx_HAL_Driver\Src\stm32f2xx_hal_tim.o
 .text.HAL_TIM_IC_Stop_IT
                0x00000000       0x6c Drivers\STM32F2xx_HAL_Driver\Src\stm32f2xx_hal_tim.o
 .text.HAL_TIM_IC_Start_DMA
                0x00000000       0xfc Drivers\STM32F2xx_HAL_Driver\Src\stm32f2xx_hal_tim.o
 .text.HAL_TIM_IC_Stop_DMA
                0x00000000       0x88 Drivers\STM32F2xx_HAL_Driver\Src\stm32f2xx_hal_tim.o
 .text          0x00000000        0x0 Drivers\STM32F2xx_HAL_Driver\Src\stm32f2xx_hal_tim_ex.o
 .data          0x00000000        0x0 Drivers\STM32F2xx_HAL_Driver\Src\stm32f2xx_hal_tim_ex.o
 .bss           0x00000000        0x0 Drivers\STM32F2xx_HAL_Driver\Src\stm32f2xx_hal_tim_ex.o
 .text.TIM_CCxNChannelCmd
                0x00000000       0x1c Drivers\STM32F2xx_HAL_Driver\Src\stm32f2xx_hal_tim_ex.o
 .text.HAL_TIMEx_HallSensor_MspInit
                0x00000000        0x2 Drivers\STM32F2xx_HAL_Driver\Src\stm32f2xx_hal_tim_ex.o
 .text.HAL_TIMEx_HallSensor_Init
                0x00000000       0xae Drivers\STM32F2xx_HAL_Driver\Src\stm32f2xx_hal_tim_ex.o
 .text.HAL_TIMEx_HallSensor_MspDeInit
                0x00000000        0x2 Drivers\STM32F2xx_HAL_Driver\Src\stm32f2xx_hal_tim_ex.o
 .text.HAL_TIMEx_HallSensor_DeInit
                0x00000000       0x3a Drivers\STM32F2xx_HAL_Driver\Src\stm32f2xx_hal_tim_ex.o
 .text.HAL_TIMEx_HallSensor_Start
                0x00000000       0x26 Drivers\STM32F2xx_HAL_Driver\Src\stm32f2xx_hal_tim_ex.o
 .text.HAL_TIMEx_HallSensor_Stop
                0x00000000       0x30 Drivers\STM32F2xx_HAL_Driver\Src\stm32f2xx_hal_tim_ex.o
 .text.HAL_TIMEx_HallSensor_Start_IT
                0x00000000       0x2e Drivers\STM32F2xx_HAL_Driver\Src\stm32f2xx_hal_tim_ex.o
 .text.HAL_TIMEx_HallSensor_Stop_IT
                0x00000000       0x38 Drivers\STM32F2xx_HAL_Driver\Src\stm32f2xx_hal_tim_ex.o
 .text.HAL_TIMEx_HallSensor_Start_DMA
                0x00000000       0x7c Drivers\STM32F2xx_HAL_Driver\Src\stm32f2xx_hal_tim_ex.o
 .text.HAL_TIMEx_HallSensor_Stop_DMA
                0x00000000       0x40 Drivers\STM32F2xx_HAL_Driver\Src\stm32f2xx_hal_tim_ex.o
 .text.HAL_TIMEx_PWMN_Start
                0x00000000       0x2c Drivers\STM32F2xx_HAL_Driver\Src\stm32f2xx_hal_tim_ex.o
 .text.HAL_TIMEx_OCN_Start
                0x00000000        0x4 Drivers\STM32F2xx_HAL_Driver\Src\stm32f2xx_hal_tim_ex.o
 .text.HAL_TIMEx_PWMN_Start_IT
                0x00000000       0x56 Drivers\STM32F2xx_HAL_Driver\Src\stm32f2xx_hal_tim_ex.o
 .text.HAL_TIMEx_OCN_Start_IT
                0x00000000        0x4 Drivers\STM32F2xx_HAL_Driver\Src\stm32f2xx_hal_tim_ex.o
 .text.HAL_TIMEx_PWMN_Stop_IT
                0x00000000       0x84 Drivers\STM32F2xx_HAL_Driver\Src\stm32f2xx_hal_tim_ex.o
 .text.HAL_TIMEx_OCN_Stop_IT
                0x00000000        0x4 Drivers\STM32F2xx_HAL_Driver\Src\stm32f2xx_hal_tim_ex.o
 .text.HAL_TIMEx_PWMN_Start_DMA
                0x00000000       0xd4 Drivers\STM32F2xx_HAL_Driver\Src\stm32f2xx_hal_tim_ex.o
 .text.HAL_TIMEx_OCN_Start_DMA
                0x00000000        0x4 Drivers\STM32F2xx_HAL_Driver\Src\stm32f2xx_hal_tim_ex.o
 .text.HAL_TIMEx_PWMN_Stop_DMA
                0x00000000       0x8a Drivers\STM32F2xx_HAL_Driver\Src\stm32f2xx_hal_tim_ex.o
 .text.HAL_TIMEx_OCN_Stop_DMA
                0x00000000        0x4 Drivers\STM32F2xx_HAL_Driver\Src\stm32f2xx_hal_tim_ex.o
 .text.HAL_TIMEx_OnePulseN_Start
                0x00000000       0x1a Drivers\STM32F2xx_HAL_Driver\Src\stm32f2xx_hal_tim_ex.o
 .text.HAL_TIMEx_OnePulseN_Stop
                0x00000000       0x4a Drivers\STM32F2xx_HAL_Driver\Src\stm32f2xx_hal_tim_ex.o
 .text.HAL_TIMEx_PWMN_Stop
                0x00000000        0x4 Drivers\STM32F2xx_HAL_Driver\Src\stm32f2xx_hal_tim_ex.o
 .text.HAL_TIMEx_OCN_Stop
                0x00000000        0x4 Drivers\STM32F2xx_HAL_Driver\Src\stm32f2xx_hal_tim_ex.o
 .text.HAL_TIMEx_OnePulseN_Start_IT
                0x00000000       0x2a Drivers\STM32F2xx_HAL_Driver\Src\stm32f2xx_hal_tim_ex.o
 .text.HAL_TIMEx_OnePulseN_Stop_IT
                0x00000000       0x5a Drivers\STM32F2xx_HAL_Driver\Src\stm32f2xx_hal_tim_ex.o
 .text.HAL_TIMEx_ConfigCommutEvent
                0x00000000       0x5a Drivers\STM32F2xx_HAL_Driver\Src\stm32f2xx_hal_tim_ex.o
 .text.HAL_TIMEx_ConfigCommutEvent_IT
                0x00000000       0x5a Drivers\STM32F2xx_HAL_Driver\Src\stm32f2xx_hal_tim_ex.o
 .text.HAL_TIMEx_ConfigCommutEvent_DMA
                0x00000000       0x74 Drivers\STM32F2xx_HAL_Driver\Src\stm32f2xx_hal_tim_ex.o
 .text.HAL_TIMEx_ConfigBreakDeadTime
                0x00000000       0x4c Drivers\STM32F2xx_HAL_Driver\Src\stm32f2xx_hal_tim_ex.o
 .text.HAL_TIMEx_RemapConfig
                0x00000000       0x1a Drivers\STM32F2xx_HAL_Driver\Src\stm32f2xx_hal_tim_ex.o
 .text.TIMEx_DMACommutationCplt
                0x00000000       0x10 Drivers\STM32F2xx_HAL_Driver\Src\stm32f2xx_hal_tim_ex.o
 .text.HAL_TIMEx_CommutHalfCpltCallback
                0x00000000        0x2 Drivers\STM32F2xx_HAL_Driver\Src\stm32f2xx_hal_tim_ex.o
 .text.TIMEx_DMACommutationHalfCplt
                0x00000000       0x10 Drivers\STM32F2xx_HAL_Driver\Src\stm32f2xx_hal_tim_ex.o
 .text.HAL_TIMEx_HallSensor_GetState
                0x00000000        0x6 Drivers\STM32F2xx_HAL_Driver\Src\stm32f2xx_hal_tim_ex.o
 .text          0x00000000        0x0 Drivers\STM32F2xx_HAL_Driver\Src\stm32f2xx_hal_uart.o
 .data          0x00000000        0x0 Drivers\STM32F2xx_HAL_Driver\Src\stm32f2xx_hal_uart.o
 .bss           0x00000000        0x0 Drivers\STM32F2xx_HAL_Driver\Src\stm32f2xx_hal_uart.o
 .text.HAL_UART_MspInit
                0x00000000        0x2 Drivers\STM32F2xx_HAL_Driver\Src\stm32f2xx_hal_uart.o
 .text.HAL_HalfDuplex_Init
                0x00000000       0x64 Drivers\STM32F2xx_HAL_Driver\Src\stm32f2xx_hal_uart.o
 .text.HAL_LIN_Init
                0x00000000       0x76 Drivers\STM32F2xx_HAL_Driver\Src\stm32f2xx_hal_uart.o
 .text.HAL_MultiProcessor_Init
                0x00000000       0x7e Drivers\STM32F2xx_HAL_Driver\Src\stm32f2xx_hal_uart.o
 .text.HAL_UART_MspDeInit
                0x00000000        0x2 Drivers\STM32F2xx_HAL_Driver\Src\stm32f2xx_hal_uart.o
 .text.HAL_UART_DeInit
                0x00000000       0x30 Drivers\STM32F2xx_HAL_Driver\Src\stm32f2xx_hal_uart.o
 .text.HAL_UART_Receive
                0x00000000       0xbe Drivers\STM32F2xx_HAL_Driver\Src\stm32f2xx_hal_uart.o
 .text.HAL_UART_Transmit_IT
                0x00000000       0x3e Drivers\STM32F2xx_HAL_Driver\Src\stm32f2xx_hal_uart.o
 .text.HAL_UART_Receive_IT
                0x00000000       0x4e Drivers\STM32F2xx_HAL_Driver\Src\stm32f2xx_hal_uart.o
 .text.HAL_UART_DMAPause
                0x00000000       0x5a Drivers\STM32F2xx_HAL_Driver\Src\stm32f2xx_hal_uart.o
 .text.HAL_UART_DMAResume
                0x00000000       0x62 Drivers\STM32F2xx_HAL_Driver\Src\stm32f2xx_hal_uart.o
 .text.HAL_UART_DMAStop
                0x00000000       0x5e Drivers\STM32F2xx_HAL_Driver\Src\stm32f2xx_hal_uart.o
 .text.HAL_UART_Abort
                0x00000000       0x80 Drivers\STM32F2xx_HAL_Driver\Src\stm32f2xx_hal_uart.o
 .text.HAL_UART_AbortTransmit
                0x00000000       0x48 Drivers\STM32F2xx_HAL_Driver\Src\stm32f2xx_hal_uart.o
 .text.HAL_UART_AbortReceive
                0x00000000       0x50 Drivers\STM32F2xx_HAL_Driver\Src\stm32f2xx_hal_uart.o
 .text.HAL_UART_RxCpltCallback
                0x00000000        0x2 Drivers\STM32F2xx_HAL_Driver\Src\stm32f2xx_hal_uart.o
 .text.HAL_UART_AbortCpltCallback
                0x00000000        0x2 Drivers\STM32F2xx_HAL_Driver\Src\stm32f2xx_hal_uart.o
 .text.HAL_UART_Abort_IT
                0x00000000       0xa8 Drivers\STM32F2xx_HAL_Driver\Src\stm32f2xx_hal_uart.o
 .text.UART_DMARxAbortCallback
                0x00000000       0x28 Drivers\STM32F2xx_HAL_Driver\Src\stm32f2xx_hal_uart.o
 .text.UART_DMATxAbortCallback
                0x00000000       0x28 Drivers\STM32F2xx_HAL_Driver\Src\stm32f2xx_hal_uart.o
 .text.HAL_UART_AbortTransmitCpltCallback
                0x00000000        0x2 Drivers\STM32F2xx_HAL_Driver\Src\stm32f2xx_hal_uart.o
 .text.HAL_UART_AbortTransmit_IT
                0x00000000       0x50 Drivers\STM32F2xx_HAL_Driver\Src\stm32f2xx_hal_uart.o
 .text.UART_DMATxOnlyAbortCallback
                0x00000000       0x14 Drivers\STM32F2xx_HAL_Driver\Src\stm32f2xx_hal_uart.o
 .text.HAL_UART_AbortReceiveCpltCallback
                0x00000000        0x2 Drivers\STM32F2xx_HAL_Driver\Src\stm32f2xx_hal_uart.o
 .text.HAL_UART_AbortReceive_IT
                0x00000000       0x58 Drivers\STM32F2xx_HAL_Driver\Src\stm32f2xx_hal_uart.o
 .text.UART_DMARxOnlyAbortCallback
                0x00000000       0x14 Drivers\STM32F2xx_HAL_Driver\Src\stm32f2xx_hal_uart.o
 .text.HAL_LIN_SendBreak
                0x00000000       0x2c Drivers\STM32F2xx_HAL_Driver\Src\stm32f2xx_hal_uart.o
 .text.HAL_MultiProcessor_EnterMuteMode
                0x00000000       0x2c Drivers\STM32F2xx_HAL_Driver\Src\stm32f2xx_hal_uart.o
 .text.HAL_MultiProcessor_ExitMuteMode
                0x00000000       0x2c Drivers\STM32F2xx_HAL_Driver\Src\stm32f2xx_hal_uart.o
 .text.HAL_HalfDuplex_EnableTransmitter
                0x00000000       0x30 Drivers\STM32F2xx_HAL_Driver\Src\stm32f2xx_hal_uart.o
 .text.HAL_HalfDuplex_EnableReceiver
                0x00000000       0x30 Drivers\STM32F2xx_HAL_Driver\Src\stm32f2xx_hal_uart.o
 .text.HAL_UART_GetState
                0x00000000        0xc Drivers\STM32F2xx_HAL_Driver\Src\stm32f2xx_hal_uart.o
 .text.HAL_UART_GetError
                0x00000000        0x4 Drivers\STM32F2xx_HAL_Driver\Src\stm32f2xx_hal_uart.o
 .text          0x00000000        0x0 Src\Character_lcd.o
 .data          0x00000000        0x0 Src\Character_lcd.o
 .bss           0x00000000        0x0 Src\Character_lcd.o
 .text.LCD_Button_Read
                0x00000000       0xc4 Src\Character_lcd.o
 .text.Layer_Set
                0x00000000        0xc Src\Character_lcd.o
 .text.CharacterLCD_ButtonSetFunc
                0x00000000        0xc Src\Character_lcd.o
 .text.CharacterLCD_ButtonGetFunc
                0x00000000        0xc Src\Character_lcd.o
 .data.prev_layer
                0x00000000        0x1 Src\Character_lcd.o
 .text          0x00000000        0x0 Src\atten_ctrl.o
 .data          0x00000000        0x0 Src\atten_ctrl.o
 .bss           0x00000000        0x0 Src\atten_ctrl.o
 .text.Atten_Offset_Calc
                0x00000000       0x86 Src\atten_ctrl.o
 .text.Atten_Table_Read
                0x00000000       0x5c Src\atten_ctrl.o
 .bss.printf_if
                0x00000000        0x1 Src\atten_ctrl.o
 .text          0x00000000        0x0 Src\eeprom.o
 .data          0x00000000        0x0 Src\eeprom.o
 .bss           0x00000000        0x0 Src\eeprom.o
 .text          0x00000000        0x0 Src\main.o
 .data          0x00000000        0x0 Src\main.o
 .bss           0x00000000        0x0 Src\main.o
 .text.buttonChatteringset
                0x00000000        0xc Src\main.o
 .text.buttonChatteringget
                0x00000000        0xc Src\main.o
 .text.Atten_ButtonPressSet
                0x00000000        0xc Src\main.o
 .text.Atten_ButtonPressGet
                0x00000000        0xc Src\main.o
 .text.Atten_ButtonUnPressSet
                0x00000000        0xc Src\main.o
 .text.Atten_ButtonUnPressGet
                0x00000000        0xc Src\main.o
 .text.UartDataRecvSet
                0x00000000        0xc Src\main.o
 .text.UartDataRecvGet
                0x00000000        0xc Src\main.o
 .bss.ButtonNext_TimerCnt
                0x00000000        0x4 Src\main.o
 .bss.ButtonPressed
                0x00000000        0x1 Src\main.o
 .bss.chattering
                0x00000000        0x1 Src\main.o
 .bss.switchcnt
                0x00000000        0x5 Src\main.o
 .text          0x00000000        0x0 Src\sth30_crc.o
 .data          0x00000000        0x0 Src\sth30_crc.o
 .bss           0x00000000        0x0 Src\sth30_crc.o
 .text.genCRC16
                0x00000000       0x48 Src\sth30_crc.o
 .data.Table_CRC16
                0x00000000      0x200 Src\sth30_crc.o
 .text          0x00000000        0x0 Src\stm32f2xx_hal_msp.o
 .data          0x00000000        0x0 Src\stm32f2xx_hal_msp.o
 .bss           0x00000000        0x0 Src\stm32f2xx_hal_msp.o
 .text.HAL_I2C_MspDeInit
                0x00000000       0x40 Src\stm32f2xx_hal_msp.o
 .text.HAL_TIM_Base_MspDeInit
                0x00000000       0x24 Src\stm32f2xx_hal_msp.o
 .text.HAL_UART_MspDeInit
                0x00000000       0x44 Src\stm32f2xx_hal_msp.o
 .text          0x00000000        0x0 Src\stm32f2xx_it.o
 .data          0x00000000        0x0 Src\stm32f2xx_it.o
 .bss           0x00000000        0x0 Src\stm32f2xx_it.o
 .text          0x00000000        0x0 Src\syscalls.o
 .data          0x00000000        0x0 Src\syscalls.o
 .bss           0x00000000        0x0 Src\syscalls.o
 .text.initialise_monitor_handles
                0x00000000        0x2 Src\syscalls.o
 .text._getpid  0x00000000        0x4 Src\syscalls.o
 .text._kill    0x00000000       0x10 Src\syscalls.o
 .text._exit    0x00000000        0xc Src\syscalls.o
 .text._write   0x00000000       0x1c Src\syscalls.o
 .text._open    0x00000000        0xa Src\syscalls.o
 .text._wait    0x00000000       0x10 Src\syscalls.o
 .text._unlink  0x00000000       0x10 Src\syscalls.o
 .text._times   0x00000000        0x6 Src\syscalls.o
 .text._stat    0x00000000        0xa Src\syscalls.o
 .text._link    0x00000000       0x10 Src\syscalls.o
 .text._fork    0x00000000       0x10 Src\syscalls.o
 .text._execve  0x00000000       0x10 Src\syscalls.o
 .bss.__env     0x00000000        0x4 Src\syscalls.o
 .data.environ  0x00000000        0x4 Src\syscalls.o
 .text          0x00000000        0x0 Src\system_stm32f2xx.o
 .data          0x00000000        0x0 Src\system_stm32f2xx.o
 .bss           0x00000000        0x0 Src\system_stm32f2xx.o
 .text.SystemCoreClockUpdate
                0x00000000       0x74 Src\system_stm32f2xx.o
 .text          0x00000000        0x0 Src\uart.o
 .data          0x00000000        0x0 Src\uart.o
 .bss           0x00000000        0x0 Src\uart.o
 .text.GetDataFromUartQueue
                0x00000000       0x4c Src\uart.o
 .text.PutDataToUartQueue
                0x00000000       0x34 Src\uart.o
 .text.Uart1_Data_Send
                0x00000000       0x10 Src\uart.o
 .text.Uart3_Data_Send
                0x00000000       0x10 Src\uart.o
 .text          0x00000000       0x14 startup\startup_stm32f207xx.o
 .data          0x00000000        0x0 startup\startup_stm32f207xx.o
 .bss           0x00000000        0x0 startup\startup_stm32f207xx.o
 .text          0x00000000        0x0 c:/program files (x86)/atollic/truestudio for stm32 9.3.0/armtools/bin/../lib/gcc/arm-atollic-eabi/6.3.1/../../../../arm-atollic-eabi/lib/armv7-m\libc_nano.a(lib_a-errno.o)
 .data          0x00000000        0x0 c:/program files (x86)/atollic/truestudio for stm32 9.3.0/armtools/bin/../lib/gcc/arm-atollic-eabi/6.3.1/../../../../arm-atollic-eabi/lib/armv7-m\libc_nano.a(lib_a-errno.o)
 .bss           0x00000000        0x0 c:/program files (x86)/atollic/truestudio for stm32 9.3.0/armtools/bin/../lib/gcc/arm-atollic-eabi/6.3.1/../../../../arm-atollic-eabi/lib/armv7-m\libc_nano.a(lib_a-errno.o)
 .text          0x00000000        0x0 c:/program files (x86)/atollic/truestudio for stm32 9.3.0/armtools/bin/../lib/gcc/arm-atollic-eabi/6.3.1/../../../../arm-atollic-eabi/lib/armv7-m\libc_nano.a(lib_a-impure.o)
 .data          0x00000000        0x0 c:/program files (x86)/atollic/truestudio for stm32 9.3.0/armtools/bin/../lib/gcc/arm-atollic-eabi/6.3.1/../../../../arm-atollic-eabi/lib/armv7-m\libc_nano.a(lib_a-impure.o)
 .bss           0x00000000        0x0 c:/program files (x86)/atollic/truestudio for stm32 9.3.0/armtools/bin/../lib/gcc/arm-atollic-eabi/6.3.1/../../../../arm-atollic-eabi/lib/armv7-m\libc_nano.a(lib_a-impure.o)
 .text          0x00000000        0x0 c:/program files (x86)/atollic/truestudio for stm32 9.3.0/armtools/bin/../lib/gcc/arm-atollic-eabi/6.3.1/../../../../arm-atollic-eabi/lib/armv7-m\libc_nano.a(lib_a-init.o)
 .data          0x00000000        0x0 c:/program files (x86)/atollic/truestudio for stm32 9.3.0/armtools/bin/../lib/gcc/arm-atollic-eabi/6.3.1/../../../../arm-atollic-eabi/lib/armv7-m\libc_nano.a(lib_a-init.o)
 .bss           0x00000000        0x0 c:/program files (x86)/atollic/truestudio for stm32 9.3.0/armtools/bin/../lib/gcc/arm-atollic-eabi/6.3.1/../../../../arm-atollic-eabi/lib/armv7-m\libc_nano.a(lib_a-init.o)
 .text          0x00000000        0x0 c:/program files (x86)/atollic/truestudio for stm32 9.3.0/armtools/bin/../lib/gcc/arm-atollic-eabi/6.3.1/../../../../arm-atollic-eabi/lib/armv7-m\libc_nano.a(lib_a-memcpy-stub.o)
 .data          0x00000000        0x0 c:/program files (x86)/atollic/truestudio for stm32 9.3.0/armtools/bin/../lib/gcc/arm-atollic-eabi/6.3.1/../../../../arm-atollic-eabi/lib/armv7-m\libc_nano.a(lib_a-memcpy-stub.o)
 .bss           0x00000000        0x0 c:/program files (x86)/atollic/truestudio for stm32 9.3.0/armtools/bin/../lib/gcc/arm-atollic-eabi/6.3.1/../../../../arm-atollic-eabi/lib/armv7-m\libc_nano.a(lib_a-memcpy-stub.o)
 .text          0x00000000        0x0 c:/program files (x86)/atollic/truestudio for stm32 9.3.0/armtools/bin/../lib/gcc/arm-atollic-eabi/6.3.1/../../../../arm-atollic-eabi/lib/armv7-m\libc_nano.a(lib_a-memset.o)
 .data          0x00000000        0x0 c:/program files (x86)/atollic/truestudio for stm32 9.3.0/armtools/bin/../lib/gcc/arm-atollic-eabi/6.3.1/../../../../arm-atollic-eabi/lib/armv7-m\libc_nano.a(lib_a-memset.o)
 .bss           0x00000000        0x0 c:/program files (x86)/atollic/truestudio for stm32 9.3.0/armtools/bin/../lib/gcc/arm-atollic-eabi/6.3.1/../../../../arm-atollic-eabi/lib/armv7-m\libc_nano.a(lib_a-memset.o)
 .text          0x00000000        0x0 c:/program files (x86)/atollic/truestudio for stm32 9.3.0/armtools/bin/../lib/gcc/arm-atollic-eabi/6.3.1/../../../../arm-atollic-eabi/lib/armv7-m\libc_nano.a(lib_a-nano-vfprintf_float.o)
 .data          0x00000000        0x0 c:/program files (x86)/atollic/truestudio for stm32 9.3.0/armtools/bin/../lib/gcc/arm-atollic-eabi/6.3.1/../../../../arm-atollic-eabi/lib/armv7-m\libc_nano.a(lib_a-nano-vfprintf_float.o)
 .bss           0x00000000        0x0 c:/program files (x86)/atollic/truestudio for stm32 9.3.0/armtools/bin/../lib/gcc/arm-atollic-eabi/6.3.1/../../../../arm-atollic-eabi/lib/armv7-m\libc_nano.a(lib_a-nano-vfprintf_float.o)
 .text          0x00000000        0x0 c:/program files (x86)/atollic/truestudio for stm32 9.3.0/armtools/bin/../lib/gcc/arm-atollic-eabi/6.3.1/../../../../arm-atollic-eabi/lib/armv7-m\libc_nano.a(lib_a-nano-vfprintf_i.o)
 .data          0x00000000        0x0 c:/program files (x86)/atollic/truestudio for stm32 9.3.0/armtools/bin/../lib/gcc/arm-atollic-eabi/6.3.1/../../../../arm-atollic-eabi/lib/armv7-m\libc_nano.a(lib_a-nano-vfprintf_i.o)
 .bss           0x00000000        0x0 c:/program files (x86)/atollic/truestudio for stm32 9.3.0/armtools/bin/../lib/gcc/arm-atollic-eabi/6.3.1/../../../../arm-atollic-eabi/lib/armv7-m\libc_nano.a(lib_a-nano-vfprintf_i.o)
 .text          0x00000000        0x0 c:/program files (x86)/atollic/truestudio for stm32 9.3.0/armtools/bin/../lib/gcc/arm-atollic-eabi/6.3.1/../../../../arm-atollic-eabi/lib/armv7-m\libc_nano.a(lib_a-printf.o)
 .data          0x00000000        0x0 c:/program files (x86)/atollic/truestudio for stm32 9.3.0/armtools/bin/../lib/gcc/arm-atollic-eabi/6.3.1/../../../../arm-atollic-eabi/lib/armv7-m\libc_nano.a(lib_a-printf.o)
 .bss           0x00000000        0x0 c:/program files (x86)/atollic/truestudio for stm32 9.3.0/armtools/bin/../lib/gcc/arm-atollic-eabi/6.3.1/../../../../arm-atollic-eabi/lib/armv7-m\libc_nano.a(lib_a-printf.o)
 .text._printf_r
                0x00000000       0x28 c:/program files (x86)/atollic/truestudio for stm32 9.3.0/armtools/bin/../lib/gcc/arm-atollic-eabi/6.3.1/../../../../arm-atollic-eabi/lib/armv7-m\libc_nano.a(lib_a-printf.o)
 .text          0x00000000        0x0 c:/program files (x86)/atollic/truestudio for stm32 9.3.0/armtools/bin/../lib/gcc/arm-atollic-eabi/6.3.1/../../../../arm-atollic-eabi/lib/armv7-m\libc_nano.a(lib_a-puts.o)
 .data          0x00000000        0x0 c:/program files (x86)/atollic/truestudio for stm32 9.3.0/armtools/bin/../lib/gcc/arm-atollic-eabi/6.3.1/../../../../arm-atollic-eabi/lib/armv7-m\libc_nano.a(lib_a-puts.o)
 .bss           0x00000000        0x0 c:/program files (x86)/atollic/truestudio for stm32 9.3.0/armtools/bin/../lib/gcc/arm-atollic-eabi/6.3.1/../../../../arm-atollic-eabi/lib/armv7-m\libc_nano.a(lib_a-puts.o)
 .text          0x00000000        0x0 c:/program files (x86)/atollic/truestudio for stm32 9.3.0/armtools/bin/../lib/gcc/arm-atollic-eabi/6.3.1/../../../../arm-atollic-eabi/lib/armv7-m\libc_nano.a(lib_a-setbuf.o)
 .data          0x00000000        0x0 c:/program files (x86)/atollic/truestudio for stm32 9.3.0/armtools/bin/../lib/gcc/arm-atollic-eabi/6.3.1/../../../../arm-atollic-eabi/lib/armv7-m\libc_nano.a(lib_a-setbuf.o)
 .bss           0x00000000        0x0 c:/program files (x86)/atollic/truestudio for stm32 9.3.0/armtools/bin/../lib/gcc/arm-atollic-eabi/6.3.1/../../../../arm-atollic-eabi/lib/armv7-m\libc_nano.a(lib_a-setbuf.o)
 .text          0x00000000        0x0 c:/program files (x86)/atollic/truestudio for stm32 9.3.0/armtools/bin/../lib/gcc/arm-atollic-eabi/6.3.1/../../../../arm-atollic-eabi/lib/armv7-m\libc_nano.a(lib_a-setvbuf.o)
 .data          0x00000000        0x0 c:/program files (x86)/atollic/truestudio for stm32 9.3.0/armtools/bin/../lib/gcc/arm-atollic-eabi/6.3.1/../../../../arm-atollic-eabi/lib/armv7-m\libc_nano.a(lib_a-setvbuf.o)
 .bss           0x00000000        0x0 c:/program files (x86)/atollic/truestudio for stm32 9.3.0/armtools/bin/../lib/gcc/arm-atollic-eabi/6.3.1/../../../../arm-atollic-eabi/lib/armv7-m\libc_nano.a(lib_a-setvbuf.o)
 .text          0x00000000        0x0 c:/program files (x86)/atollic/truestudio for stm32 9.3.0/armtools/bin/../lib/gcc/arm-atollic-eabi/6.3.1/../../../../arm-atollic-eabi/lib/armv7-m\libc_nano.a(lib_a-sprintf.o)
 .data          0x00000000        0x0 c:/program files (x86)/atollic/truestudio for stm32 9.3.0/armtools/bin/../lib/gcc/arm-atollic-eabi/6.3.1/../../../../arm-atollic-eabi/lib/armv7-m\libc_nano.a(lib_a-sprintf.o)
 .bss           0x00000000        0x0 c:/program files (x86)/atollic/truestudio for stm32 9.3.0/armtools/bin/../lib/gcc/arm-atollic-eabi/6.3.1/../../../../arm-atollic-eabi/lib/armv7-m\libc_nano.a(lib_a-sprintf.o)
 .text._sprintf_r
                0x00000000       0x40 c:/program files (x86)/atollic/truestudio for stm32 9.3.0/armtools/bin/../lib/gcc/arm-atollic-eabi/6.3.1/../../../../arm-atollic-eabi/lib/armv7-m\libc_nano.a(lib_a-sprintf.o)
 .text          0x00000000        0x0 c:/program files (x86)/atollic/truestudio for stm32 9.3.0/armtools/bin/../lib/gcc/arm-atollic-eabi/6.3.1/../../../../arm-atollic-eabi/lib/armv7-m\libc_nano.a(lib_a-strcpy.o)
 .data          0x00000000        0x0 c:/program files (x86)/atollic/truestudio for stm32 9.3.0/armtools/bin/../lib/gcc/arm-atollic-eabi/6.3.1/../../../../arm-atollic-eabi/lib/armv7-m\libc_nano.a(lib_a-strcpy.o)
 .bss           0x00000000        0x0 c:/program files (x86)/atollic/truestudio for stm32 9.3.0/armtools/bin/../lib/gcc/arm-atollic-eabi/6.3.1/../../../../arm-atollic-eabi/lib/armv7-m\libc_nano.a(lib_a-strcpy.o)
 .data          0x00000000        0x0 c:/program files (x86)/atollic/truestudio for stm32 9.3.0/armtools/bin/../lib/gcc/arm-atollic-eabi/6.3.1/../../../../arm-atollic-eabi/lib/armv7-m\libc_nano.a(lib_a-strlen.o)
 .bss           0x00000000        0x0 c:/program files (x86)/atollic/truestudio for stm32 9.3.0/armtools/bin/../lib/gcc/arm-atollic-eabi/6.3.1/../../../../arm-atollic-eabi/lib/armv7-m\libc_nano.a(lib_a-strlen.o)
 .text          0x00000000        0x0 c:/program files (x86)/atollic/truestudio for stm32 9.3.0/armtools/bin/../lib/gcc/arm-atollic-eabi/6.3.1/../../../../arm-atollic-eabi/lib/armv7-m\libc_nano.a(lib_a-wbuf.o)
 .data          0x00000000        0x0 c:/program files (x86)/atollic/truestudio for stm32 9.3.0/armtools/bin/../lib/gcc/arm-atollic-eabi/6.3.1/../../../../arm-atollic-eabi/lib/armv7-m\libc_nano.a(lib_a-wbuf.o)
 .bss           0x00000000        0x0 c:/program files (x86)/atollic/truestudio for stm32 9.3.0/armtools/bin/../lib/gcc/arm-atollic-eabi/6.3.1/../../../../arm-atollic-eabi/lib/armv7-m\libc_nano.a(lib_a-wbuf.o)
 .text.__swbuf  0x00000000       0x10 c:/program files (x86)/atollic/truestudio for stm32 9.3.0/armtools/bin/../lib/gcc/arm-atollic-eabi/6.3.1/../../../../arm-atollic-eabi/lib/armv7-m\libc_nano.a(lib_a-wbuf.o)
 .text          0x00000000        0x0 c:/program files (x86)/atollic/truestudio for stm32 9.3.0/armtools/bin/../lib/gcc/arm-atollic-eabi/6.3.1/../../../../arm-atollic-eabi/lib/armv7-m\libc_nano.a(lib_a-wsetup.o)
 .data          0x00000000        0x0 c:/program files (x86)/atollic/truestudio for stm32 9.3.0/armtools/bin/../lib/gcc/arm-atollic-eabi/6.3.1/../../../../arm-atollic-eabi/lib/armv7-m\libc_nano.a(lib_a-wsetup.o)
 .bss           0x00000000        0x0 c:/program files (x86)/atollic/truestudio for stm32 9.3.0/armtools/bin/../lib/gcc/arm-atollic-eabi/6.3.1/../../../../arm-atollic-eabi/lib/armv7-m\libc_nano.a(lib_a-wsetup.o)
 .text          0x00000000        0x0 c:/program files (x86)/atollic/truestudio for stm32 9.3.0/armtools/bin/../lib/gcc/arm-atollic-eabi/6.3.1/../../../../arm-atollic-eabi/lib/armv7-m\libc_nano.a(lib_a-dtoa.o)
 .data          0x00000000        0x0 c:/program files (x86)/atollic/truestudio for stm32 9.3.0/armtools/bin/../lib/gcc/arm-atollic-eabi/6.3.1/../../../../arm-atollic-eabi/lib/armv7-m\libc_nano.a(lib_a-dtoa.o)
 .bss           0x00000000        0x0 c:/program files (x86)/atollic/truestudio for stm32 9.3.0/armtools/bin/../lib/gcc/arm-atollic-eabi/6.3.1/../../../../arm-atollic-eabi/lib/armv7-m\libc_nano.a(lib_a-dtoa.o)
 .text          0x00000000        0x0 c:/program files (x86)/atollic/truestudio for stm32 9.3.0/armtools/bin/../lib/gcc/arm-atollic-eabi/6.3.1/../../../../arm-atollic-eabi/lib/armv7-m\libc_nano.a(lib_a-fflush.o)
 .data          0x00000000        0x0 c:/program files (x86)/atollic/truestudio for stm32 9.3.0/armtools/bin/../lib/gcc/arm-atollic-eabi/6.3.1/../../../../arm-atollic-eabi/lib/armv7-m\libc_nano.a(lib_a-fflush.o)
 .bss           0x00000000        0x0 c:/program files (x86)/atollic/truestudio for stm32 9.3.0/armtools/bin/../lib/gcc/arm-atollic-eabi/6.3.1/../../../../arm-atollic-eabi/lib/armv7-m\libc_nano.a(lib_a-fflush.o)
 .text.fflush   0x00000000       0x24 c:/program files (x86)/atollic/truestudio for stm32 9.3.0/armtools/bin/../lib/gcc/arm-atollic-eabi/6.3.1/../../../../arm-atollic-eabi/lib/armv7-m\libc_nano.a(lib_a-fflush.o)
 .text          0x00000000        0x0 c:/program files (x86)/atollic/truestudio for stm32 9.3.0/armtools/bin/../lib/gcc/arm-atollic-eabi/6.3.1/../../../../arm-atollic-eabi/lib/armv7-m\libc_nano.a(lib_a-findfp.o)
 .data          0x00000000        0x0 c:/program files (x86)/atollic/truestudio for stm32 9.3.0/armtools/bin/../lib/gcc/arm-atollic-eabi/6.3.1/../../../../arm-atollic-eabi/lib/armv7-m\libc_nano.a(lib_a-findfp.o)
 .bss           0x00000000        0x0 c:/program files (x86)/atollic/truestudio for stm32 9.3.0/armtools/bin/../lib/gcc/arm-atollic-eabi/6.3.1/../../../../arm-atollic-eabi/lib/armv7-m\libc_nano.a(lib_a-findfp.o)
 .text.__fp_unlock
                0x00000000        0x4 c:/program files (x86)/atollic/truestudio for stm32 9.3.0/armtools/bin/../lib/gcc/arm-atollic-eabi/6.3.1/../../../../arm-atollic-eabi/lib/armv7-m\libc_nano.a(lib_a-findfp.o)
 .text.__fp_lock
                0x00000000        0x4 c:/program files (x86)/atollic/truestudio for stm32 9.3.0/armtools/bin/../lib/gcc/arm-atollic-eabi/6.3.1/../../../../arm-atollic-eabi/lib/armv7-m\libc_nano.a(lib_a-findfp.o)
 .text._cleanup
                0x00000000        0xc c:/program files (x86)/atollic/truestudio for stm32 9.3.0/armtools/bin/../lib/gcc/arm-atollic-eabi/6.3.1/../../../../arm-atollic-eabi/lib/armv7-m\libc_nano.a(lib_a-findfp.o)
 .text.__sfp_lock_acquire
                0x00000000        0x2 c:/program files (x86)/atollic/truestudio for stm32 9.3.0/armtools/bin/../lib/gcc/arm-atollic-eabi/6.3.1/../../../../arm-atollic-eabi/lib/armv7-m\libc_nano.a(lib_a-findfp.o)
 .text.__sfp_lock_release
                0x00000000        0x2 c:/program files (x86)/atollic/truestudio for stm32 9.3.0/armtools/bin/../lib/gcc/arm-atollic-eabi/6.3.1/../../../../arm-atollic-eabi/lib/armv7-m\libc_nano.a(lib_a-findfp.o)
 .text.__sinit_lock_acquire
                0x00000000        0x2 c:/program files (x86)/atollic/truestudio for stm32 9.3.0/armtools/bin/../lib/gcc/arm-atollic-eabi/6.3.1/../../../../arm-atollic-eabi/lib/armv7-m\libc_nano.a(lib_a-findfp.o)
 .text.__sinit_lock_release
                0x00000000        0x2 c:/program files (x86)/atollic/truestudio for stm32 9.3.0/armtools/bin/../lib/gcc/arm-atollic-eabi/6.3.1/../../../../arm-atollic-eabi/lib/armv7-m\libc_nano.a(lib_a-findfp.o)
 .text.__fp_lock_all
                0x00000000       0x14 c:/program files (x86)/atollic/truestudio for stm32 9.3.0/armtools/bin/../lib/gcc/arm-atollic-eabi/6.3.1/../../../../arm-atollic-eabi/lib/armv7-m\libc_nano.a(lib_a-findfp.o)
 .text.__fp_unlock_all
                0x00000000       0x14 c:/program files (x86)/atollic/truestudio for stm32 9.3.0/armtools/bin/../lib/gcc/arm-atollic-eabi/6.3.1/../../../../arm-atollic-eabi/lib/armv7-m\libc_nano.a(lib_a-findfp.o)
 .text          0x00000000        0x0 c:/program files (x86)/atollic/truestudio for stm32 9.3.0/armtools/bin/../lib/gcc/arm-atollic-eabi/6.3.1/../../../../arm-atollic-eabi/lib/armv7-m\libc_nano.a(lib_a-fwalk.o)
 .data          0x00000000        0x0 c:/program files (x86)/atollic/truestudio for stm32 9.3.0/armtools/bin/../lib/gcc/arm-atollic-eabi/6.3.1/../../../../arm-atollic-eabi/lib/armv7-m\libc_nano.a(lib_a-fwalk.o)
 .bss           0x00000000        0x0 c:/program files (x86)/atollic/truestudio for stm32 9.3.0/armtools/bin/../lib/gcc/arm-atollic-eabi/6.3.1/../../../../arm-atollic-eabi/lib/armv7-m\libc_nano.a(lib_a-fwalk.o)
 .text._fwalk   0x00000000       0x38 c:/program files (x86)/atollic/truestudio for stm32 9.3.0/armtools/bin/../lib/gcc/arm-atollic-eabi/6.3.1/../../../../arm-atollic-eabi/lib/armv7-m\libc_nano.a(lib_a-fwalk.o)
 .text          0x00000000        0x0 c:/program files (x86)/atollic/truestudio for stm32 9.3.0/armtools/bin/../lib/gcc/arm-atollic-eabi/6.3.1/../../../../arm-atollic-eabi/lib/armv7-m\libc_nano.a(lib_a-localeconv.o)
 .data          0x00000000        0x0 c:/program files (x86)/atollic/truestudio for stm32 9.3.0/armtools/bin/../lib/gcc/arm-atollic-eabi/6.3.1/../../../../arm-atollic-eabi/lib/armv7-m\libc_nano.a(lib_a-localeconv.o)
 .bss           0x00000000        0x0 c:/program files (x86)/atollic/truestudio for stm32 9.3.0/armtools/bin/../lib/gcc/arm-atollic-eabi/6.3.1/../../../../arm-atollic-eabi/lib/armv7-m\libc_nano.a(lib_a-localeconv.o)
 .text.__localeconv_l
                0x00000000        0x4 c:/program files (x86)/atollic/truestudio for stm32 9.3.0/armtools/bin/../lib/gcc/arm-atollic-eabi/6.3.1/../../../../arm-atollic-eabi/lib/armv7-m\libc_nano.a(lib_a-localeconv.o)
 .text.localeconv
                0x00000000       0x1c c:/program files (x86)/atollic/truestudio for stm32 9.3.0/armtools/bin/../lib/gcc/arm-atollic-eabi/6.3.1/../../../../arm-atollic-eabi/lib/armv7-m\libc_nano.a(lib_a-localeconv.o)
 .text          0x00000000        0x0 c:/program files (x86)/atollic/truestudio for stm32 9.3.0/armtools/bin/../lib/gcc/arm-atollic-eabi/6.3.1/../../../../arm-atollic-eabi/lib/armv7-m\libc_nano.a(lib_a-makebuf.o)
 .data          0x00000000        0x0 c:/program files (x86)/atollic/truestudio for stm32 9.3.0/armtools/bin/../lib/gcc/arm-atollic-eabi/6.3.1/../../../../arm-atollic-eabi/lib/armv7-m\libc_nano.a(lib_a-makebuf.o)
 .bss           0x00000000        0x0 c:/program files (x86)/atollic/truestudio for stm32 9.3.0/armtools/bin/../lib/gcc/arm-atollic-eabi/6.3.1/../../../../arm-atollic-eabi/lib/armv7-m\libc_nano.a(lib_a-makebuf.o)
 .text          0x00000000        0x0 c:/program files (x86)/atollic/truestudio for stm32 9.3.0/armtools/bin/../lib/gcc/arm-atollic-eabi/6.3.1/../../../../arm-atollic-eabi/lib/armv7-m\libc_nano.a(lib_a-malloc.o)
 .data          0x00000000        0x0 c:/program files (x86)/atollic/truestudio for stm32 9.3.0/armtools/bin/../lib/gcc/arm-atollic-eabi/6.3.1/../../../../arm-atollic-eabi/lib/armv7-m\libc_nano.a(lib_a-malloc.o)
 .bss           0x00000000        0x0 c:/program files (x86)/atollic/truestudio for stm32 9.3.0/armtools/bin/../lib/gcc/arm-atollic-eabi/6.3.1/../../../../arm-atollic-eabi/lib/armv7-m\libc_nano.a(lib_a-malloc.o)
 .text.free     0x00000000       0x10 c:/program files (x86)/atollic/truestudio for stm32 9.3.0/armtools/bin/../lib/gcc/arm-atollic-eabi/6.3.1/../../../../arm-atollic-eabi/lib/armv7-m\libc_nano.a(lib_a-malloc.o)
 .text          0x00000000        0x0 c:/program files (x86)/atollic/truestudio for stm32 9.3.0/armtools/bin/../lib/gcc/arm-atollic-eabi/6.3.1/../../../../arm-atollic-eabi/lib/armv7-m\libc_nano.a(lib_a-memchr-stub.o)
 .data          0x00000000        0x0 c:/program files (x86)/atollic/truestudio for stm32 9.3.0/armtools/bin/../lib/gcc/arm-atollic-eabi/6.3.1/../../../../arm-atollic-eabi/lib/armv7-m\libc_nano.a(lib_a-memchr-stub.o)
 .bss           0x00000000        0x0 c:/program files (x86)/atollic/truestudio for stm32 9.3.0/armtools/bin/../lib/gcc/arm-atollic-eabi/6.3.1/../../../../arm-atollic-eabi/lib/armv7-m\libc_nano.a(lib_a-memchr-stub.o)
 .text          0x00000000        0x0 c:/program files (x86)/atollic/truestudio for stm32 9.3.0/armtools/bin/../lib/gcc/arm-atollic-eabi/6.3.1/../../../../arm-atollic-eabi/lib/armv7-m\libc_nano.a(lib_a-mprec.o)
 .data          0x00000000        0x0 c:/program files (x86)/atollic/truestudio for stm32 9.3.0/armtools/bin/../lib/gcc/arm-atollic-eabi/6.3.1/../../../../arm-atollic-eabi/lib/armv7-m\libc_nano.a(lib_a-mprec.o)
 .bss           0x00000000        0x0 c:/program files (x86)/atollic/truestudio for stm32 9.3.0/armtools/bin/../lib/gcc/arm-atollic-eabi/6.3.1/../../../../arm-atollic-eabi/lib/armv7-m\libc_nano.a(lib_a-mprec.o)
 .text.__s2b    0x00000000       0x7c c:/program files (x86)/atollic/truestudio for stm32 9.3.0/armtools/bin/../lib/gcc/arm-atollic-eabi/6.3.1/../../../../arm-atollic-eabi/lib/armv7-m\libc_nano.a(lib_a-mprec.o)
 .text.__ulp    0x00000000       0x48 c:/program files (x86)/atollic/truestudio for stm32 9.3.0/armtools/bin/../lib/gcc/arm-atollic-eabi/6.3.1/../../../../arm-atollic-eabi/lib/armv7-m\libc_nano.a(lib_a-mprec.o)
 .text.__b2d    0x00000000       0xa4 c:/program files (x86)/atollic/truestudio for stm32 9.3.0/armtools/bin/../lib/gcc/arm-atollic-eabi/6.3.1/../../../../arm-atollic-eabi/lib/armv7-m\libc_nano.a(lib_a-mprec.o)
 .text.__ratio  0x00000000       0x50 c:/program files (x86)/atollic/truestudio for stm32 9.3.0/armtools/bin/../lib/gcc/arm-atollic-eabi/6.3.1/../../../../arm-atollic-eabi/lib/armv7-m\libc_nano.a(lib_a-mprec.o)
 .text._mprec_log10
                0x00000000       0x38 c:/program files (x86)/atollic/truestudio for stm32 9.3.0/armtools/bin/../lib/gcc/arm-atollic-eabi/6.3.1/../../../../arm-atollic-eabi/lib/armv7-m\libc_nano.a(lib_a-mprec.o)
 .text.__copybits
                0x00000000       0x34 c:/program files (x86)/atollic/truestudio for stm32 9.3.0/armtools/bin/../lib/gcc/arm-atollic-eabi/6.3.1/../../../../arm-atollic-eabi/lib/armv7-m\libc_nano.a(lib_a-mprec.o)
 .text.__any_on
                0x00000000       0x42 c:/program files (x86)/atollic/truestudio for stm32 9.3.0/armtools/bin/../lib/gcc/arm-atollic-eabi/6.3.1/../../../../arm-atollic-eabi/lib/armv7-m\libc_nano.a(lib_a-mprec.o)
 .rodata.__mprec_tinytens
                0x00000000       0x28 c:/program files (x86)/atollic/truestudio for stm32 9.3.0/armtools/bin/../lib/gcc/arm-atollic-eabi/6.3.1/../../../../arm-atollic-eabi/lib/armv7-m\libc_nano.a(lib_a-mprec.o)
 .text          0x00000000        0x0 c:/program files (x86)/atollic/truestudio for stm32 9.3.0/armtools/bin/../lib/gcc/arm-atollic-eabi/6.3.1/../../../../arm-atollic-eabi/lib/armv7-m\libc_nano.a(lib_a-nano-callocr.o)
 .data          0x00000000        0x0 c:/program files (x86)/atollic/truestudio for stm32 9.3.0/armtools/bin/../lib/gcc/arm-atollic-eabi/6.3.1/../../../../arm-atollic-eabi/lib/armv7-m\libc_nano.a(lib_a-nano-callocr.o)
 .bss           0x00000000        0x0 c:/program files (x86)/atollic/truestudio for stm32 9.3.0/armtools/bin/../lib/gcc/arm-atollic-eabi/6.3.1/../../../../arm-atollic-eabi/lib/armv7-m\libc_nano.a(lib_a-nano-callocr.o)
 .text          0x00000000        0x0 c:/program files (x86)/atollic/truestudio for stm32 9.3.0/armtools/bin/../lib/gcc/arm-atollic-eabi/6.3.1/../../../../arm-atollic-eabi/lib/armv7-m\libc_nano.a(lib_a-nano-freer.o)
 .data          0x00000000        0x0 c:/program files (x86)/atollic/truestudio for stm32 9.3.0/armtools/bin/../lib/gcc/arm-atollic-eabi/6.3.1/../../../../arm-atollic-eabi/lib/armv7-m\libc_nano.a(lib_a-nano-freer.o)
 .bss           0x00000000        0x0 c:/program files (x86)/atollic/truestudio for stm32 9.3.0/armtools/bin/../lib/gcc/arm-atollic-eabi/6.3.1/../../../../arm-atollic-eabi/lib/armv7-m\libc_nano.a(lib_a-nano-freer.o)
 .text          0x00000000        0x0 c:/program files (x86)/atollic/truestudio for stm32 9.3.0/armtools/bin/../lib/gcc/arm-atollic-eabi/6.3.1/../../../../arm-atollic-eabi/lib/armv7-m\libc_nano.a(lib_a-nano-mallocr.o)
 .data          0x00000000        0x0 c:/program files (x86)/atollic/truestudio for stm32 9.3.0/armtools/bin/../lib/gcc/arm-atollic-eabi/6.3.1/../../../../arm-atollic-eabi/lib/armv7-m\libc_nano.a(lib_a-nano-mallocr.o)
 .bss           0x00000000        0x0 c:/program files (x86)/atollic/truestudio for stm32 9.3.0/armtools/bin/../lib/gcc/arm-atollic-eabi/6.3.1/../../../../arm-atollic-eabi/lib/armv7-m\libc_nano.a(lib_a-nano-mallocr.o)
 .text          0x00000000        0x0 c:/program files (x86)/atollic/truestudio for stm32 9.3.0/armtools/bin/../lib/gcc/arm-atollic-eabi/6.3.1/../../../../arm-atollic-eabi/lib/armv7-m\libc_nano.a(lib_a-nano-svfprintf.o)
 .data          0x00000000        0x0 c:/program files (x86)/atollic/truestudio for stm32 9.3.0/armtools/bin/../lib/gcc/arm-atollic-eabi/6.3.1/../../../../arm-atollic-eabi/lib/armv7-m\libc_nano.a(lib_a-nano-svfprintf.o)
 .bss           0x00000000        0x0 c:/program files (x86)/atollic/truestudio for stm32 9.3.0/armtools/bin/../lib/gcc/arm-atollic-eabi/6.3.1/../../../../arm-atollic-eabi/lib/armv7-m\libc_nano.a(lib_a-nano-svfprintf.o)
 .text.__ssprint_r
                0x00000000       0xf4 c:/program files (x86)/atollic/truestudio for stm32 9.3.0/armtools/bin/../lib/gcc/arm-atollic-eabi/6.3.1/../../../../arm-atollic-eabi/lib/armv7-m\libc_nano.a(lib_a-nano-svfprintf.o)
 .text          0x00000000        0x0 c:/program files (x86)/atollic/truestudio for stm32 9.3.0/armtools/bin/../lib/gcc/arm-atollic-eabi/6.3.1/../../../../arm-atollic-eabi/lib/armv7-m\libc_nano.a(lib_a-nano-vfprintf.o)
 .data          0x00000000        0x0 c:/program files (x86)/atollic/truestudio for stm32 9.3.0/armtools/bin/../lib/gcc/arm-atollic-eabi/6.3.1/../../../../arm-atollic-eabi/lib/armv7-m\libc_nano.a(lib_a-nano-vfprintf.o)
 .bss           0x00000000        0x0 c:/program files (x86)/atollic/truestudio for stm32 9.3.0/armtools/bin/../lib/gcc/arm-atollic-eabi/6.3.1/../../../../arm-atollic-eabi/lib/armv7-m\libc_nano.a(lib_a-nano-vfprintf.o)
 .text.__sprint_r
                0x00000000       0x1a c:/program files (x86)/atollic/truestudio for stm32 9.3.0/armtools/bin/../lib/gcc/arm-atollic-eabi/6.3.1/../../../../arm-atollic-eabi/lib/armv7-m\libc_nano.a(lib_a-nano-vfprintf.o)
 .text.vfprintf
                0x00000000       0x14 c:/program files (x86)/atollic/truestudio for stm32 9.3.0/armtools/bin/../lib/gcc/arm-atollic-eabi/6.3.1/../../../../arm-atollic-eabi/lib/armv7-m\libc_nano.a(lib_a-nano-vfprintf.o)
 .text          0x00000000        0x0 c:/program files (x86)/atollic/truestudio for stm32 9.3.0/armtools/bin/../lib/gcc/arm-atollic-eabi/6.3.1/../../../../arm-atollic-eabi/lib/armv7-m\libc_nano.a(lib_a-sbrkr.o)
 .data          0x00000000        0x0 c:/program files (x86)/atollic/truestudio for stm32 9.3.0/armtools/bin/../lib/gcc/arm-atollic-eabi/6.3.1/../../../../arm-atollic-eabi/lib/armv7-m\libc_nano.a(lib_a-sbrkr.o)
 .bss           0x00000000        0x0 c:/program files (x86)/atollic/truestudio for stm32 9.3.0/armtools/bin/../lib/gcc/arm-atollic-eabi/6.3.1/../../../../arm-atollic-eabi/lib/armv7-m\libc_nano.a(lib_a-sbrkr.o)
 .text          0x00000000        0x0 c:/program files (x86)/atollic/truestudio for stm32 9.3.0/armtools/bin/../lib/gcc/arm-atollic-eabi/6.3.1/../../../../arm-atollic-eabi/lib/armv7-m\libc_nano.a(lib_a-stdio.o)
 .data          0x00000000        0x0 c:/program files (x86)/atollic/truestudio for stm32 9.3.0/armtools/bin/../lib/gcc/arm-atollic-eabi/6.3.1/../../../../arm-atollic-eabi/lib/armv7-m\libc_nano.a(lib_a-stdio.o)
 .bss           0x00000000        0x0 c:/program files (x86)/atollic/truestudio for stm32 9.3.0/armtools/bin/../lib/gcc/arm-atollic-eabi/6.3.1/../../../../arm-atollic-eabi/lib/armv7-m\libc_nano.a(lib_a-stdio.o)
 .text.__seofread
                0x00000000        0x4 c:/program files (x86)/atollic/truestudio for stm32 9.3.0/armtools/bin/../lib/gcc/arm-atollic-eabi/6.3.1/../../../../arm-atollic-eabi/lib/armv7-m\libc_nano.a(lib_a-stdio.o)
 .text          0x00000000        0x0 c:/program files (x86)/atollic/truestudio for stm32 9.3.0/armtools/bin/../lib/gcc/arm-atollic-eabi/6.3.1/../../../../arm-atollic-eabi/lib/armv7-m\libc_nano.a(lib_a-writer.o)
 .data          0x00000000        0x0 c:/program files (x86)/atollic/truestudio for stm32 9.3.0/armtools/bin/../lib/gcc/arm-atollic-eabi/6.3.1/../../../../arm-atollic-eabi/lib/armv7-m\libc_nano.a(lib_a-writer.o)
 .bss           0x00000000        0x0 c:/program files (x86)/atollic/truestudio for stm32 9.3.0/armtools/bin/../lib/gcc/arm-atollic-eabi/6.3.1/../../../../arm-atollic-eabi/lib/armv7-m\libc_nano.a(lib_a-writer.o)
 .text          0x00000000        0x0 c:/program files (x86)/atollic/truestudio for stm32 9.3.0/armtools/bin/../lib/gcc/arm-atollic-eabi/6.3.1/../../../../arm-atollic-eabi/lib/armv7-m\libc_nano.a(lib_a-closer.o)
 .data          0x00000000        0x0 c:/program files (x86)/atollic/truestudio for stm32 9.3.0/armtools/bin/../lib/gcc/arm-atollic-eabi/6.3.1/../../../../arm-atollic-eabi/lib/armv7-m\libc_nano.a(lib_a-closer.o)
 .bss           0x00000000        0x0 c:/program files (x86)/atollic/truestudio for stm32 9.3.0/armtools/bin/../lib/gcc/arm-atollic-eabi/6.3.1/../../../../arm-atollic-eabi/lib/armv7-m\libc_nano.a(lib_a-closer.o)
 .text          0x00000000        0x0 c:/program files (x86)/atollic/truestudio for stm32 9.3.0/armtools/bin/../lib/gcc/arm-atollic-eabi/6.3.1/../../../../arm-atollic-eabi/lib/armv7-m\libc_nano.a(lib_a-fstatr.o)
 .data          0x00000000        0x0 c:/program files (x86)/atollic/truestudio for stm32 9.3.0/armtools/bin/../lib/gcc/arm-atollic-eabi/6.3.1/../../../../arm-atollic-eabi/lib/armv7-m\libc_nano.a(lib_a-fstatr.o)
 .bss           0x00000000        0x0 c:/program files (x86)/atollic/truestudio for stm32 9.3.0/armtools/bin/../lib/gcc/arm-atollic-eabi/6.3.1/../../../../arm-atollic-eabi/lib/armv7-m\libc_nano.a(lib_a-fstatr.o)
 .text          0x00000000        0x0 c:/program files (x86)/atollic/truestudio for stm32 9.3.0/armtools/bin/../lib/gcc/arm-atollic-eabi/6.3.1/../../../../arm-atollic-eabi/lib/armv7-m\libc_nano.a(lib_a-fvwrite.o)
 .data          0x00000000        0x0 c:/program files (x86)/atollic/truestudio for stm32 9.3.0/armtools/bin/../lib/gcc/arm-atollic-eabi/6.3.1/../../../../arm-atollic-eabi/lib/armv7-m\libc_nano.a(lib_a-fvwrite.o)
 .bss           0x00000000        0x0 c:/program files (x86)/atollic/truestudio for stm32 9.3.0/armtools/bin/../lib/gcc/arm-atollic-eabi/6.3.1/../../../../arm-atollic-eabi/lib/armv7-m\libc_nano.a(lib_a-fvwrite.o)
 .text.__sfvwrite_r
                0x00000000      0x29c c:/program files (x86)/atollic/truestudio for stm32 9.3.0/armtools/bin/../lib/gcc/arm-atollic-eabi/6.3.1/../../../../arm-atollic-eabi/lib/armv7-m\libc_nano.a(lib_a-fvwrite.o)
 .debug_frame   0x00000000       0x3c c:/program files (x86)/atollic/truestudio for stm32 9.3.0/armtools/bin/../lib/gcc/arm-atollic-eabi/6.3.1/../../../../arm-atollic-eabi/lib/armv7-m\libc_nano.a(lib_a-fvwrite.o)
 .ARM.attributes
                0x00000000       0x2d c:/program files (x86)/atollic/truestudio for stm32 9.3.0/armtools/bin/../lib/gcc/arm-atollic-eabi/6.3.1/../../../../arm-atollic-eabi/lib/armv7-m\libc_nano.a(lib_a-fvwrite.o)
 .text          0x00000000        0x0 c:/program files (x86)/atollic/truestudio for stm32 9.3.0/armtools/bin/../lib/gcc/arm-atollic-eabi/6.3.1/../../../../arm-atollic-eabi/lib/armv7-m\libc_nano.a(lib_a-isattyr.o)
 .data          0x00000000        0x0 c:/program files (x86)/atollic/truestudio for stm32 9.3.0/armtools/bin/../lib/gcc/arm-atollic-eabi/6.3.1/../../../../arm-atollic-eabi/lib/armv7-m\libc_nano.a(lib_a-isattyr.o)
 .bss           0x00000000        0x0 c:/program files (x86)/atollic/truestudio for stm32 9.3.0/armtools/bin/../lib/gcc/arm-atollic-eabi/6.3.1/../../../../arm-atollic-eabi/lib/armv7-m\libc_nano.a(lib_a-isattyr.o)
 .text          0x00000000        0x0 c:/program files (x86)/atollic/truestudio for stm32 9.3.0/armtools/bin/../lib/gcc/arm-atollic-eabi/6.3.1/../../../../arm-atollic-eabi/lib/armv7-m\libc_nano.a(lib_a-locale.o)
 .data          0x00000000        0x0 c:/program files (x86)/atollic/truestudio for stm32 9.3.0/armtools/bin/../lib/gcc/arm-atollic-eabi/6.3.1/../../../../arm-atollic-eabi/lib/armv7-m\libc_nano.a(lib_a-locale.o)
 .bss           0x00000000        0x0 c:/program files (x86)/atollic/truestudio for stm32 9.3.0/armtools/bin/../lib/gcc/arm-atollic-eabi/6.3.1/../../../../arm-atollic-eabi/lib/armv7-m\libc_nano.a(lib_a-locale.o)
 .text._setlocale_r
                0x00000000       0x38 c:/program files (x86)/atollic/truestudio for stm32 9.3.0/armtools/bin/../lib/gcc/arm-atollic-eabi/6.3.1/../../../../arm-atollic-eabi/lib/armv7-m\libc_nano.a(lib_a-locale.o)
 .text.__locale_mb_cur_max
                0x00000000       0x1c c:/program files (x86)/atollic/truestudio for stm32 9.3.0/armtools/bin/../lib/gcc/arm-atollic-eabi/6.3.1/../../../../arm-atollic-eabi/lib/armv7-m\libc_nano.a(lib_a-locale.o)
 .text.__locale_ctype_ptr_l
                0x00000000        0x6 c:/program files (x86)/atollic/truestudio for stm32 9.3.0/armtools/bin/../lib/gcc/arm-atollic-eabi/6.3.1/../../../../arm-atollic-eabi/lib/armv7-m\libc_nano.a(lib_a-locale.o)
 .text.__locale_ctype_ptr
                0x00000000       0x1c c:/program files (x86)/atollic/truestudio for stm32 9.3.0/armtools/bin/../lib/gcc/arm-atollic-eabi/6.3.1/../../../../arm-atollic-eabi/lib/armv7-m\libc_nano.a(lib_a-locale.o)
 .text.setlocale
                0x00000000       0x10 c:/program files (x86)/atollic/truestudio for stm32 9.3.0/armtools/bin/../lib/gcc/arm-atollic-eabi/6.3.1/../../../../arm-atollic-eabi/lib/armv7-m\libc_nano.a(lib_a-locale.o)
 .bss._PathLocale
                0x00000000        0x4 c:/program files (x86)/atollic/truestudio for stm32 9.3.0/armtools/bin/../lib/gcc/arm-atollic-eabi/6.3.1/../../../../arm-atollic-eabi/lib/armv7-m\libc_nano.a(lib_a-locale.o)
 .text          0x00000000        0x0 c:/program files (x86)/atollic/truestudio for stm32 9.3.0/armtools/bin/../lib/gcc/arm-atollic-eabi/6.3.1/../../../../arm-atollic-eabi/lib/armv7-m\libc_nano.a(lib_a-lseekr.o)
 .data          0x00000000        0x0 c:/program files (x86)/atollic/truestudio for stm32 9.3.0/armtools/bin/../lib/gcc/arm-atollic-eabi/6.3.1/../../../../arm-atollic-eabi/lib/armv7-m\libc_nano.a(lib_a-lseekr.o)
 .bss           0x00000000        0x0 c:/program files (x86)/atollic/truestudio for stm32 9.3.0/armtools/bin/../lib/gcc/arm-atollic-eabi/6.3.1/../../../../arm-atollic-eabi/lib/armv7-m\libc_nano.a(lib_a-lseekr.o)
 .text          0x00000000        0x0 c:/program files (x86)/atollic/truestudio for stm32 9.3.0/armtools/bin/../lib/gcc/arm-atollic-eabi/6.3.1/../../../../arm-atollic-eabi/lib/armv7-m\libc_nano.a(lib_a-mbtowc_r.o)
 .data          0x00000000        0x0 c:/program files (x86)/atollic/truestudio for stm32 9.3.0/armtools/bin/../lib/gcc/arm-atollic-eabi/6.3.1/../../../../arm-atollic-eabi/lib/armv7-m\libc_nano.a(lib_a-mbtowc_r.o)
 .bss           0x00000000        0x0 c:/program files (x86)/atollic/truestudio for stm32 9.3.0/armtools/bin/../lib/gcc/arm-atollic-eabi/6.3.1/../../../../arm-atollic-eabi/lib/armv7-m\libc_nano.a(lib_a-mbtowc_r.o)
 .text._mbtowc_r
                0x00000000       0x24 c:/program files (x86)/atollic/truestudio for stm32 9.3.0/armtools/bin/../lib/gcc/arm-atollic-eabi/6.3.1/../../../../arm-atollic-eabi/lib/armv7-m\libc_nano.a(lib_a-mbtowc_r.o)
 .text          0x00000000        0x0 c:/program files (x86)/atollic/truestudio for stm32 9.3.0/armtools/bin/../lib/gcc/arm-atollic-eabi/6.3.1/../../../../arm-atollic-eabi/lib/armv7-m\libc_nano.a(lib_a-memmove.o)
 .data          0x00000000        0x0 c:/program files (x86)/atollic/truestudio for stm32 9.3.0/armtools/bin/../lib/gcc/arm-atollic-eabi/6.3.1/../../../../arm-atollic-eabi/lib/armv7-m\libc_nano.a(lib_a-memmove.o)
 .bss           0x00000000        0x0 c:/program files (x86)/atollic/truestudio for stm32 9.3.0/armtools/bin/../lib/gcc/arm-atollic-eabi/6.3.1/../../../../arm-atollic-eabi/lib/armv7-m\libc_nano.a(lib_a-memmove.o)
 .text          0x00000000        0x0 c:/program files (x86)/atollic/truestudio for stm32 9.3.0/armtools/bin/../lib/gcc/arm-atollic-eabi/6.3.1/../../../../arm-atollic-eabi/lib/armv7-m\libc_nano.a(lib_a-mlock.o)
 .data          0x00000000        0x0 c:/program files (x86)/atollic/truestudio for stm32 9.3.0/armtools/bin/../lib/gcc/arm-atollic-eabi/6.3.1/../../../../arm-atollic-eabi/lib/armv7-m\libc_nano.a(lib_a-mlock.o)
 .bss           0x00000000        0x0 c:/program files (x86)/atollic/truestudio for stm32 9.3.0/armtools/bin/../lib/gcc/arm-atollic-eabi/6.3.1/../../../../arm-atollic-eabi/lib/armv7-m\libc_nano.a(lib_a-mlock.o)
 .text          0x00000000        0x0 c:/program files (x86)/atollic/truestudio for stm32 9.3.0/armtools/bin/../lib/gcc/arm-atollic-eabi/6.3.1/../../../../arm-atollic-eabi/lib/armv7-m\libc_nano.a(lib_a-nano-reallocr.o)
 .data          0x00000000        0x0 c:/program files (x86)/atollic/truestudio for stm32 9.3.0/armtools/bin/../lib/gcc/arm-atollic-eabi/6.3.1/../../../../arm-atollic-eabi/lib/armv7-m\libc_nano.a(lib_a-nano-reallocr.o)
 .bss           0x00000000        0x0 c:/program files (x86)/atollic/truestudio for stm32 9.3.0/armtools/bin/../lib/gcc/arm-atollic-eabi/6.3.1/../../../../arm-atollic-eabi/lib/armv7-m\libc_nano.a(lib_a-nano-reallocr.o)
 .text          0x00000000        0x0 c:/program files (x86)/atollic/truestudio for stm32 9.3.0/armtools/bin/../lib/gcc/arm-atollic-eabi/6.3.1/../../../../arm-atollic-eabi/lib/armv7-m\libc_nano.a(lib_a-readr.o)
 .data          0x00000000        0x0 c:/program files (x86)/atollic/truestudio for stm32 9.3.0/armtools/bin/../lib/gcc/arm-atollic-eabi/6.3.1/../../../../arm-atollic-eabi/lib/armv7-m\libc_nano.a(lib_a-readr.o)
 .bss           0x00000000        0x0 c:/program files (x86)/atollic/truestudio for stm32 9.3.0/armtools/bin/../lib/gcc/arm-atollic-eabi/6.3.1/../../../../arm-atollic-eabi/lib/armv7-m\libc_nano.a(lib_a-readr.o)
 .text          0x00000000        0x0 c:/program files (x86)/atollic/truestudio for stm32 9.3.0/armtools/bin/../lib/gcc/arm-atollic-eabi/6.3.1/../../../../arm-atollic-eabi/lib/armv7-m\libc_nano.a(lib_a-reent.o)
 .data          0x00000000        0x0 c:/program files (x86)/atollic/truestudio for stm32 9.3.0/armtools/bin/../lib/gcc/arm-atollic-eabi/6.3.1/../../../../arm-atollic-eabi/lib/armv7-m\libc_nano.a(lib_a-reent.o)
 .bss           0x00000000        0x0 c:/program files (x86)/atollic/truestudio for stm32 9.3.0/armtools/bin/../lib/gcc/arm-atollic-eabi/6.3.1/../../../../arm-atollic-eabi/lib/armv7-m\libc_nano.a(lib_a-reent.o)
 .text.cleanup_glue
                0x00000000       0x1a c:/program files (x86)/atollic/truestudio for stm32 9.3.0/armtools/bin/../lib/gcc/arm-atollic-eabi/6.3.1/../../../../arm-atollic-eabi/lib/armv7-m\libc_nano.a(lib_a-reent.o)
 .text._reclaim_reent
                0x00000000       0xb8 c:/program files (x86)/atollic/truestudio for stm32 9.3.0/armtools/bin/../lib/gcc/arm-atollic-eabi/6.3.1/../../../../arm-atollic-eabi/lib/armv7-m\libc_nano.a(lib_a-reent.o)
 .text          0x00000000       0x14 c:/program files (x86)/atollic/truestudio for stm32 9.3.0/armtools/bin/../lib/gcc/arm-atollic-eabi/6.3.1/../../../../arm-atollic-eabi/lib/armv7-m\libc_nano.a(lib_a-strcmp.o)
 .data          0x00000000        0x0 c:/program files (x86)/atollic/truestudio for stm32 9.3.0/armtools/bin/../lib/gcc/arm-atollic-eabi/6.3.1/../../../../arm-atollic-eabi/lib/armv7-m\libc_nano.a(lib_a-strcmp.o)
 .bss           0x00000000        0x0 c:/program files (x86)/atollic/truestudio for stm32 9.3.0/armtools/bin/../lib/gcc/arm-atollic-eabi/6.3.1/../../../../arm-atollic-eabi/lib/armv7-m\libc_nano.a(lib_a-strcmp.o)
 .debug_frame   0x00000000       0x20 c:/program files (x86)/atollic/truestudio for stm32 9.3.0/armtools/bin/../lib/gcc/arm-atollic-eabi/6.3.1/../../../../arm-atollic-eabi/lib/armv7-m\libc_nano.a(lib_a-strcmp.o)
 .ARM.attributes
                0x00000000       0x1b c:/program files (x86)/atollic/truestudio for stm32 9.3.0/armtools/bin/../lib/gcc/arm-atollic-eabi/6.3.1/../../../../arm-atollic-eabi/lib/armv7-m\libc_nano.a(lib_a-strcmp.o)
 .text          0x00000000        0x0 c:/program files (x86)/atollic/truestudio for stm32 9.3.0/armtools/bin/../lib/gcc/arm-atollic-eabi/6.3.1/../../../../arm-atollic-eabi/lib/armv7-m\libc_nano.a(lib_a-wctomb_r.o)
 .data          0x00000000        0x0 c:/program files (x86)/atollic/truestudio for stm32 9.3.0/armtools/bin/../lib/gcc/arm-atollic-eabi/6.3.1/../../../../arm-atollic-eabi/lib/armv7-m\libc_nano.a(lib_a-wctomb_r.o)
 .bss           0x00000000        0x0 c:/program files (x86)/atollic/truestudio for stm32 9.3.0/armtools/bin/../lib/gcc/arm-atollic-eabi/6.3.1/../../../../arm-atollic-eabi/lib/armv7-m\libc_nano.a(lib_a-wctomb_r.o)
 .text._wctomb_r
                0x00000000       0x24 c:/program files (x86)/atollic/truestudio for stm32 9.3.0/armtools/bin/../lib/gcc/arm-atollic-eabi/6.3.1/../../../../arm-atollic-eabi/lib/armv7-m\libc_nano.a(lib_a-wctomb_r.o)
 .text          0x00000000        0x0 c:/program files (x86)/atollic/truestudio for stm32 9.3.0/armtools/bin/../lib/gcc/arm-atollic-eabi/6.3.1/../../../../arm-atollic-eabi/lib/armv7-m\libc_nano.a(lib_a-ctype_.o)
 .data          0x00000000        0x0 c:/program files (x86)/atollic/truestudio for stm32 9.3.0/armtools/bin/../lib/gcc/arm-atollic-eabi/6.3.1/../../../../arm-atollic-eabi/lib/armv7-m\libc_nano.a(lib_a-ctype_.o)
 .bss           0x00000000        0x0 c:/program files (x86)/atollic/truestudio for stm32 9.3.0/armtools/bin/../lib/gcc/arm-atollic-eabi/6.3.1/../../../../arm-atollic-eabi/lib/armv7-m\libc_nano.a(lib_a-ctype_.o)
 .text          0x00000000        0x0 c:/program files (x86)/atollic/truestudio for stm32 9.3.0/armtools/bin/../lib/gcc/arm-atollic-eabi/6.3.1/../../../../arm-atollic-eabi/lib/armv7-m\libc_nano.a(lib_a-nano-msizer.o)
 .data          0x00000000        0x0 c:/program files (x86)/atollic/truestudio for stm32 9.3.0/armtools/bin/../lib/gcc/arm-atollic-eabi/6.3.1/../../../../arm-atollic-eabi/lib/armv7-m\libc_nano.a(lib_a-nano-msizer.o)
 .bss           0x00000000        0x0 c:/program files (x86)/atollic/truestudio for stm32 9.3.0/armtools/bin/../lib/gcc/arm-atollic-eabi/6.3.1/../../../../arm-atollic-eabi/lib/armv7-m\libc_nano.a(lib_a-nano-msizer.o)
 .data          0x00000000        0x0 c:/program files (x86)/atollic/truestudio for stm32 9.3.0/armtools/bin/../lib/gcc/arm-atollic-eabi/6.3.1/armv7-m\libgcc.a(_arm_addsubdf3.o)
 .bss           0x00000000        0x0 c:/program files (x86)/atollic/truestudio for stm32 9.3.0/armtools/bin/../lib/gcc/arm-atollic-eabi/6.3.1/armv7-m\libgcc.a(_arm_addsubdf3.o)
 .data          0x00000000        0x0 c:/program files (x86)/atollic/truestudio for stm32 9.3.0/armtools/bin/../lib/gcc/arm-atollic-eabi/6.3.1/armv7-m\libgcc.a(_arm_muldivdf3.o)
 .bss           0x00000000        0x0 c:/program files (x86)/atollic/truestudio for stm32 9.3.0/armtools/bin/../lib/gcc/arm-atollic-eabi/6.3.1/armv7-m\libgcc.a(_arm_muldivdf3.o)
 .data          0x00000000        0x0 c:/program files (x86)/atollic/truestudio for stm32 9.3.0/armtools/bin/../lib/gcc/arm-atollic-eabi/6.3.1/armv7-m\libgcc.a(_arm_cmpdf2.o)
 .bss           0x00000000        0x0 c:/program files (x86)/atollic/truestudio for stm32 9.3.0/armtools/bin/../lib/gcc/arm-atollic-eabi/6.3.1/armv7-m\libgcc.a(_arm_cmpdf2.o)
 .data          0x00000000        0x0 c:/program files (x86)/atollic/truestudio for stm32 9.3.0/armtools/bin/../lib/gcc/arm-atollic-eabi/6.3.1/armv7-m\libgcc.a(_arm_unorddf2.o)
 .bss           0x00000000        0x0 c:/program files (x86)/atollic/truestudio for stm32 9.3.0/armtools/bin/../lib/gcc/arm-atollic-eabi/6.3.1/armv7-m\libgcc.a(_arm_unorddf2.o)
 .data          0x00000000        0x0 c:/program files (x86)/atollic/truestudio for stm32 9.3.0/armtools/bin/../lib/gcc/arm-atollic-eabi/6.3.1/armv7-m\libgcc.a(_arm_fixdfsi.o)
 .bss           0x00000000        0x0 c:/program files (x86)/atollic/truestudio for stm32 9.3.0/armtools/bin/../lib/gcc/arm-atollic-eabi/6.3.1/armv7-m\libgcc.a(_arm_fixdfsi.o)
 .data          0x00000000        0x0 c:/program files (x86)/atollic/truestudio for stm32 9.3.0/armtools/bin/../lib/gcc/arm-atollic-eabi/6.3.1/armv7-m\libgcc.a(_arm_addsubsf3.o)
 .bss           0x00000000        0x0 c:/program files (x86)/atollic/truestudio for stm32 9.3.0/armtools/bin/../lib/gcc/arm-atollic-eabi/6.3.1/armv7-m\libgcc.a(_arm_addsubsf3.o)
 .data          0x00000000        0x0 c:/program files (x86)/atollic/truestudio for stm32 9.3.0/armtools/bin/../lib/gcc/arm-atollic-eabi/6.3.1/armv7-m\libgcc.a(_arm_cmpsf2.o)
 .bss           0x00000000        0x0 c:/program files (x86)/atollic/truestudio for stm32 9.3.0/armtools/bin/../lib/gcc/arm-atollic-eabi/6.3.1/armv7-m\libgcc.a(_arm_cmpsf2.o)
 .data          0x00000000        0x0 c:/program files (x86)/atollic/truestudio for stm32 9.3.0/armtools/bin/../lib/gcc/arm-atollic-eabi/6.3.1/armv7-m\libgcc.a(_arm_fixunssfsi.o)
 .bss           0x00000000        0x0 c:/program files (x86)/atollic/truestudio for stm32 9.3.0/armtools/bin/../lib/gcc/arm-atollic-eabi/6.3.1/armv7-m\libgcc.a(_arm_fixunssfsi.o)
 .data          0x00000000        0x0 c:/program files (x86)/atollic/truestudio for stm32 9.3.0/armtools/bin/../lib/gcc/arm-atollic-eabi/6.3.1/armv7-m\libgcc.a(_aeabi_uldivmod.o)
 .bss           0x00000000        0x0 c:/program files (x86)/atollic/truestudio for stm32 9.3.0/armtools/bin/../lib/gcc/arm-atollic-eabi/6.3.1/armv7-m\libgcc.a(_aeabi_uldivmod.o)
 .data          0x00000000        0x0 c:/program files (x86)/atollic/truestudio for stm32 9.3.0/armtools/bin/../lib/gcc/arm-atollic-eabi/6.3.1/armv7-m\libgcc.a(_udivmoddi4.o)
 .bss           0x00000000        0x0 c:/program files (x86)/atollic/truestudio for stm32 9.3.0/armtools/bin/../lib/gcc/arm-atollic-eabi/6.3.1/armv7-m\libgcc.a(_udivmoddi4.o)
 .ARM.extab     0x00000000        0x0 c:/program files (x86)/atollic/truestudio for stm32 9.3.0/armtools/bin/../lib/gcc/arm-atollic-eabi/6.3.1/armv7-m\libgcc.a(_udivmoddi4.o)
 .data          0x00000000        0x0 c:/program files (x86)/atollic/truestudio for stm32 9.3.0/armtools/bin/../lib/gcc/arm-atollic-eabi/6.3.1/armv7-m\libgcc.a(_dvmd_tls.o)
 .bss           0x00000000        0x0 c:/program files (x86)/atollic/truestudio for stm32 9.3.0/armtools/bin/../lib/gcc/arm-atollic-eabi/6.3.1/armv7-m\libgcc.a(_dvmd_tls.o)
 .text          0x00000000        0x0 c:/program files (x86)/atollic/truestudio for stm32 9.3.0/armtools/bin/../lib/gcc/arm-atollic-eabi/6.3.1/armv7-m/crtend.o
 .data          0x00000000        0x0 c:/program files (x86)/atollic/truestudio for stm32 9.3.0/armtools/bin/../lib/gcc/arm-atollic-eabi/6.3.1/armv7-m/crtend.o
 .bss           0x00000000        0x0 c:/program files (x86)/atollic/truestudio for stm32 9.3.0/armtools/bin/../lib/gcc/arm-atollic-eabi/6.3.1/armv7-m/crtend.o
 .eh_frame      0x00000000        0x4 c:/program files (x86)/atollic/truestudio for stm32 9.3.0/armtools/bin/../lib/gcc/arm-atollic-eabi/6.3.1/armv7-m/crtend.o
 .ARM.attributes
                0x00000000       0x2d c:/program files (x86)/atollic/truestudio for stm32 9.3.0/armtools/bin/../lib/gcc/arm-atollic-eabi/6.3.1/armv7-m/crtend.o
 .text          0x00000000        0x0 c:/program files (x86)/atollic/truestudio for stm32 9.3.0/armtools/bin/../lib/gcc/arm-atollic-eabi/6.3.1/armv7-m/crtn.o
 .data          0x00000000        0x0 c:/program files (x86)/atollic/truestudio for stm32 9.3.0/armtools/bin/../lib/gcc/arm-atollic-eabi/6.3.1/armv7-m/crtn.o
 .bss           0x00000000        0x0 c:/program files (x86)/atollic/truestudio for stm32 9.3.0/armtools/bin/../lib/gcc/arm-atollic-eabi/6.3.1/armv7-m/crtn.o

Memory Configuration

Name             Origin             Length             Attributes
RAM              0x20000000         0x00020000         xrw
FLASH            0x08000000         0x00040000         xr
*default*        0x00000000         0xffffffff

Linker script and memory map

LOAD c:/program files (x86)/atollic/truestudio for stm32 9.3.0/armtools/bin/../lib/gcc/arm-atollic-eabi/6.3.1/armv7-m/crti.o
LOAD c:/program files (x86)/atollic/truestudio for stm32 9.3.0/armtools/bin/../lib/gcc/arm-atollic-eabi/6.3.1/armv7-m/crtbegin.o
LOAD Drivers\STM32F2xx_HAL_Driver\Src\stm32f2xx_hal.o
LOAD Drivers\STM32F2xx_HAL_Driver\Src\stm32f2xx_hal_cortex.o
LOAD Drivers\STM32F2xx_HAL_Driver\Src\stm32f2xx_hal_dma.o
LOAD Drivers\STM32F2xx_HAL_Driver\Src\stm32f2xx_hal_dma_ex.o
LOAD Drivers\STM32F2xx_HAL_Driver\Src\stm32f2xx_hal_exti.o
LOAD Drivers\STM32F2xx_HAL_Driver\Src\stm32f2xx_hal_flash.o
LOAD Drivers\STM32F2xx_HAL_Driver\Src\stm32f2xx_hal_flash_ex.o
LOAD Drivers\STM32F2xx_HAL_Driver\Src\stm32f2xx_hal_gpio.o
LOAD Drivers\STM32F2xx_HAL_Driver\Src\stm32f2xx_hal_i2c.o
LOAD Drivers\STM32F2xx_HAL_Driver\Src\stm32f2xx_hal_pwr.o
LOAD Drivers\STM32F2xx_HAL_Driver\Src\stm32f2xx_hal_pwr_ex.o
LOAD Drivers\STM32F2xx_HAL_Driver\Src\stm32f2xx_hal_rcc.o
LOAD Drivers\STM32F2xx_HAL_Driver\Src\stm32f2xx_hal_rcc_ex.o
LOAD Drivers\STM32F2xx_HAL_Driver\Src\stm32f2xx_hal_tim.o
LOAD Drivers\STM32F2xx_HAL_Driver\Src\stm32f2xx_hal_tim_ex.o
LOAD Drivers\STM32F2xx_HAL_Driver\Src\stm32f2xx_hal_uart.o
LOAD Src\Character_lcd.o
LOAD Src\atten_ctrl.o
LOAD Src\eeprom.o
LOAD Src\main.o
LOAD Src\sth30_crc.o
LOAD Src\stm32f2xx_hal_msp.o
LOAD Src\stm32f2xx_it.o
LOAD Src\syscalls.o
LOAD Src\system_stm32f2xx.o
LOAD Src\uart.o
LOAD startup\startup_stm32f207xx.o
                0x00000080                malloc_getpagesize_P = 0x80
START GROUP
LOAD c:/program files (x86)/atollic/truestudio for stm32 9.3.0/armtools/bin/../lib/gcc/arm-atollic-eabi/6.3.1/../../../../arm-atollic-eabi/lib/armv7-m\libc_nano.a
LOAD c:/program files (x86)/atollic/truestudio for stm32 9.3.0/armtools/bin/../lib/gcc/arm-atollic-eabi/6.3.1/../../../../arm-atollic-eabi/lib/armv7-m\libm.a
END GROUP
START GROUP
LOAD c:/program files (x86)/atollic/truestudio for stm32 9.3.0/armtools/bin/../lib/gcc/arm-atollic-eabi/6.3.1/armv7-m\libgcc.a
LOAD c:/program files (x86)/atollic/truestudio for stm32 9.3.0/armtools/bin/../lib/gcc/arm-atollic-eabi/6.3.1/../../../../arm-atollic-eabi/lib/armv7-m\libc_nano.a
END GROUP
START GROUP
LOAD c:/program files (x86)/atollic/truestudio for stm32 9.3.0/armtools/bin/../lib/gcc/arm-atollic-eabi/6.3.1/armv7-m\libgcc.a
LOAD c:/program files (x86)/atollic/truestudio for stm32 9.3.0/armtools/bin/../lib/gcc/arm-atollic-eabi/6.3.1/../../../../arm-atollic-eabi/lib/armv7-m\libc_nano.a
LOAD c:/program files (x86)/atollic/truestudio for stm32 9.3.0/armtools/bin/../lib/gcc/arm-atollic-eabi/6.3.1/../../../../arm-atollic-eabi/lib/armv7-m\libnosys.a
END GROUP
START GROUP
LOAD c:/program files (x86)/atollic/truestudio for stm32 9.3.0/armtools/bin/../lib/gcc/arm-atollic-eabi/6.3.1/armv7-m\libgcc.a
LOAD c:/program files (x86)/atollic/truestudio for stm32 9.3.0/armtools/bin/../lib/gcc/arm-atollic-eabi/6.3.1/../../../../arm-atollic-eabi/lib/armv7-m\libc_nano.a
LOAD c:/program files (x86)/atollic/truestudio for stm32 9.3.0/armtools/bin/../lib/gcc/arm-atollic-eabi/6.3.1/../../../../arm-atollic-eabi/lib/armv7-m\libnosys.a
END GROUP
LOAD c:/program files (x86)/atollic/truestudio for stm32 9.3.0/armtools/bin/../lib/gcc/arm-atollic-eabi/6.3.1/armv7-m/crtend.o
LOAD c:/program files (x86)/atollic/truestudio for stm32 9.3.0/armtools/bin/../lib/gcc/arm-atollic-eabi/6.3.1/armv7-m/crtn.o
                0x20020000                _estack = 0x20020000
                0x00000200                _Min_Heap_Size = 0x200
                0x00000400                _Min_Stack_Size = 0x400

.isr_vector     0x08000000      0x184
                0x08000000                . = ALIGN (0x4)
 *(.isr_vector)
 .isr_vector    0x08000000      0x184 startup\startup_stm32f207xx.o
                0x08000000                g_pfnVectors
                0x08000184                . = ALIGN (0x4)

.text           0x08000188     0xb98c
                0x08000188                . = ALIGN (0x4)
 *(.text)
 .text          0x08000188       0x40 c:/program files (x86)/atollic/truestudio for stm32 9.3.0/armtools/bin/../lib/gcc/arm-atollic-eabi/6.3.1/armv7-m/crtbegin.o
 .text          0x080001c8       0x10 c:/program files (x86)/atollic/truestudio for stm32 9.3.0/armtools/bin/../lib/gcc/arm-atollic-eabi/6.3.1/../../../../arm-atollic-eabi/lib/armv7-m\libc_nano.a(lib_a-strlen.o)
                0x080001c8                strlen
 .text          0x080001d8      0x370 c:/program files (x86)/atollic/truestudio for stm32 9.3.0/armtools/bin/../lib/gcc/arm-atollic-eabi/6.3.1/armv7-m\libgcc.a(_arm_addsubdf3.o)
                0x080001d8                __aeabi_drsub
                0x080001e0                __aeabi_dsub
                0x080001e0                __subdf3
                0x080001e4                __aeabi_dadd
                0x080001e4                __adddf3
                0x0800045c                __floatunsidf
                0x0800045c                __aeabi_ui2d
                0x0800047c                __floatsidf
                0x0800047c                __aeabi_i2d
                0x080004a0                __aeabi_f2d
                0x080004a0                __extendsfdf2
                0x080004dc                __floatundidf
                0x080004dc                __aeabi_ul2d
                0x080004ec                __floatdidf
                0x080004ec                __aeabi_l2d
 .text          0x08000548      0x424 c:/program files (x86)/atollic/truestudio for stm32 9.3.0/armtools/bin/../lib/gcc/arm-atollic-eabi/6.3.1/armv7-m\libgcc.a(_arm_muldivdf3.o)
                0x08000548                __aeabi_dmul
                0x08000548                __muldf3
                0x0800079c                __divdf3
                0x0800079c                __aeabi_ddiv
 .text          0x0800096c      0x110 c:/program files (x86)/atollic/truestudio for stm32 9.3.0/armtools/bin/../lib/gcc/arm-atollic-eabi/6.3.1/armv7-m\libgcc.a(_arm_cmpdf2.o)
                0x0800096c                __gtdf2
                0x0800096c                __gedf2
                0x08000974                __ltdf2
                0x08000974                __ledf2
                0x0800097c                __nedf2
                0x0800097c                __eqdf2
                0x0800097c                __cmpdf2
                0x080009f8                __aeabi_cdrcmple
                0x08000a08                __aeabi_cdcmpeq
                0x08000a08                __aeabi_cdcmple
                0x08000a18                __aeabi_dcmpeq
                0x08000a2c                __aeabi_dcmplt
                0x08000a40                __aeabi_dcmple
                0x08000a54                __aeabi_dcmpge
                0x08000a68                __aeabi_dcmpgt
 .text          0x08000a7c       0x2c c:/program files (x86)/atollic/truestudio for stm32 9.3.0/armtools/bin/../lib/gcc/arm-atollic-eabi/6.3.1/armv7-m\libgcc.a(_arm_unorddf2.o)
                0x08000a7c                __unorddf2
                0x08000a7c                __aeabi_dcmpun
 .text          0x08000aa8       0x50 c:/program files (x86)/atollic/truestudio for stm32 9.3.0/armtools/bin/../lib/gcc/arm-atollic-eabi/6.3.1/armv7-m\libgcc.a(_arm_fixdfsi.o)
                0x08000aa8                __aeabi_d2iz
                0x08000aa8                __fixdfsi
 .text          0x08000af8      0x21c c:/program files (x86)/atollic/truestudio for stm32 9.3.0/armtools/bin/../lib/gcc/arm-atollic-eabi/6.3.1/armv7-m\libgcc.a(_arm_addsubsf3.o)
                0x08000af8                __aeabi_frsub
                0x08000b00                __subsf3
                0x08000b00                __aeabi_fsub
                0x08000b04                __aeabi_fadd
                0x08000b04                __addsf3
                0x08000c64                __aeabi_ui2f
                0x08000c64                __floatunsisf
                0x08000c6c                __aeabi_i2f
                0x08000c6c                __floatsisf
                0x08000c88                __aeabi_ul2f
                0x08000c88                __floatundisf
                0x08000c98                __aeabi_l2f
                0x08000c98                __floatdisf
 .text          0x08000d14       0xec c:/program files (x86)/atollic/truestudio for stm32 9.3.0/armtools/bin/../lib/gcc/arm-atollic-eabi/6.3.1/armv7-m\libgcc.a(_arm_cmpsf2.o)
                0x08000d14                __gesf2
                0x08000d14                __gtsf2
                0x08000d1c                __lesf2
                0x08000d1c                __ltsf2
                0x08000d24                __nesf2
                0x08000d24                __eqsf2
                0x08000d24                __cmpsf2
                0x08000d84                __aeabi_cfrcmple
                0x08000d8c                __aeabi_cfcmpeq
                0x08000d8c                __aeabi_cfcmple
                0x08000d9c                __aeabi_fcmpeq
                0x08000db0                __aeabi_fcmplt
                0x08000dc4                __aeabi_fcmple
                0x08000dd8                __aeabi_fcmpge
                0x08000dec                __aeabi_fcmpgt
 .text          0x08000e00       0x40 c:/program files (x86)/atollic/truestudio for stm32 9.3.0/armtools/bin/../lib/gcc/arm-atollic-eabi/6.3.1/armv7-m\libgcc.a(_arm_fixunssfsi.o)
                0x08000e00                __fixunssfsi
                0x08000e00                __aeabi_f2uiz
 .text          0x08000e40       0x30 c:/program files (x86)/atollic/truestudio for stm32 9.3.0/armtools/bin/../lib/gcc/arm-atollic-eabi/6.3.1/armv7-m\libgcc.a(_aeabi_uldivmod.o)
                0x08000e40                __aeabi_uldivmod
 .text          0x08000e70      0x2dc c:/program files (x86)/atollic/truestudio for stm32 9.3.0/armtools/bin/../lib/gcc/arm-atollic-eabi/6.3.1/armv7-m\libgcc.a(_udivmoddi4.o)
                0x08000e70                __udivmoddi4
 .text          0x0800114c        0x4 c:/program files (x86)/atollic/truestudio for stm32 9.3.0/armtools/bin/../lib/gcc/arm-atollic-eabi/6.3.1/armv7-m\libgcc.a(_dvmd_tls.o)
                0x0800114c                __aeabi_idiv0
                0x0800114c                __aeabi_ldiv0
 *(.text*)
 .text.HAL_InitTick
                0x08001150       0x48 Drivers\STM32F2xx_HAL_Driver\Src\stm32f2xx_hal.o
                0x08001150                HAL_InitTick
 .text.HAL_Init
                0x08001198       0x34 Drivers\STM32F2xx_HAL_Driver\Src\stm32f2xx_hal.o
                0x08001198                HAL_Init
 .text.HAL_IncTick
                0x080011cc       0x18 Drivers\STM32F2xx_HAL_Driver\Src\stm32f2xx_hal.o
                0x080011cc                HAL_IncTick
 .text.HAL_GetTick
                0x080011e4        0xc Drivers\STM32F2xx_HAL_Driver\Src\stm32f2xx_hal.o
                0x080011e4                HAL_GetTick
 .text.HAL_Delay
                0x080011f0       0x28 Drivers\STM32F2xx_HAL_Driver\Src\stm32f2xx_hal.o
                0x080011f0                HAL_Delay
 .text.HAL_NVIC_SetPriorityGrouping
                0x08001218       0x24 Drivers\STM32F2xx_HAL_Driver\Src\stm32f2xx_hal_cortex.o
                0x08001218                HAL_NVIC_SetPriorityGrouping
 .text.HAL_NVIC_SetPriority
                0x0800123c       0x68 Drivers\STM32F2xx_HAL_Driver\Src\stm32f2xx_hal_cortex.o
                0x0800123c                HAL_NVIC_SetPriority
 .text.HAL_NVIC_EnableIRQ
                0x080012a4       0x1c Drivers\STM32F2xx_HAL_Driver\Src\stm32f2xx_hal_cortex.o
                0x080012a4                HAL_NVIC_EnableIRQ
 .text.HAL_SYSTICK_Config
                0x080012c0       0x2c Drivers\STM32F2xx_HAL_Driver\Src\stm32f2xx_hal_cortex.o
                0x080012c0                HAL_SYSTICK_Config
 .text.DMA_CalcBaseAndBitshift
                0x080012ec       0x2c Drivers\STM32F2xx_HAL_Driver\Src\stm32f2xx_hal_dma.o
 .text.HAL_DMA_Init
                0x08001318       0xfc Drivers\STM32F2xx_HAL_Driver\Src\stm32f2xx_hal_dma.o
                0x08001318                HAL_DMA_Init
 .text.HAL_DMA_Start_IT
                0x08001414       0x76 Drivers\STM32F2xx_HAL_Driver\Src\stm32f2xx_hal_dma.o
                0x08001414                HAL_DMA_Start_IT
 .text.HAL_DMA_Abort_IT
                0x0800148a       0x24 Drivers\STM32F2xx_HAL_Driver\Src\stm32f2xx_hal_dma.o
                0x0800148a                HAL_DMA_Abort_IT
 *fill*         0x080014ae        0x2 
 .text.HAL_DMA_IRQHandler
                0x080014b0      0x174 Drivers\STM32F2xx_HAL_Driver\Src\stm32f2xx_hal_dma.o
                0x080014b0                HAL_DMA_IRQHandler
 .text.HAL_GPIO_Init
                0x08001624      0x1c4 Drivers\STM32F2xx_HAL_Driver\Src\stm32f2xx_hal_gpio.o
                0x08001624                HAL_GPIO_Init
 .text.HAL_GPIO_ReadPin
                0x080017e8        0xc Drivers\STM32F2xx_HAL_Driver\Src\stm32f2xx_hal_gpio.o
                0x080017e8                HAL_GPIO_ReadPin
 .text.HAL_GPIO_WritePin
                0x080017f4        0xa Drivers\STM32F2xx_HAL_Driver\Src\stm32f2xx_hal_gpio.o
                0x080017f4                HAL_GPIO_WritePin
 .text.HAL_GPIO_TogglePin
                0x080017fe        0xc Drivers\STM32F2xx_HAL_Driver\Src\stm32f2xx_hal_gpio.o
                0x080017fe                HAL_GPIO_TogglePin
 *fill*         0x0800180a        0x2 
 .text.HAL_GPIO_EXTI_IRQHandler
                0x0800180c       0x18 Drivers\STM32F2xx_HAL_Driver\Src\stm32f2xx_hal_gpio.o
                0x0800180c                HAL_GPIO_EXTI_IRQHandler
 .text.I2C_IsAcknowledgeFailed
                0x08001824       0x32 Drivers\STM32F2xx_HAL_Driver\Src\stm32f2xx_hal_i2c.o
 .text.I2C_WaitOnMasterAddressFlagUntilTimeout
                0x08001856       0x8a Drivers\STM32F2xx_HAL_Driver\Src\stm32f2xx_hal_i2c.o
 .text.I2C_WaitOnBTFFlagUntilTimeout
                0x080018e0       0x4c Drivers\STM32F2xx_HAL_Driver\Src\stm32f2xx_hal_i2c.o
 .text.I2C_WaitOnRXNEFlagUntilTimeout
                0x0800192c       0x5e Drivers\STM32F2xx_HAL_Driver\Src\stm32f2xx_hal_i2c.o
 .text.I2C_WaitOnFlagUntilTimeout
                0x0800198a       0x64 Drivers\STM32F2xx_HAL_Driver\Src\stm32f2xx_hal_i2c.o
 .text.I2C_WaitOnTXEFlagUntilTimeout
                0x080019ee       0x4c Drivers\STM32F2xx_HAL_Driver\Src\stm32f2xx_hal_i2c.o
 *fill*         0x08001a3a        0x2 
 .text.I2C_RequestMemoryWrite
                0x08001a3c       0x9c Drivers\STM32F2xx_HAL_Driver\Src\stm32f2xx_hal_i2c.o
 .text.I2C_RequestMemoryRead
                0x08001ad8       0xec Drivers\STM32F2xx_HAL_Driver\Src\stm32f2xx_hal_i2c.o
 .text.HAL_I2C_Init
                0x08001bc4      0x148 Drivers\STM32F2xx_HAL_Driver\Src\stm32f2xx_hal_i2c.o
                0x08001bc4                HAL_I2C_Init
 .text.HAL_I2C_Mem_Write
                0x08001d0c      0x120 Drivers\STM32F2xx_HAL_Driver\Src\stm32f2xx_hal_i2c.o
                0x08001d0c                HAL_I2C_Mem_Write
 .text.HAL_I2C_Mem_Read
                0x08001e2c      0x218 Drivers\STM32F2xx_HAL_Driver\Src\stm32f2xx_hal_i2c.o
                0x08001e2c                HAL_I2C_Mem_Read
 .text.HAL_RCC_OscConfig
                0x08002044      0x344 Drivers\STM32F2xx_HAL_Driver\Src\stm32f2xx_hal_rcc.o
                0x08002044                HAL_RCC_OscConfig
 .text.HAL_RCC_GetSysClockFreq
                0x08002388       0x5c Drivers\STM32F2xx_HAL_Driver\Src\stm32f2xx_hal_rcc.o
                0x08002388                HAL_RCC_GetSysClockFreq
 .text.HAL_RCC_ClockConfig
                0x080023e4      0x140 Drivers\STM32F2xx_HAL_Driver\Src\stm32f2xx_hal_rcc.o
                0x080023e4                HAL_RCC_ClockConfig
 .text.HAL_RCC_GetPCLK1Freq
                0x08002524       0x30 Drivers\STM32F2xx_HAL_Driver\Src\stm32f2xx_hal_rcc.o
                0x08002524                HAL_RCC_GetPCLK1Freq
 .text.HAL_RCC_GetPCLK2Freq
                0x08002554       0x30 Drivers\STM32F2xx_HAL_Driver\Src\stm32f2xx_hal_rcc.o
                0x08002554                HAL_RCC_GetPCLK2Freq
 .text.HAL_TIM_Base_Start_IT
                0x08002584       0x20 Drivers\STM32F2xx_HAL_Driver\Src\stm32f2xx_hal_tim.o
                0x08002584                HAL_TIM_Base_Start_IT
 .text.HAL_TIM_OC_DelayElapsedCallback
                0x080025a4        0x2 Drivers\STM32F2xx_HAL_Driver\Src\stm32f2xx_hal_tim.o
                0x080025a4                HAL_TIM_OC_DelayElapsedCallback
 .text.HAL_TIM_IC_CaptureCallback
                0x080025a6        0x2 Drivers\STM32F2xx_HAL_Driver\Src\stm32f2xx_hal_tim.o
                0x080025a6                HAL_TIM_IC_CaptureCallback
 .text.HAL_TIM_PWM_PulseFinishedCallback
                0x080025a8        0x2 Drivers\STM32F2xx_HAL_Driver\Src\stm32f2xx_hal_tim.o
                0x080025a8                HAL_TIM_PWM_PulseFinishedCallback
 .text.HAL_TIM_TriggerCallback
                0x080025aa        0x2 Drivers\STM32F2xx_HAL_Driver\Src\stm32f2xx_hal_tim.o
                0x080025aa                HAL_TIM_TriggerCallback
 .text.HAL_TIM_IRQHandler
                0x080025ac      0x144 Drivers\STM32F2xx_HAL_Driver\Src\stm32f2xx_hal_tim.o
                0x080025ac                HAL_TIM_IRQHandler
 .text.TIM_Base_SetConfig
                0x080026f0       0xcc Drivers\STM32F2xx_HAL_Driver\Src\stm32f2xx_hal_tim.o
                0x080026f0                TIM_Base_SetConfig
 .text.HAL_TIM_Base_Init
                0x080027bc       0x34 Drivers\STM32F2xx_HAL_Driver\Src\stm32f2xx_hal_tim.o
                0x080027bc                HAL_TIM_Base_Init
 .text.HAL_TIMEx_MasterConfigSynchronization
                0x080027f0       0x3c Drivers\STM32F2xx_HAL_Driver\Src\stm32f2xx_hal_tim_ex.o
                0x080027f0                HAL_TIMEx_MasterConfigSynchronization
 .text.HAL_TIMEx_CommutCallback
                0x0800282c        0x2 Drivers\STM32F2xx_HAL_Driver\Src\stm32f2xx_hal_tim_ex.o
                0x0800282c                HAL_TIMEx_CommutCallback
 .text.HAL_TIMEx_BreakCallback
                0x0800282e        0x2 Drivers\STM32F2xx_HAL_Driver\Src\stm32f2xx_hal_tim_ex.o
                0x0800282e                HAL_TIMEx_BreakCallback
 .text.UART_EndRxTransfer
                0x08002830       0x1a Drivers\STM32F2xx_HAL_Driver\Src\stm32f2xx_hal_uart.o
 *fill*         0x0800284a        0x2 
 .text.UART_SetConfig
                0x0800284c       0xd0 Drivers\STM32F2xx_HAL_Driver\Src\stm32f2xx_hal_uart.o
 .text.UART_WaitOnFlagUntilTimeout.constprop.3
                0x0800291c       0x50 Drivers\STM32F2xx_HAL_Driver\Src\stm32f2xx_hal_uart.o
 .text.HAL_UART_Init
                0x0800296c       0x5c Drivers\STM32F2xx_HAL_Driver\Src\stm32f2xx_hal_uart.o
                0x0800296c                HAL_UART_Init
 .text.HAL_UART_Transmit
                0x080029c8       0xb8 Drivers\STM32F2xx_HAL_Driver\Src\stm32f2xx_hal_uart.o
                0x080029c8                HAL_UART_Transmit
 .text.HAL_UART_Transmit_DMA
                0x08002a80       0x74 Drivers\STM32F2xx_HAL_Driver\Src\stm32f2xx_hal_uart.o
                0x08002a80                HAL_UART_Transmit_DMA
 .text.HAL_UART_Receive_DMA
                0x08002af4       0x90 Drivers\STM32F2xx_HAL_Driver\Src\stm32f2xx_hal_uart.o
                0x08002af4                HAL_UART_Receive_DMA
 .text.HAL_UART_TxCpltCallback
                0x08002b84        0x2 Drivers\STM32F2xx_HAL_Driver\Src\stm32f2xx_hal_uart.o
                0x08002b84                HAL_UART_TxCpltCallback
 .text.UART_DMATransmitCplt
                0x08002b86       0x2c Drivers\STM32F2xx_HAL_Driver\Src\stm32f2xx_hal_uart.o
 .text.HAL_UART_TxHalfCpltCallback
                0x08002bb2        0x2 Drivers\STM32F2xx_HAL_Driver\Src\stm32f2xx_hal_uart.o
                0x08002bb2                HAL_UART_TxHalfCpltCallback
 .text.UART_DMATxHalfCplt
                0x08002bb4        0xa Drivers\STM32F2xx_HAL_Driver\Src\stm32f2xx_hal_uart.o
 .text.UART_DMAReceiveCplt
                0x08002bbe       0x38 Drivers\STM32F2xx_HAL_Driver\Src\stm32f2xx_hal_uart.o
 .text.UART_Receive_IT
                0x08002bf6       0x7c Drivers\STM32F2xx_HAL_Driver\Src\stm32f2xx_hal_uart.o
 .text.HAL_UART_RxHalfCpltCallback
                0x08002c72        0x2 Drivers\STM32F2xx_HAL_Driver\Src\stm32f2xx_hal_uart.o
                0x08002c72                HAL_UART_RxHalfCpltCallback
 .text.UART_DMARxHalfCplt
                0x08002c74        0xa Drivers\STM32F2xx_HAL_Driver\Src\stm32f2xx_hal_uart.o
 .text.HAL_UART_ErrorCallback
                0x08002c7e        0x2 Drivers\STM32F2xx_HAL_Driver\Src\stm32f2xx_hal_uart.o
                0x08002c7e                HAL_UART_ErrorCallback
 .text.UART_DMAError
                0x08002c80       0x4e Drivers\STM32F2xx_HAL_Driver\Src\stm32f2xx_hal_uart.o
 *fill*         0x08002cce        0x2 
 .text.HAL_UART_IRQHandler
                0x08002cd0      0x140 Drivers\STM32F2xx_HAL_Driver\Src\stm32f2xx_hal_uart.o
                0x08002cd0                HAL_UART_IRQHandler
 .text.UART_DMAAbortOnError
                0x08002e10       0x10 Drivers\STM32F2xx_HAL_Driver\Src\stm32f2xx_hal_uart.o
 .text.ButtonDataSet
                0x08002e20        0xc Src\Character_lcd.o
                0x08002e20                ButtonDataSet
 .text.ButtonDataGet
                0x08002e2c        0xc Src\Character_lcd.o
                0x08002e2c                ButtonDataGet
 .text.LCD_M68_Data_Save_150M
                0x08002e38        0xe Src\Character_lcd.o
                0x08002e38                LCD_M68_Data_Save_150M
 .text.LCD_M68_Data_Save_Wifi
                0x08002e46       0x40 Src\Character_lcd.o
                0x08002e46                LCD_M68_Data_Save_Wifi
 .text.LCD_M68_Data_Save_30G
                0x08002e86       0x30 Src\Character_lcd.o
                0x08002e86                LCD_M68_Data_Save_30G
 *fill*         0x08002eb6        0x2 
 .text.Data_Freq_LoadFunc
                0x08002eb8       0xec Src\Character_lcd.o
                0x08002eb8                Data_Freq_LoadFunc
 .text.LCD_Str_Filter
                0x08002fa4       0x10 Src\Character_lcd.o
                0x08002fa4                LCD_Str_Filter
 .text.LCD_M68_DataWrite_COMMAND2
                0x08002fb4      0x17c Src\Character_lcd.o
                0x08002fb4                LCD_M68_DataWrite_COMMAND2
 .text.LCD_M68_DataWrite_COMMAND_Init
                0x08003130      0x31c Src\Character_lcd.o
                0x08003130                LCD_M68_DataWrite_COMMAND_Init
 .text.LCD_M68_DataWrite_COMMAND_Cusor_ON
                0x0800344c        0xa Src\Character_lcd.o
                0x0800344c                LCD_M68_DataWrite_COMMAND_Cusor_ON
 .text.LCD_M68_DataWrite_COMMAND_Cusor_OFF
                0x08003456        0xa Src\Character_lcd.o
                0x08003456                LCD_M68_DataWrite_COMMAND_Cusor_OFF
 .text.LCD_M68_DataWrite_Clear
                0x08003460        0xa Src\Character_lcd.o
                0x08003460                LCD_M68_DataWrite_Clear
 .text.LCD_M68_DataWrite_LineChage
                0x0800346a       0x10 Src\Character_lcd.o
                0x0800346a                LCD_M68_DataWrite_LineChage
 *fill*         0x0800347a        0x2 
 .text.LCD_M68_DataWrite_COMMAND
                0x0800347c      0x1c8 Src\Character_lcd.o
                0x0800347c                LCD_M68_DataWrite_COMMAND
 .text.Layer_Get
                0x08003644        0xc Src\Character_lcd.o
                0x08003644                Layer_Get
 .text.Lcd_AchSetting_Display
                0x08003650       0x4c Src\Character_lcd.o
                0x08003650                Lcd_AchSetting_Display
 .text.Lcd_Ach150M_Display
                0x0800369c       0x5c Src\Character_lcd.o
                0x0800369c                Lcd_Ach150M_Display
 .text.Lcd_AchWifi_Display
                0x080036f8       0x64 Src\Character_lcd.o
                0x080036f8                Lcd_AchWifi_Display
 .text.Lcd_Ach30G_Display
                0x0800375c       0x5c Src\Character_lcd.o
                0x0800375c                Lcd_Ach30G_Display
 .text.Lcd_BchSetting_Display
                0x080037b8       0x4c Src\Character_lcd.o
                0x080037b8                Lcd_BchSetting_Display
 .text.Lcd_Bch150M_Display
                0x08003804       0x5c Src\Character_lcd.o
                0x08003804                Lcd_Bch150M_Display
 .text.Lcd_BchWifi_Display
                0x08003860       0x64 Src\Character_lcd.o
                0x08003860                Lcd_BchWifi_Display
 .text.Lcd_Bch30G_Display
                0x080038c4       0x5c Src\Character_lcd.o
                0x080038c4                Lcd_Bch30G_Display
 .text.LCD_150M_ValueChange_Display
                0x08003920       0x68 Src\Character_lcd.o
                0x08003920                LCD_150M_ValueChange_Display
 .text.LCD_Wifi_ValueChange_Display
                0x08003988       0x68 Src\Character_lcd.o
                0x08003988                LCD_Wifi_ValueChange_Display
 .text.LCD_30G_ValueChange_Display
                0x080039f0       0x68 Src\Character_lcd.o
                0x080039f0                LCD_30G_ValueChange_Display
 .text.LCD_Wifi_Freq_Select_Display
                0x08003a58       0x80 Src\Character_lcd.o
                0x08003a58                LCD_Wifi_Freq_Select_Display
 .text.LCD_30G_Freq_Select_Display
                0x08003ad8       0xb4 Src\Character_lcd.o
                0x08003ad8                LCD_30G_Freq_Select_Display
 .text.Character_Lcd_chMenu
                0x08003b8c      0x6e8 Src\Character_lcd.o
                0x08003b8c                Character_Lcd_chMenu
 .text.Atten_PE43711_TraceValue_Func
                0x08004274       0x8c Src\atten_ctrl.o
                0x08004274                Atten_PE43711_TraceValue_Func
 .text.Atten_QPC6614_TraceValue_Func
                0x08004300       0x90 Src\atten_ctrl.o
                0x08004300                Atten_QPC6614_TraceValue_Func
 .text.Atten_ADRF5720_TraceValue_Func
                0x08004390       0x90 Src\atten_ctrl.o
                0x08004390                Atten_ADRF5720_TraceValue_Func
 .text.Atten_HMC939_TraceValue_Func
                0x08004420       0x84 Src\atten_ctrl.o
                0x08004420                Atten_HMC939_TraceValue_Func
 .text.PE43711_Atten_Rx_DataCheck
                0x080044a4       0xdc Src\atten_ctrl.o
                0x080044a4                PE43711_Atten_Rx_DataCheck
 .text.QPC6614_Atten_Rx_DataCheck
                0x08004580       0xe0 Src\atten_ctrl.o
                0x08004580                QPC6614_Atten_Rx_DataCheck
 .text.ADRF5720_Atten_Rx_DataCheck
                0x08004660       0xe8 Src\atten_ctrl.o
                0x08004660                ADRF5720_Atten_Rx_DataCheck
 .text.HMC939_Atten_Rx_DataCheck
                0x08004748       0x54 Src\atten_ctrl.o
                0x08004748                HMC939_Atten_Rx_DataCheck
 .text.Atten_150M_DataSet
                0x0800479c       0x60 Src\atten_ctrl.o
                0x0800479c                Atten_150M_DataSet
 .text.Atten_Wifi_DataSet
                0x080047fc       0xe8 Src\atten_ctrl.o
                0x080047fc                Atten_Wifi_DataSet
 .text.Atten_30G_DataSet
                0x080048e4       0xc0 Src\atten_ctrl.o
                0x080048e4                Atten_30G_DataSet
 .text.PE43711_Ach_atten_ctrl
                0x080049a4       0xd0 Src\atten_ctrl.o
                0x080049a4                PE43711_Ach_atten_ctrl
 .text.PE43711_Bch_atten_ctrl
                0x08004a74       0xe8 Src\atten_ctrl.o
                0x08004a74                PE43711_Bch_atten_ctrl
 .text.QPC6614_Ach_atten_ctrl
                0x08004b5c       0xb8 Src\atten_ctrl.o
                0x08004b5c                QPC6614_Ach_atten_ctrl
 .text.QPC6614_Bch_atten_ctrl
                0x08004c14       0xc4 Src\atten_ctrl.o
                0x08004c14                QPC6614_Bch_atten_ctrl
 .text.ADRF5720_Ach_atten_ctrl
                0x08004cd8       0xac Src\atten_ctrl.o
                0x08004cd8                ADRF5720_Ach_atten_ctrl
 .text.ADRF5720_Bch_atten_ctrl
                0x08004d84       0xa4 Src\atten_ctrl.o
                0x08004d84                ADRF5720_Bch_atten_ctrl
 .text.HMC939_Ach_atten_ctrl
                0x08004e28       0xa8 Src\atten_ctrl.o
                0x08004e28                HMC939_Ach_atten_ctrl
 .text.HMC939_Bch_atten_ctrl
                0x08004ed0       0xa8 Src\atten_ctrl.o
                0x08004ed0                HMC939_Bch_atten_ctrl
 .text.Atten_Alarm_Read
                0x08004f78       0x68 Src\atten_ctrl.o
                0x08004f78                Atten_Alarm_Read
 .text.Alarm_Operate
                0x08004fe0       0x9c Src\atten_ctrl.o
                0x08004fe0                Alarm_Operate
 .text.Uart_Data_Send
                0x0800507c       0x10 Src\atten_ctrl.o
                0x0800507c                Uart_Data_Send
 .text.Atten_Table_Read.constprop.0
                0x0800508c       0x5c Src\atten_ctrl.o
 .text.Atten_Offset_QPC6614
                0x080050e8      0x210 Src\atten_ctrl.o
                0x080050e8                Atten_Offset_QPC6614
 .text.Atten_Offset_PE43711
                0x080052f8      0x2d0 Src\atten_ctrl.o
                0x080052f8                Atten_Offset_PE43711
 .text.Atten_Offset_ADRF5720
                0x080055c8      0x1f0 Src\atten_ctrl.o
                0x080055c8                Atten_Offset_ADRF5720
 .text.Atten_Offset_HMC939
                0x080057b8      0x10c Src\atten_ctrl.o
                0x080057b8                Atten_Offset_HMC939
 .text.Atten_Init
                0x080058c4       0x88 Src\atten_ctrl.o
                0x080058c4                Atten_Init
 .text.Atten_Operate
                0x0800594c      0xd70 Src\atten_ctrl.o
                0x0800594c                Atten_Operate
 .text.Atten_Operate_Mem_RW
                0x080066bc     0x17fc Src\atten_ctrl.o
                0x080066bc                Atten_Operate_Mem_RW
 .text.EEPROM_IM24CM01P_write
                0x08007eb8       0x28 Src\eeprom.o
                0x08007eb8                EEPROM_IM24CM01P_write
 .text.EEPROM_IM24CM01P_Read
                0x08007ee0       0x28 Src\eeprom.o
                0x08007ee0                EEPROM_IM24CM01P_Read
 .text.EEPROM_IM24CM01P_Init
                0x08007f08      0x434 Src\eeprom.o
                0x08007f08                EEPROM_IM24CM01P_Init
 .text._write   0x0800833c       0x14 Src\main.o
                0x0800833c                _write
 .text.HAL_TIM_PeriodElapsedCallback
                0x08008350       0x48 Src\main.o
                0x08008350                HAL_TIM_PeriodElapsedCallback
 .text.HAL_UART_RxCpltCallback
                0x08008398       0x54 Src\main.o
                0x08008398                HAL_UART_RxCpltCallback
 .text.HAL_GPIO_EXTI_Callback
                0x080083ec       0xc8 Src\main.o
                0x080083ec                HAL_GPIO_EXTI_Callback
 .text.SystemClock_Config
                0x080084b4       0x5c Src\main.o
                0x080084b4                SystemClock_Config
 .text.startup.main
                0x08008510      0x540 Src\main.o
                0x08008510                main
 .text.Error_Handler
                0x08008a50        0x2 Src\main.o
                0x08008a50                Error_Handler
 .text.STH30_CreateCrc
                0x08008a52       0x36 Src\sth30_crc.o
                0x08008a52                STH30_CreateCrc
 .text.STH30_CheckCrc
                0x08008a88       0x3a Src\sth30_crc.o
                0x08008a88                STH30_CheckCrc
 *fill*         0x08008ac2        0x2 
 .text.HAL_MspInit
                0x08008ac4       0x38 Src\stm32f2xx_hal_msp.o
                0x08008ac4                HAL_MspInit
 .text.HAL_I2C_MspInit
                0x08008afc       0xb0 Src\stm32f2xx_hal_msp.o
                0x08008afc                HAL_I2C_MspInit
 .text.HAL_TIM_Base_MspInit
                0x08008bac       0x30 Src\stm32f2xx_hal_msp.o
                0x08008bac                HAL_TIM_Base_MspInit
 .text.HAL_UART_MspInit
                0x08008bdc       0xe4 Src\stm32f2xx_hal_msp.o
                0x08008bdc                HAL_UART_MspInit
 .text.NMI_Handler
                0x08008cc0        0x2 Src\stm32f2xx_it.o
                0x08008cc0                NMI_Handler
 .text.HardFault_Handler
                0x08008cc2        0x2 Src\stm32f2xx_it.o
                0x08008cc2                HardFault_Handler
 .text.MemManage_Handler
                0x08008cc4        0x2 Src\stm32f2xx_it.o
                0x08008cc4                MemManage_Handler
 .text.BusFault_Handler
                0x08008cc6        0x2 Src\stm32f2xx_it.o
                0x08008cc6                BusFault_Handler
 .text.UsageFault_Handler
                0x08008cc8        0x2 Src\stm32f2xx_it.o
                0x08008cc8                UsageFault_Handler
 .text.SVC_Handler
                0x08008cca        0x2 Src\stm32f2xx_it.o
                0x08008cca                SVC_Handler
 .text.DebugMon_Handler
                0x08008ccc        0x2 Src\stm32f2xx_it.o
                0x08008ccc                DebugMon_Handler
 .text.PendSV_Handler
                0x08008cce        0x2 Src\stm32f2xx_it.o
                0x08008cce                PendSV_Handler
 .text.SysTick_Handler
                0x08008cd0        0x4 Src\stm32f2xx_it.o
                0x08008cd0                SysTick_Handler
 .text.DMA1_Stream1_IRQHandler
                0x08008cd4        0xc Src\stm32f2xx_it.o
                0x08008cd4                DMA1_Stream1_IRQHandler
 .text.DMA1_Stream4_IRQHandler
                0x08008ce0        0xc Src\stm32f2xx_it.o
                0x08008ce0                DMA1_Stream4_IRQHandler
 .text.EXTI9_5_IRQHandler
                0x08008cec        0x8 Src\stm32f2xx_it.o
                0x08008cec                EXTI9_5_IRQHandler
 .text.USART3_IRQHandler
                0x08008cf4        0xc Src\stm32f2xx_it.o
                0x08008cf4                USART3_IRQHandler
 .text.EXTI15_10_IRQHandler
                0x08008d00       0x26 Src\stm32f2xx_it.o
                0x08008d00                EXTI15_10_IRQHandler
 *fill*         0x08008d26        0x2 
 .text.TIM6_DAC_IRQHandler
                0x08008d28        0xc Src\stm32f2xx_it.o
                0x08008d28                TIM6_DAC_IRQHandler
 .text._read    0x08008d34       0x1c Src\syscalls.o
                0x08008d34                _read
 .text._sbrk    0x08008d50       0x34 Src\syscalls.o
                0x08008d50                _sbrk
 .text._close   0x08008d84        0x6 Src\syscalls.o
                0x08008d84                _close
 .text._fstat   0x08008d8a        0xa Src\syscalls.o
                0x08008d8a                _fstat
 .text._isatty  0x08008d94        0x4 Src\syscalls.o
                0x08008d94                _isatty
 .text._lseek   0x08008d98        0x4 Src\syscalls.o
                0x08008d98                _lseek
 .text.SystemInit
                0x08008d9c       0x40 Src\system_stm32f2xx.o
                0x08008d9c                SystemInit
 .text.InitUartQueue
                0x08008ddc        0xa Src\uart.o
                0x08008ddc                InitUartQueue
 *fill*         0x08008de6        0x2 
 .text.Reset_Handler
                0x08008de8       0x50 startup\startup_stm32f207xx.o
                0x08008de8                Reset_Handler
 .text.Default_Handler
                0x08008e38        0x2 startup\startup_stm32f207xx.o
                0x08008e38                RTC_Alarm_IRQHandler
                0x08008e38                HASH_RNG_IRQHandler
                0x08008e38                EXTI2_IRQHandler
                0x08008e38                TIM8_CC_IRQHandler
                0x08008e38                TIM1_CC_IRQHandler
                0x08008e38                DMA2_Stream5_IRQHandler
                0x08008e38                DMA1_Stream5_IRQHandler
                0x08008e38                PVD_IRQHandler
                0x08008e38                SDIO_IRQHandler
                0x08008e38                TAMP_STAMP_IRQHandler
                0x08008e38                CAN2_RX1_IRQHandler
                0x08008e38                EXTI3_IRQHandler
                0x08008e38                TIM8_TRG_COM_TIM14_IRQHandler
                0x08008e38                TIM1_UP_TIM10_IRQHandler
                0x08008e38                TIM8_UP_TIM13_IRQHandler
                0x08008e38                I2C3_ER_IRQHandler
                0x08008e38                EXTI0_IRQHandler
                0x08008e38                I2C2_EV_IRQHandler
                0x08008e38                DMA1_Stream2_IRQHandler
                0x08008e38                CAN1_RX0_IRQHandler
                0x08008e38                OTG_HS_WKUP_IRQHandler
                0x08008e38                CAN2_SCE_IRQHandler
                0x08008e38                DMA2_Stream2_IRQHandler
                0x08008e38                SPI1_IRQHandler
                0x08008e38                TIM1_BRK_TIM9_IRQHandler
                0x08008e38                DCMI_IRQHandler
                0x08008e38                CAN2_RX0_IRQHandler
                0x08008e38                DMA2_Stream3_IRQHandler
                0x08008e38                USART6_IRQHandler
                0x08008e38                CAN1_RX1_IRQHandler
                0x08008e38                UART5_IRQHandler
                0x08008e38                DMA2_Stream0_IRQHandler
                0x08008e38                TIM4_IRQHandler
                0x08008e38                I2C1_EV_IRQHandler
                0x08008e38                DMA1_Stream6_IRQHandler
                0x08008e38                UART4_IRQHandler
                0x08008e38                TIM3_IRQHandler
                0x08008e38                RCC_IRQHandler
                0x08008e38                TIM8_BRK_TIM12_IRQHandler
                0x08008e38                Default_Handler
                0x08008e38                ADC_IRQHandler
                0x08008e38                DMA1_Stream7_IRQHandler
                0x08008e38                TIM7_IRQHandler
                0x08008e38                CAN2_TX_IRQHandler
                0x08008e38                TIM5_IRQHandler
                0x08008e38                DMA2_Stream7_IRQHandler
                0x08008e38                I2C3_EV_IRQHandler
                0x08008e38                RTC_WKUP_IRQHandler
                0x08008e38                ETH_WKUP_IRQHandler
                0x08008e38                SPI2_IRQHandler
                0x08008e38                OTG_HS_EP1_IN_IRQHandler
                0x08008e38                DMA1_Stream0_IRQHandler
                0x08008e38                CAN1_TX_IRQHandler
                0x08008e38                EXTI4_IRQHandler
                0x08008e38                FSMC_IRQHandler
                0x08008e38                ETH_IRQHandler
                0x08008e38                OTG_HS_EP1_OUT_IRQHandler
                0x08008e38                WWDG_IRQHandler
                0x08008e38                TIM2_IRQHandler
                0x08008e38                OTG_FS_WKUP_IRQHandler
                0x08008e38                TIM1_TRG_COM_TIM11_IRQHandler
                0x08008e38                OTG_HS_IRQHandler
                0x08008e38                EXTI1_IRQHandler
                0x08008e38                USART2_IRQHandler
                0x08008e38                I2C2_ER_IRQHandler
                0x08008e38                DMA2_Stream1_IRQHandler
                0x08008e38                CAN1_SCE_IRQHandler
                0x08008e38                FLASH_IRQHandler
                0x08008e38                DMA2_Stream4_IRQHandler
                0x08008e38                USART1_IRQHandler
                0x08008e38                OTG_FS_IRQHandler
                0x08008e38                SPI3_IRQHandler
                0x08008e38                I2C1_ER_IRQHandler
                0x08008e38                DMA2_Stream6_IRQHandler
                0x08008e38                DMA1_Stream3_IRQHandler
 *fill*         0x08008e3a        0x2 
 .text.__errno  0x08008e3c        0xc c:/program files (x86)/atollic/truestudio for stm32 9.3.0/armtools/bin/../lib/gcc/arm-atollic-eabi/6.3.1/../../../../arm-atollic-eabi/lib/armv7-m\libc_nano.a(lib_a-errno.o)
                0x08008e3c                __errno
 .text.__libc_init_array
                0x08008e48       0x48 c:/program files (x86)/atollic/truestudio for stm32 9.3.0/armtools/bin/../lib/gcc/arm-atollic-eabi/6.3.1/../../../../arm-atollic-eabi/lib/armv7-m\libc_nano.a(lib_a-init.o)
                0x08008e48                __libc_init_array
 .text.memcpy   0x08008e90       0x16 c:/program files (x86)/atollic/truestudio for stm32 9.3.0/armtools/bin/../lib/gcc/arm-atollic-eabi/6.3.1/../../../../arm-atollic-eabi/lib/armv7-m\libc_nano.a(lib_a-memcpy-stub.o)
                0x08008e90                memcpy
 .text.memset   0x08008ea6       0x10 c:/program files (x86)/atollic/truestudio for stm32 9.3.0/armtools/bin/../lib/gcc/arm-atollic-eabi/6.3.1/../../../../arm-atollic-eabi/lib/armv7-m\libc_nano.a(lib_a-memset.o)
                0x08008ea6                memset
 .text.__cvt    0x08008eb6       0xb8 c:/program files (x86)/atollic/truestudio for stm32 9.3.0/armtools/bin/../lib/gcc/arm-atollic-eabi/6.3.1/../../../../arm-atollic-eabi/lib/armv7-m\libc_nano.a(lib_a-nano-vfprintf_float.o)
                0x08008eb6                __cvt
 .text.__exponent
                0x08008f6e       0x6a c:/program files (x86)/atollic/truestudio for stm32 9.3.0/armtools/bin/../lib/gcc/arm-atollic-eabi/6.3.1/../../../../arm-atollic-eabi/lib/armv7-m\libc_nano.a(lib_a-nano-vfprintf_float.o)
                0x08008f6e                __exponent
 .text._printf_float
                0x08008fd8      0x470 c:/program files (x86)/atollic/truestudio for stm32 9.3.0/armtools/bin/../lib/gcc/arm-atollic-eabi/6.3.1/../../../../arm-atollic-eabi/lib/armv7-m\libc_nano.a(lib_a-nano-vfprintf_float.o)
                0x08008fd8                _printf_float
 .text._printf_common
                0x08009448       0xee c:/program files (x86)/atollic/truestudio for stm32 9.3.0/armtools/bin/../lib/gcc/arm-atollic-eabi/6.3.1/../../../../arm-atollic-eabi/lib/armv7-m\libc_nano.a(lib_a-nano-vfprintf_i.o)
                0x08009448                _printf_common
 *fill*         0x08009536        0x2 
 .text._printf_i
                0x08009538      0x240 c:/program files (x86)/atollic/truestudio for stm32 9.3.0/armtools/bin/../lib/gcc/arm-atollic-eabi/6.3.1/../../../../arm-atollic-eabi/lib/armv7-m\libc_nano.a(lib_a-nano-vfprintf_i.o)
                0x08009538                _printf_i
 .text.printf   0x08009778       0x30 c:/program files (x86)/atollic/truestudio for stm32 9.3.0/armtools/bin/../lib/gcc/arm-atollic-eabi/6.3.1/../../../../arm-atollic-eabi/lib/armv7-m\libc_nano.a(lib_a-printf.o)
                0x08009778                iprintf
                0x08009778                printf
 .text._puts_r  0x080097a8       0xb8 c:/program files (x86)/atollic/truestudio for stm32 9.3.0/armtools/bin/../lib/gcc/arm-atollic-eabi/6.3.1/../../../../arm-atollic-eabi/lib/armv7-m\libc_nano.a(lib_a-puts.o)
                0x080097a8                _puts_r
 .text.puts     0x08009860       0x10 c:/program files (x86)/atollic/truestudio for stm32 9.3.0/armtools/bin/../lib/gcc/arm-atollic-eabi/6.3.1/../../../../arm-atollic-eabi/lib/armv7-m\libc_nano.a(lib_a-puts.o)
                0x08009860                puts
 .text.setbuf   0x08009870       0x10 c:/program files (x86)/atollic/truestudio for stm32 9.3.0/armtools/bin/../lib/gcc/arm-atollic-eabi/6.3.1/../../../../arm-atollic-eabi/lib/armv7-m\libc_nano.a(lib_a-setbuf.o)
                0x08009870                setbuf
 .text.setvbuf  0x08009880      0x15c c:/program files (x86)/atollic/truestudio for stm32 9.3.0/armtools/bin/../lib/gcc/arm-atollic-eabi/6.3.1/../../../../arm-atollic-eabi/lib/armv7-m\libc_nano.a(lib_a-setvbuf.o)
                0x08009880                setvbuf
 .text.sprintf  0x080099dc       0x48 c:/program files (x86)/atollic/truestudio for stm32 9.3.0/armtools/bin/../lib/gcc/arm-atollic-eabi/6.3.1/../../../../arm-atollic-eabi/lib/armv7-m\libc_nano.a(lib_a-sprintf.o)
                0x080099dc                siprintf
                0x080099dc                sprintf
 .text.strcpy   0x08009a24       0x10 c:/program files (x86)/atollic/truestudio for stm32 9.3.0/armtools/bin/../lib/gcc/arm-atollic-eabi/6.3.1/../../../../arm-atollic-eabi/lib/armv7-m\libc_nano.a(lib_a-strcpy.o)
                0x08009a24                strcpy
 .text.__swbuf_r
                0x08009a34       0xa4 c:/program files (x86)/atollic/truestudio for stm32 9.3.0/armtools/bin/../lib/gcc/arm-atollic-eabi/6.3.1/../../../../arm-atollic-eabi/lib/armv7-m\libc_nano.a(lib_a-wbuf.o)
                0x08009a34                __swbuf_r
 .text.__swsetup_r
                0x08009ad8       0xdc c:/program files (x86)/atollic/truestudio for stm32 9.3.0/armtools/bin/../lib/gcc/arm-atollic-eabi/6.3.1/../../../../arm-atollic-eabi/lib/armv7-m\libc_nano.a(lib_a-wsetup.o)
                0x08009ad8                __swsetup_r
 .text.quorem   0x08009bb4      0x118 c:/program files (x86)/atollic/truestudio for stm32 9.3.0/armtools/bin/../lib/gcc/arm-atollic-eabi/6.3.1/../../../../arm-atollic-eabi/lib/armv7-m\libc_nano.a(lib_a-dtoa.o)
 *fill*         0x08009ccc        0x4 
 .text._dtoa_r  0x08009cd0      0xba8 c:/program files (x86)/atollic/truestudio for stm32 9.3.0/armtools/bin/../lib/gcc/arm-atollic-eabi/6.3.1/../../../../arm-atollic-eabi/lib/armv7-m\libc_nano.a(lib_a-dtoa.o)
                0x08009cd0                _dtoa_r
 .text.__sflush_r
                0x0800a878      0x110 c:/program files (x86)/atollic/truestudio for stm32 9.3.0/armtools/bin/../lib/gcc/arm-atollic-eabi/6.3.1/../../../../arm-atollic-eabi/lib/armv7-m\libc_nano.a(lib_a-fflush.o)
                0x0800a878                __sflush_r
 .text._fflush_r
                0x0800a988       0x54 c:/program files (x86)/atollic/truestudio for stm32 9.3.0/armtools/bin/../lib/gcc/arm-atollic-eabi/6.3.1/../../../../arm-atollic-eabi/lib/armv7-m\libc_nano.a(lib_a-fflush.o)
                0x0800a988                _fflush_r
 .text._cleanup_r
                0x0800a9dc        0xc c:/program files (x86)/atollic/truestudio for stm32 9.3.0/armtools/bin/../lib/gcc/arm-atollic-eabi/6.3.1/../../../../arm-atollic-eabi/lib/armv7-m\libc_nano.a(lib_a-findfp.o)
                0x0800a9dc                _cleanup_r
 .text.std.isra.0
                0x0800a9e8       0x48 c:/program files (x86)/atollic/truestudio for stm32 9.3.0/armtools/bin/../lib/gcc/arm-atollic-eabi/6.3.1/../../../../arm-atollic-eabi/lib/armv7-m\libc_nano.a(lib_a-findfp.o)
 .text.__sfmoreglue
                0x0800aa30       0x2c c:/program files (x86)/atollic/truestudio for stm32 9.3.0/armtools/bin/../lib/gcc/arm-atollic-eabi/6.3.1/../../../../arm-atollic-eabi/lib/armv7-m\libc_nano.a(lib_a-findfp.o)
                0x0800aa30                __sfmoreglue
 .text.__sinit  0x0800aa5c       0x60 c:/program files (x86)/atollic/truestudio for stm32 9.3.0/armtools/bin/../lib/gcc/arm-atollic-eabi/6.3.1/../../../../arm-atollic-eabi/lib/armv7-m\libc_nano.a(lib_a-findfp.o)
                0x0800aa5c                __sinit
 .text.__sfp    0x0800aabc       0x78 c:/program files (x86)/atollic/truestudio for stm32 9.3.0/armtools/bin/../lib/gcc/arm-atollic-eabi/6.3.1/../../../../arm-atollic-eabi/lib/armv7-m\libc_nano.a(lib_a-findfp.o)
                0x0800aabc                __sfp
 .text._fwalk_reent
                0x0800ab34       0x3c c:/program files (x86)/atollic/truestudio for stm32 9.3.0/armtools/bin/../lib/gcc/arm-atollic-eabi/6.3.1/../../../../arm-atollic-eabi/lib/armv7-m\libc_nano.a(lib_a-fwalk.o)
                0x0800ab34                _fwalk_reent
 .text._localeconv_r
                0x0800ab70       0x1c c:/program files (x86)/atollic/truestudio for stm32 9.3.0/armtools/bin/../lib/gcc/arm-atollic-eabi/6.3.1/../../../../arm-atollic-eabi/lib/armv7-m\libc_nano.a(lib_a-localeconv.o)
                0x0800ab70                _localeconv_r
 .text.__swhatbuf_r
                0x0800ab8c       0x48 c:/program files (x86)/atollic/truestudio for stm32 9.3.0/armtools/bin/../lib/gcc/arm-atollic-eabi/6.3.1/../../../../arm-atollic-eabi/lib/armv7-m\libc_nano.a(lib_a-makebuf.o)
                0x0800ab8c                __swhatbuf_r
 .text.__smakebuf_r
                0x0800abd4       0x80 c:/program files (x86)/atollic/truestudio for stm32 9.3.0/armtools/bin/../lib/gcc/arm-atollic-eabi/6.3.1/../../../../arm-atollic-eabi/lib/armv7-m\libc_nano.a(lib_a-makebuf.o)
                0x0800abd4                __smakebuf_r
 .text.malloc   0x0800ac54       0x10 c:/program files (x86)/atollic/truestudio for stm32 9.3.0/armtools/bin/../lib/gcc/arm-atollic-eabi/6.3.1/../../../../arm-atollic-eabi/lib/armv7-m\libc_nano.a(lib_a-malloc.o)
                0x0800ac54                malloc
 .text.memchr   0x0800ac64       0x1c c:/program files (x86)/atollic/truestudio for stm32 9.3.0/armtools/bin/../lib/gcc/arm-atollic-eabi/6.3.1/../../../../arm-atollic-eabi/lib/armv7-m\libc_nano.a(lib_a-memchr-stub.o)
                0x0800ac64                memchr
 .text._Balloc  0x0800ac80       0x68 c:/program files (x86)/atollic/truestudio for stm32 9.3.0/armtools/bin/../lib/gcc/arm-atollic-eabi/6.3.1/../../../../arm-atollic-eabi/lib/armv7-m\libc_nano.a(lib_a-mprec.o)
                0x0800ac80                _Balloc
 .text._Bfree   0x0800ace8       0x2e c:/program files (x86)/atollic/truestudio for stm32 9.3.0/armtools/bin/../lib/gcc/arm-atollic-eabi/6.3.1/../../../../arm-atollic-eabi/lib/armv7-m\libc_nano.a(lib_a-mprec.o)
                0x0800ace8                _Bfree
 .text.__multadd
                0x0800ad16       0x76 c:/program files (x86)/atollic/truestudio for stm32 9.3.0/armtools/bin/../lib/gcc/arm-atollic-eabi/6.3.1/../../../../arm-atollic-eabi/lib/armv7-m\libc_nano.a(lib_a-mprec.o)
                0x0800ad16                __multadd
 .text.__hi0bits
                0x0800ad8c       0x3e c:/program files (x86)/atollic/truestudio for stm32 9.3.0/armtools/bin/../lib/gcc/arm-atollic-eabi/6.3.1/../../../../arm-atollic-eabi/lib/armv7-m\libc_nano.a(lib_a-mprec.o)
                0x0800ad8c                __hi0bits
 .text.__lo0bits
                0x0800adca       0x5e c:/program files (x86)/atollic/truestudio for stm32 9.3.0/armtools/bin/../lib/gcc/arm-atollic-eabi/6.3.1/../../../../arm-atollic-eabi/lib/armv7-m\libc_nano.a(lib_a-mprec.o)
                0x0800adca                __lo0bits
 .text.__i2b    0x0800ae28       0x12 c:/program files (x86)/atollic/truestudio for stm32 9.3.0/armtools/bin/../lib/gcc/arm-atollic-eabi/6.3.1/../../../../arm-atollic-eabi/lib/armv7-m\libc_nano.a(lib_a-mprec.o)
                0x0800ae28                __i2b
 .text.__multiply
                0x0800ae3a      0x118 c:/program files (x86)/atollic/truestudio for stm32 9.3.0/armtools/bin/../lib/gcc/arm-atollic-eabi/6.3.1/../../../../arm-atollic-eabi/lib/armv7-m\libc_nano.a(lib_a-mprec.o)
                0x0800ae3a                __multiply
 *fill*         0x0800af52        0x2 
 .text.__pow5mult
                0x0800af54       0x9c c:/program files (x86)/atollic/truestudio for stm32 9.3.0/armtools/bin/../lib/gcc/arm-atollic-eabi/6.3.1/../../../../arm-atollic-eabi/lib/armv7-m\libc_nano.a(lib_a-mprec.o)
                0x0800af54                __pow5mult
 .text.__lshift
                0x0800aff0       0xa2 c:/program files (x86)/atollic/truestudio for stm32 9.3.0/armtools/bin/../lib/gcc/arm-atollic-eabi/6.3.1/../../../../arm-atollic-eabi/lib/armv7-m\libc_nano.a(lib_a-mprec.o)
                0x0800aff0                __lshift
 .text.__mcmp   0x0800b092       0x34 c:/program files (x86)/atollic/truestudio for stm32 9.3.0/armtools/bin/../lib/gcc/arm-atollic-eabi/6.3.1/../../../../arm-atollic-eabi/lib/armv7-m\libc_nano.a(lib_a-mprec.o)
                0x0800b092                __mcmp
 .text.__mdiff  0x0800b0c6       0xbe c:/program files (x86)/atollic/truestudio for stm32 9.3.0/armtools/bin/../lib/gcc/arm-atollic-eabi/6.3.1/../../../../arm-atollic-eabi/lib/armv7-m\libc_nano.a(lib_a-mprec.o)
                0x0800b0c6                __mdiff
 .text.__d2b    0x0800b184       0x9e c:/program files (x86)/atollic/truestudio for stm32 9.3.0/armtools/bin/../lib/gcc/arm-atollic-eabi/6.3.1/../../../../arm-atollic-eabi/lib/armv7-m\libc_nano.a(lib_a-mprec.o)
                0x0800b184                __d2b
 .text._calloc_r
                0x0800b222       0x1c c:/program files (x86)/atollic/truestudio for stm32 9.3.0/armtools/bin/../lib/gcc/arm-atollic-eabi/6.3.1/../../../../arm-atollic-eabi/lib/armv7-m\libc_nano.a(lib_a-nano-callocr.o)
                0x0800b222                _calloc_r
 *fill*         0x0800b23e        0x2 
 .text._free_r  0x0800b240       0x98 c:/program files (x86)/atollic/truestudio for stm32 9.3.0/armtools/bin/../lib/gcc/arm-atollic-eabi/6.3.1/../../../../arm-atollic-eabi/lib/armv7-m\libc_nano.a(lib_a-nano-freer.o)
                0x0800b240                _free_r
 .text._malloc_r
                0x0800b2d8       0xbc c:/program files (x86)/atollic/truestudio for stm32 9.3.0/armtools/bin/../lib/gcc/arm-atollic-eabi/6.3.1/../../../../arm-atollic-eabi/lib/armv7-m\libc_nano.a(lib_a-nano-mallocr.o)
                0x0800b2d8                _malloc_r
 .text.__ssputs_r
                0x0800b394       0xb6 c:/program files (x86)/atollic/truestudio for stm32 9.3.0/armtools/bin/../lib/gcc/arm-atollic-eabi/6.3.1/../../../../arm-atollic-eabi/lib/armv7-m\libc_nano.a(lib_a-nano-svfprintf.o)
                0x0800b394                __ssputs_r
 *fill*         0x0800b44a        0x2 
 .text._svfprintf_r
                0x0800b44c      0x1e8 c:/program files (x86)/atollic/truestudio for stm32 9.3.0/armtools/bin/../lib/gcc/arm-atollic-eabi/6.3.1/../../../../arm-atollic-eabi/lib/armv7-m\libc_nano.a(lib_a-nano-svfprintf.o)
                0x0800b44c                _svfiprintf_r
                0x0800b44c                _svfprintf_r
 .text.__sfputc_r
                0x0800b634       0x2c c:/program files (x86)/atollic/truestudio for stm32 9.3.0/armtools/bin/../lib/gcc/arm-atollic-eabi/6.3.1/../../../../arm-atollic-eabi/lib/armv7-m\libc_nano.a(lib_a-nano-vfprintf.o)
 .text.__sfputs_r
                0x0800b660       0x24 c:/program files (x86)/atollic/truestudio for stm32 9.3.0/armtools/bin/../lib/gcc/arm-atollic-eabi/6.3.1/../../../../arm-atollic-eabi/lib/armv7-m\libc_nano.a(lib_a-nano-vfprintf.o)
                0x0800b660                __sfputs_r
 .text._vfprintf_r
                0x0800b684      0x22c c:/program files (x86)/atollic/truestudio for stm32 9.3.0/armtools/bin/../lib/gcc/arm-atollic-eabi/6.3.1/../../../../arm-atollic-eabi/lib/armv7-m\libc_nano.a(lib_a-nano-vfprintf.o)
                0x0800b684                _vfprintf_r
                0x0800b684                _vfiprintf_r
 .text._sbrk_r  0x0800b8b0       0x20 c:/program files (x86)/atollic/truestudio for stm32 9.3.0/armtools/bin/../lib/gcc/arm-atollic-eabi/6.3.1/../../../../arm-atollic-eabi/lib/armv7-m\libc_nano.a(lib_a-sbrkr.o)
                0x0800b8b0                _sbrk_r
 .text.__sread  0x0800b8d0       0x22 c:/program files (x86)/atollic/truestudio for stm32 9.3.0/armtools/bin/../lib/gcc/arm-atollic-eabi/6.3.1/../../../../arm-atollic-eabi/lib/armv7-m\libc_nano.a(lib_a-stdio.o)
                0x0800b8d0                __sread
 .text.__swrite
                0x0800b8f2       0x38 c:/program files (x86)/atollic/truestudio for stm32 9.3.0/armtools/bin/../lib/gcc/arm-atollic-eabi/6.3.1/../../../../arm-atollic-eabi/lib/armv7-m\libc_nano.a(lib_a-stdio.o)
                0x0800b8f2                __swrite
 .text.__sseek  0x0800b92a       0x24 c:/program files (x86)/atollic/truestudio for stm32 9.3.0/armtools/bin/../lib/gcc/arm-atollic-eabi/6.3.1/../../../../arm-atollic-eabi/lib/armv7-m\libc_nano.a(lib_a-stdio.o)
                0x0800b92a                __sseek
 .text.__sclose
                0x0800b94e        0x8 c:/program files (x86)/atollic/truestudio for stm32 9.3.0/armtools/bin/../lib/gcc/arm-atollic-eabi/6.3.1/../../../../arm-atollic-eabi/lib/armv7-m\libc_nano.a(lib_a-stdio.o)
                0x0800b94e                __sclose
 *fill*         0x0800b956        0x2 
 .text._write_r
                0x0800b958       0x24 c:/program files (x86)/atollic/truestudio for stm32 9.3.0/armtools/bin/../lib/gcc/arm-atollic-eabi/6.3.1/../../../../arm-atollic-eabi/lib/armv7-m\libc_nano.a(lib_a-writer.o)
                0x0800b958                _write_r
 .text._close_r
                0x0800b97c       0x20 c:/program files (x86)/atollic/truestudio for stm32 9.3.0/armtools/bin/../lib/gcc/arm-atollic-eabi/6.3.1/../../../../arm-atollic-eabi/lib/armv7-m\libc_nano.a(lib_a-closer.o)
                0x0800b97c                _close_r
 .text._fstat_r
                0x0800b99c       0x24 c:/program files (x86)/atollic/truestudio for stm32 9.3.0/armtools/bin/../lib/gcc/arm-atollic-eabi/6.3.1/../../../../arm-atollic-eabi/lib/armv7-m\libc_nano.a(lib_a-fstatr.o)
                0x0800b99c                _fstat_r
 .text._isatty_r
                0x0800b9c0       0x20 c:/program files (x86)/atollic/truestudio for stm32 9.3.0/armtools/bin/../lib/gcc/arm-atollic-eabi/6.3.1/../../../../arm-atollic-eabi/lib/armv7-m\libc_nano.a(lib_a-isattyr.o)
                0x0800b9c0                _isatty_r
 .text._lseek_r
                0x0800b9e0       0x24 c:/program files (x86)/atollic/truestudio for stm32 9.3.0/armtools/bin/../lib/gcc/arm-atollic-eabi/6.3.1/../../../../arm-atollic-eabi/lib/armv7-m\libc_nano.a(lib_a-lseekr.o)
                0x0800b9e0                _lseek_r
 .text.__ascii_mbtowc
                0x0800ba04       0x24 c:/program files (x86)/atollic/truestudio for stm32 9.3.0/armtools/bin/../lib/gcc/arm-atollic-eabi/6.3.1/../../../../arm-atollic-eabi/lib/armv7-m\libc_nano.a(lib_a-mbtowc_r.o)
                0x0800ba04                __ascii_mbtowc
 .text.memmove  0x0800ba28       0x34 c:/program files (x86)/atollic/truestudio for stm32 9.3.0/armtools/bin/../lib/gcc/arm-atollic-eabi/6.3.1/../../../../arm-atollic-eabi/lib/armv7-m\libc_nano.a(lib_a-memmove.o)
                0x0800ba28                memmove
 .text.__malloc_lock
                0x0800ba5c        0x2 c:/program files (x86)/atollic/truestudio for stm32 9.3.0/armtools/bin/../lib/gcc/arm-atollic-eabi/6.3.1/../../../../arm-atollic-eabi/lib/armv7-m\libc_nano.a(lib_a-mlock.o)
                0x0800ba5c                __malloc_lock
 .text.__malloc_unlock
                0x0800ba5e        0x2 c:/program files (x86)/atollic/truestudio for stm32 9.3.0/armtools/bin/../lib/gcc/arm-atollic-eabi/6.3.1/../../../../arm-atollic-eabi/lib/armv7-m\libc_nano.a(lib_a-mlock.o)
                0x0800ba5e                __malloc_unlock
 .text._realloc_r
                0x0800ba60       0x4c c:/program files (x86)/atollic/truestudio for stm32 9.3.0/armtools/bin/../lib/gcc/arm-atollic-eabi/6.3.1/../../../../arm-atollic-eabi/lib/armv7-m\libc_nano.a(lib_a-nano-reallocr.o)
                0x0800ba60                _realloc_r
 .text._read_r  0x0800baac       0x24 c:/program files (x86)/atollic/truestudio for stm32 9.3.0/armtools/bin/../lib/gcc/arm-atollic-eabi/6.3.1/../../../../arm-atollic-eabi/lib/armv7-m\libc_nano.a(lib_a-readr.o)
                0x0800baac                _read_r
 .text.__ascii_wctomb
                0x0800bad0       0x1a c:/program files (x86)/atollic/truestudio for stm32 9.3.0/armtools/bin/../lib/gcc/arm-atollic-eabi/6.3.1/../../../../arm-atollic-eabi/lib/armv7-m\libc_nano.a(lib_a-wctomb_r.o)
                0x0800bad0                __ascii_wctomb
 .text._malloc_usable_size_r
                0x0800baea       0x12 c:/program files (x86)/atollic/truestudio for stm32 9.3.0/armtools/bin/../lib/gcc/arm-atollic-eabi/6.3.1/../../../../arm-atollic-eabi/lib/armv7-m\libc_nano.a(lib_a-nano-msizer.o)
                0x0800baea                _malloc_usable_size_r
 *(.glue_7)
 .glue_7        0x0800bafc        0x0 linker stubs
 *(.glue_7t)
 .glue_7t       0x0800bafc        0x0 linker stubs
 *(.eh_frame)
 .eh_frame      0x0800bafc        0x0 c:/program files (x86)/atollic/truestudio for stm32 9.3.0/armtools/bin/../lib/gcc/arm-atollic-eabi/6.3.1/armv7-m/crtbegin.o
 *(.init)
 .init          0x0800bafc        0x4 c:/program files (x86)/atollic/truestudio for stm32 9.3.0/armtools/bin/../lib/gcc/arm-atollic-eabi/6.3.1/armv7-m/crti.o
                0x0800bafc                _init
 .init          0x0800bb00        0x8 c:/program files (x86)/atollic/truestudio for stm32 9.3.0/armtools/bin/../lib/gcc/arm-atollic-eabi/6.3.1/armv7-m/crtn.o
 *(.fini)
 .fini          0x0800bb08        0x4 c:/program files (x86)/atollic/truestudio for stm32 9.3.0/armtools/bin/../lib/gcc/arm-atollic-eabi/6.3.1/armv7-m/crti.o
                0x0800bb08                _fini
 .fini          0x0800bb0c        0x8 c:/program files (x86)/atollic/truestudio for stm32 9.3.0/armtools/bin/../lib/gcc/arm-atollic-eabi/6.3.1/armv7-m/crtn.o
                0x0800bb14                . = ALIGN (0x4)
                0x0800bb14                _etext = .

.vfp11_veneer   0x0800bb14        0x0
 .vfp11_veneer  0x0800bb14        0x0 linker stubs

.v4_bx          0x0800bb14        0x0
 .v4_bx         0x0800bb14        0x0 linker stubs

.iplt           0x0800bb14        0x0
 .iplt          0x0800bb14        0x0 c:/program files (x86)/atollic/truestudio for stm32 9.3.0/armtools/bin/../lib/gcc/arm-atollic-eabi/6.3.1/armv7-m/crtbegin.o

.rodata         0x0800bb18      0x478
                0x0800bb18                . = ALIGN (0x4)
 *(.rodata)
 *(.rodata*)
 .rodata.flagBitshiftOffset.6770
                0x0800bb18        0x8 Drivers\STM32F2xx_HAL_Driver\Src\stm32f2xx_hal_dma.o
 .rodata.Character_Lcd_chMenu.str1.1
                0x0800bb20       0x21 Src\Character_lcd.o
 .rodata.LCD_30G_Freq_Select_Display.str1.1
                0x0800bb41       0x3d Src\Character_lcd.o
 .rodata.LCD_Wifi_Freq_Select_Display.str1.1
                0x0800bb7e       0x20 Src\Character_lcd.o
 .rodata.Lcd_Ach150M_Display.str1.1
                0x0800bb9e       0x1f Src\Character_lcd.o
 .rodata.Lcd_Ach30G_Display.str1.1
                0x0800bbbd        0xc Src\Character_lcd.o
 .rodata.Lcd_AchSetting_Display.str1.1
                0x0800bbc9       0x1c Src\Character_lcd.o
 .rodata.Lcd_AchWifi_Display.str1.1
                0x0800bbe5        0xf Src\Character_lcd.o
 .rodata.Lcd_Bch150M_Display.str1.1
                0x0800bbf4        0xf Src\Character_lcd.o
 .rodata.Lcd_Bch30G_Display.str1.1
                0x0800bc03        0xc Src\Character_lcd.o
 .rodata.Lcd_BchSetting_Display.str1.1
                0x0800bc0f        0xc Src\Character_lcd.o
 .rodata.Lcd_BchWifi_Display.str1.1
                0x0800bc1b        0xe Src\Character_lcd.o
 .rodata.Atten_Offset_QPC6614.str1.1
                0x0800bc29       0x10 Src\atten_ctrl.o
 .rodata.Atten_Operate_Mem_RW.str1.1
                0x0800bc39       0x27 Src\atten_ctrl.o
 .rodata.__func__.9698
                0x0800bc60       0x15 Src\atten_ctrl.o
 .rodata.main.str1.1
                0x0800bc75       0x41 Src\main.o
                                 0x43 (size before relaxing)
 .rodata.AHBPrescTable
                0x0800bcb6       0x10 Src\system_stm32f2xx.o
                0x0800bcb6                AHBPrescTable
 .rodata.APBPrescTable
                0x0800bcc6        0x8 Src\system_stm32f2xx.o
                0x0800bcc6                APBPrescTable
 *fill*         0x0800bcce        0x2 
 .rodata._global_impure_ptr
                0x0800bcd0        0x4 c:/program files (x86)/atollic/truestudio for stm32 9.3.0/armtools/bin/../lib/gcc/arm-atollic-eabi/6.3.1/../../../../arm-atollic-eabi/lib/armv7-m\libc_nano.a(lib_a-impure.o)
                0x0800bcd0                _global_impure_ptr
 .rodata._printf_float.str1.1
                0x0800bcd4       0x12 c:/program files (x86)/atollic/truestudio for stm32 9.3.0/armtools/bin/../lib/gcc/arm-atollic-eabi/6.3.1/../../../../arm-atollic-eabi/lib/armv7-m\libc_nano.a(lib_a-nano-vfprintf_float.o)
 .rodata._printf_i.str1.1
                0x0800bce6       0x22 c:/program files (x86)/atollic/truestudio for stm32 9.3.0/armtools/bin/../lib/gcc/arm-atollic-eabi/6.3.1/../../../../arm-atollic-eabi/lib/armv7-m\libc_nano.a(lib_a-nano-vfprintf_i.o)
 .rodata._dtoa_r.str1.1
                0x0800bd08        0xd c:/program files (x86)/atollic/truestudio for stm32 9.3.0/armtools/bin/../lib/gcc/arm-atollic-eabi/6.3.1/../../../../arm-atollic-eabi/lib/armv7-m\libc_nano.a(lib_a-dtoa.o)
                                  0xf (size before relaxing)
 *fill*         0x0800bd15        0x3 
 .rodata.__sf_fake_stderr
                0x0800bd18       0x20 c:/program files (x86)/atollic/truestudio for stm32 9.3.0/armtools/bin/../lib/gcc/arm-atollic-eabi/6.3.1/../../../../arm-atollic-eabi/lib/armv7-m\libc_nano.a(lib_a-findfp.o)
                0x0800bd18                __sf_fake_stderr
 .rodata.__sf_fake_stdin
                0x0800bd38       0x20 c:/program files (x86)/atollic/truestudio for stm32 9.3.0/armtools/bin/../lib/gcc/arm-atollic-eabi/6.3.1/../../../../arm-atollic-eabi/lib/armv7-m\libc_nano.a(lib_a-findfp.o)
                0x0800bd38                __sf_fake_stdin
 .rodata.__sf_fake_stdout
                0x0800bd58       0x20 c:/program files (x86)/atollic/truestudio for stm32 9.3.0/armtools/bin/../lib/gcc/arm-atollic-eabi/6.3.1/../../../../arm-atollic-eabi/lib/armv7-m\libc_nano.a(lib_a-findfp.o)
                0x0800bd58                __sf_fake_stdout
 .rodata.__mprec_bigtens
                0x0800bd78       0x28 c:/program files (x86)/atollic/truestudio for stm32 9.3.0/armtools/bin/../lib/gcc/arm-atollic-eabi/6.3.1/../../../../arm-atollic-eabi/lib/armv7-m\libc_nano.a(lib_a-mprec.o)
                0x0800bd78                __mprec_bigtens
 .rodata.__mprec_tens
                0x0800bda0       0xc8 c:/program files (x86)/atollic/truestudio for stm32 9.3.0/armtools/bin/../lib/gcc/arm-atollic-eabi/6.3.1/../../../../arm-atollic-eabi/lib/armv7-m\libc_nano.a(lib_a-mprec.o)
                0x0800bda0                __mprec_tens
 .rodata.p05.6052
                0x0800be68        0xc c:/program files (x86)/atollic/truestudio for stm32 9.3.0/armtools/bin/../lib/gcc/arm-atollic-eabi/6.3.1/../../../../arm-atollic-eabi/lib/armv7-m\libc_nano.a(lib_a-mprec.o)
 .rodata._svfprintf_r.str1.1
                0x0800be74       0x11 c:/program files (x86)/atollic/truestudio for stm32 9.3.0/armtools/bin/../lib/gcc/arm-atollic-eabi/6.3.1/../../../../arm-atollic-eabi/lib/armv7-m\libc_nano.a(lib_a-nano-svfprintf.o)
 .rodata._vfprintf_r.str1.1
                0x0800be85       0x11 c:/program files (x86)/atollic/truestudio for stm32 9.3.0/armtools/bin/../lib/gcc/arm-atollic-eabi/6.3.1/../../../../arm-atollic-eabi/lib/armv7-m\libc_nano.a(lib_a-nano-vfprintf.o)
 .rodata._setlocale_r.str1.1
                0x0800be85        0x8 c:/program files (x86)/atollic/truestudio for stm32 9.3.0/armtools/bin/../lib/gcc/arm-atollic-eabi/6.3.1/../../../../arm-atollic-eabi/lib/armv7-m\libc_nano.a(lib_a-locale.o)
                                  0x9 (size before relaxing)
 .rodata.str1.1
                0x0800be8d        0x2 c:/program files (x86)/atollic/truestudio for stm32 9.3.0/armtools/bin/../lib/gcc/arm-atollic-eabi/6.3.1/../../../../arm-atollic-eabi/lib/armv7-m\libc_nano.a(lib_a-locale.o)
 .rodata._ctype_
                0x0800be8f      0x101 c:/program files (x86)/atollic/truestudio for stm32 9.3.0/armtools/bin/../lib/gcc/arm-atollic-eabi/6.3.1/../../../../arm-atollic-eabi/lib/armv7-m\libc_nano.a(lib_a-ctype_.o)
                0x0800be8f                _ctype_
                0x0800bf90                . = ALIGN (0x4)

.ARM.extab
 *(.ARM.extab* .gnu.linkonce.armextab.*)

.ARM            0x0800bf90        0x8
                0x0800bf90                __exidx_start = .
 *(.ARM.exidx*)
 .ARM.exidx     0x0800bf90        0x8 c:/program files (x86)/atollic/truestudio for stm32 9.3.0/armtools/bin/../lib/gcc/arm-atollic-eabi/6.3.1/armv7-m\libgcc.a(_udivmoddi4.o)
                0x0800bf98                __exidx_end = .

.rel.dyn        0x0800bf98        0x0
 .rel.iplt      0x0800bf98        0x0 c:/program files (x86)/atollic/truestudio for stm32 9.3.0/armtools/bin/../lib/gcc/arm-atollic-eabi/6.3.1/armv7-m/crtbegin.o

.preinit_array  0x0800bf98        0x0
                0x0800bf98                PROVIDE (__preinit_array_start, .)
 *(.preinit_array*)
                0x0800bf98                PROVIDE (__preinit_array_end, .)

.init_array     0x0800bf98        0x4
                0x0800bf98                PROVIDE (__init_array_start, .)
 *(SORT(.init_array.*))
 *(.init_array*)
 .init_array    0x0800bf98        0x4 c:/program files (x86)/atollic/truestudio for stm32 9.3.0/armtools/bin/../lib/gcc/arm-atollic-eabi/6.3.1/armv7-m/crtbegin.o
                0x0800bf9c                PROVIDE (__init_array_end, .)

.fini_array     0x0800bf9c        0x4
                [!provide]                PROVIDE (__fini_array_start, .)
 *(SORT(.fini_array.*))
 *(.fini_array*)
 .fini_array    0x0800bf9c        0x4 c:/program files (x86)/atollic/truestudio for stm32 9.3.0/armtools/bin/../lib/gcc/arm-atollic-eabi/6.3.1/armv7-m/crtbegin.o
                [!provide]                PROVIDE (__fini_array_end, .)
                0x0800bfa0                _sidata = LOADADDR (.data)

.data           0x20000000      0x1dc load address 0x0800bfa0
                0x20000000                . = ALIGN (0x4)
                0x20000000                _sdata = .
 *(.data)
 *(.data*)
 .data.uwTickFreq
                0x20000000        0x1 Drivers\STM32F2xx_HAL_Driver\Src\stm32f2xx_hal.o
                0x20000000                uwTickFreq
 *fill*         0x20000001        0x3 
 .data.uwTickPrio
                0x20000004        0x4 Drivers\STM32F2xx_HAL_Driver\Src\stm32f2xx_hal.o
                0x20000004                uwTickPrio
 .data.SystemCoreClock
                0x20000008        0x4 Src\system_stm32f2xx.o
                0x20000008                SystemCoreClock
 .data._impure_ptr
                0x2000000c        0x4 c:/program files (x86)/atollic/truestudio for stm32 9.3.0/armtools/bin/../lib/gcc/arm-atollic-eabi/6.3.1/../../../../arm-atollic-eabi/lib/armv7-m\libc_nano.a(lib_a-impure.o)
                0x2000000c                _impure_ptr
 .data.impure_data
                0x20000010       0x60 c:/program files (x86)/atollic/truestudio for stm32 9.3.0/armtools/bin/../lib/gcc/arm-atollic-eabi/6.3.1/../../../../arm-atollic-eabi/lib/armv7-m\libc_nano.a(lib_a-impure.o)
 .data.__global_locale
                0x20000070      0x16c c:/program files (x86)/atollic/truestudio for stm32 9.3.0/armtools/bin/../lib/gcc/arm-atollic-eabi/6.3.1/../../../../arm-atollic-eabi/lib/armv7-m\libc_nano.a(lib_a-locale.o)
                0x20000070                __global_locale
                0x200001dc                . = ALIGN (0x4)
                0x200001dc                _edata = .

.igot.plt       0x200001dc        0x0 load address 0x0800c17c
 .igot.plt      0x200001dc        0x0 c:/program files (x86)/atollic/truestudio for stm32 9.3.0/armtools/bin/../lib/gcc/arm-atollic-eabi/6.3.1/armv7-m/crtbegin.o
                0x200001dc                . = ALIGN (0x4)

.bss            0x200001dc     0x1758 load address 0x0800c17c
                0x200001dc                _sbss = .
                0x200001dc                __bss_start__ = _sbss
 *(.bss)
 .bss           0x200001dc       0x1c c:/program files (x86)/atollic/truestudio for stm32 9.3.0/armtools/bin/../lib/gcc/arm-atollic-eabi/6.3.1/armv7-m/crtbegin.o
 *(.bss*)
 .bss.Ach_150M_Value
                0x200001f8        0x4 Src\Character_lcd.o
                0x200001f8                Ach_150M_Value
 .bss.Ach_30G_28_28_5_Value
                0x200001fc        0x4 Src\Character_lcd.o
                0x200001fc                Ach_30G_28_28_5_Value
 .bss.Ach_30G_28_5_29_Value
                0x20000200        0x4 Src\Character_lcd.o
                0x20000200                Ach_30G_28_5_29_Value
 .bss.Ach_30G_29_29_5_Value
                0x20000204        0x4 Src\Character_lcd.o
                0x20000204                Ach_30G_29_29_5_Value
 .bss.Ach_30G_29_5_30_Value
                0x20000208        0x4 Src\Character_lcd.o
                0x20000208                Ach_30G_29_5_30_Value
 .bss.Ach_Wifi_2_4GHz_Value
                0x2000020c        0x4 Src\Character_lcd.o
                0x2000020c                Ach_Wifi_2_4GHz_Value
 .bss.Ach_Wifi_5_8GHz_Value
                0x20000210        0x4 Src\Character_lcd.o
                0x20000210                Ach_Wifi_5_8GHz_Value
 .bss.Bch_150M_Value
                0x20000214        0x4 Src\Character_lcd.o
                0x20000214                Bch_150M_Value
 .bss.Bch_30G_28_28_5_Value
                0x20000218        0x4 Src\Character_lcd.o
                0x20000218                Bch_30G_28_28_5_Value
 .bss.Bch_30G_28_5_29_Value
                0x2000021c        0x4 Src\Character_lcd.o
                0x2000021c                Bch_30G_28_5_29_Value
 .bss.Bch_30G_29_29_5_Value
                0x20000220        0x4 Src\Character_lcd.o
                0x20000220                Bch_30G_29_29_5_Value
 .bss.Bch_30G_29_5_30_Value
                0x20000224        0x4 Src\Character_lcd.o
                0x20000224                Bch_30G_29_5_30_Value
 .bss.Bch_Wifi_2_4GHz_Value
                0x20000228        0x4 Src\Character_lcd.o
                0x20000228                Bch_Wifi_2_4GHz_Value
 .bss.Bch_Wifi_5_8GHz_Value
                0x2000022c        0x4 Src\Character_lcd.o
                0x2000022c                Bch_Wifi_5_8GHz_Value
 .bss.Button_Data_Occur
                0x20000230        0x1 Src\Character_lcd.o
                0x20000230                Button_Data_Occur
 .bss.CharacterLCD_ButtonSetval
                0x20000231        0x1 Src\Character_lcd.o
                0x20000231                CharacterLCD_ButtonSetval
 .bss.Curr_Layer
                0x20000232        0x1 Src\Character_lcd.o
                0x20000232                Curr_Layer
 .bss.initialize.9175
                0x20000233        0x1 Src\Character_lcd.o
 .bss.temp_str.9219
                0x20000234       0x10 Src\Character_lcd.o
 .bss.temp_str.9223
                0x20000244       0x10 Src\Character_lcd.o
 .bss.temp_str.9227
                0x20000254       0x10 Src\Character_lcd.o
 .bss.temp_str.9231
                0x20000264       0x10 Src\Character_lcd.o
 .bss.temp_str.9235
                0x20000274       0x10 Src\Character_lcd.o
 .bss.temp_str.9239
                0x20000284       0x10 Src\Character_lcd.o
 .bss.temp_str.9243
                0x20000294       0x10 Src\Character_lcd.o
 .bss.temp_str.9247
                0x200002a4       0x10 Src\Character_lcd.o
 .bss.temp_str.9253
                0x200002b4       0x10 Src\Character_lcd.o
 .bss.temp_str.9259
                0x200002c4       0x10 Src\Character_lcd.o
 .bss.temp_str.9265
                0x200002d4       0x10 Src\Character_lcd.o
 .bss.temp_str.9270
                0x200002e4       0x10 Src\Character_lcd.o
 .bss.temp_str.9275
                0x200002f4       0x10 Src\Character_lcd.o
 .bss.ret.9465  0x20000304       0x64 Src\atten_ctrl.o
 .bss.ret.9591  0x20000368       0x64 Src\atten_ctrl.o
 .bss.ButtonLong_TimerCnt
                0x200003cc        0x4 Src\main.o
                0x200003cc                ButtonLong_TimerCnt
 .bss.LedTimerCnt
                0x200003d0        0x4 Src\main.o
                0x200003d0                LedTimerCnt
 .bss.UartTimerCnt
                0x200003d4        0x4 Src\main.o
                0x200003d4                UartTimerCnt
 .bss.Unbutton_press
                0x200003d8        0x1 Src\main.o
                0x200003d8                Unbutton_press
 .bss.buf       0x200003d9       0x64 Src\main.o
                0x200003d9                buf
 .bss.button_press
                0x2000043d        0x1 Src\main.o
                0x2000043d                button_press
 .bss.uartindex
                0x2000043e        0x1 Src\main.o
                0x2000043e                uartindex
 *fill*         0x2000043f        0x1 
 .bss.heap_end.5887
                0x20000440        0x4 Src\syscalls.o
 .bss.__malloc_free_list
                0x20000444        0x4 c:/program files (x86)/atollic/truestudio for stm32 9.3.0/armtools/bin/../lib/gcc/arm-atollic-eabi/6.3.1/../../../../arm-atollic-eabi/lib/armv7-m\libc_nano.a(lib_a-nano-mallocr.o)
                0x20000444                __malloc_free_list
 .bss.__malloc_sbrk_start
                0x20000448        0x4 c:/program files (x86)/atollic/truestudio for stm32 9.3.0/armtools/bin/../lib/gcc/arm-atollic-eabi/6.3.1/../../../../arm-atollic-eabi/lib/armv7-m\libc_nano.a(lib_a-nano-mallocr.o)
                0x20000448                __malloc_sbrk_start
 *(COMMON)
 COMMON         0x2000044c        0x4 Drivers\STM32F2xx_HAL_Driver\Src\stm32f2xx_hal.o
                0x2000044c                uwTick
 COMMON         0x20000450      0xac0 Src\atten_ctrl.o
                0x20000450                ATT_B_EN_WIFI4_2_4Ghz_Table
                0x20000490                ATT_A_EN_30G3_29_29_5Ghz_Table
                0x200004d0                ATT_B_EN_30G1_28_28_5Ghz_Table
                0x20000510                ATT_A_EN_WIFI4_2_4Ghz_Table
                0x20000550                ATT_A_EN_30G3_29_5_30Ghz_Table
                0x20000590                ATT_B_EN_WIFI3_5_8Ghz_Table
                0x200005d0                ATT_B_EN_30G3_28_5_29Ghz_Table
                0x20000610                ATT_A_EN_WIFI1_2_4Ghz_Table
                0x20000650                ATT_B_EN_30G2_28_28_5Ghz_Table
                0x20000690                ATT_B_EN_WIFI4_5_8Ghz_Table
                0x200006d0                ATT_A_EN_WIFI3_2_4Ghz_Table
                0x20000710                ATT_B_EN_WIFI2_2_4Ghz_Table
                0x20000750                ATT_B_EN_30G1_28_5_29Ghz_Table
                0x20000790                ATT_A_EN_30G2_28_5_29Ghz_Table
                0x200007d0                ATT_B_EN_WIFI1_2_4Ghz_Table
                0x20000810                ATT_A_EN_30G2_29_29_5Ghz_Table
                0x20000850                ATT_B_EN_30G3_29_29_5Ghz_Table
                0x20000890                ATT_B_EN_30G2_28_5_29Ghz_Table
                0x200008d0                ATT_A_EN_30G3_28_5_29Ghz_Table
                0x20000910                ATT_B_EN_WIFI2_5_8Ghz_Table
                0x20000950                ATT_A_EN_30G1_28_28_5Ghz_Table
                0x20000990                ATT_B_EN_30G1_29_29_5Ghz_Table
                0x200009d0                ATT_B_EN_30G2_29_29_5Ghz_Table
                0x20000a10                ATT_A_EN_WIFI3_5_8Ghz_Table
                0x20000a50                ATT_A_EN_30G3_28_28_5Ghz_Table
                0x20000a90                ATT_A_EN_WIFI4_5_8Ghz_Table
                0x20000ad0                Atten_Setting
                0x20000b00                ATT_A_EN_150M_Table
                0x20000b40                ATT_B_EN_WIFI3_2_4Ghz_Table
                0x20000b80                ATT_A_EN_30G2_29_5_30Ghz_Table
                0x20000bc0                ATT_A_EN_30G1_29_5_30Ghz_Table
                0x20000c00                ATT_B_EN_30G3_29_5_30Ghz_Table
                0x20000c40                ATT_A_EN_30G1_28_5_29Ghz_Table
                0x20000c80                ATT_B_EN_30G1_29_5_30Ghz_Table
                0x20000cc0                ATT_B_EN_150M_Table
                0x20000d00                ATT_B_EN_30G3_28_28_5Ghz_Table
                0x20000d40                ATT_A_EN_WIFI1_5_8Ghz_Table
                0x20000d80                ATT_B_EN_WIFI1_5_8Ghz_Table
                0x20000dc0                ATT_B_EN_30G2_29_5_30Ghz_Table
                0x20000e00                ATT_A_EN_30G2_28_28_5Ghz_Table
                0x20000e40                ATT_A_EN_WIFI2_2_4Ghz_Table
                0x20000e80                ATT_Curr_Value
                0x20000e90                ATT_A_EN_30G1_29_29_5Ghz_Table
                0x20000ed0                ATT_A_EN_WIFI2_5_8Ghz_Table
 COMMON         0x20000f10      0x208 Src\main.o
                0x20000f10                hi2c3
                0x20000f64                hdma_usart3_rx
                0x20000fc4                UartDataisReved
                0x20000fc8                huart3
                0x20001008                rx2_data
                0x2000100c                hdma_usart3_tx
                0x2000106c                count_out
                0x2000106d                count_in
                0x2000106e                ring_buf
                0x200010d4                htim6
                0x20001114                Timer10ms
 COMMON         0x20001118      0x818 Src\uart.o
                0x20001118                TerminalQueue
                0x20001524                WifiQueue
 COMMON         0x20001930        0x4 c:/program files (x86)/atollic/truestudio for stm32 9.3.0/armtools/bin/../lib/gcc/arm-atollic-eabi/6.3.1/../../../../arm-atollic-eabi/lib/armv7-m\libc_nano.a(lib_a-reent.o)
                0x20001930                errno
                0x20001934                . = ALIGN (0x4)
                0x20001934                _ebss = .
                0x20001934                __bss_end__ = _ebss

._user_heap_stack
                0x20001934      0x600 load address 0x0800c17c
                0x20001934                . = ALIGN (0x4)
                0x20001934                PROVIDE (end, .)
                [!provide]                PROVIDE (_end, .)
                0x20001b34                . = (. + _Min_Heap_Size)
 *fill*         0x20001934      0x200 
                0x20001f34                . = (. + _Min_Stack_Size)
 *fill*         0x20001b34      0x400 
                0x20001f34                . = ALIGN (0x4)

/DISCARD/
 libc.a(*)
 libm.a(*)
 libgcc.a(*)

.ARM.attributes
                0x00000000       0x29
 *(.ARM.attributes)
 .ARM.attributes
                0x00000000       0x1d c:/program files (x86)/atollic/truestudio for stm32 9.3.0/armtools/bin/../lib/gcc/arm-atollic-eabi/6.3.1/armv7-m/crti.o
 .ARM.attributes
                0x0000001d       0x2d c:/program files (x86)/atollic/truestudio for stm32 9.3.0/armtools/bin/../lib/gcc/arm-atollic-eabi/6.3.1/armv7-m/crtbegin.o
 .ARM.attributes
                0x0000004a       0x33 Drivers\STM32F2xx_HAL_Driver\Src\stm32f2xx_hal.o
 .ARM.attributes
                0x0000007d       0x33 Drivers\STM32F2xx_HAL_Driver\Src\stm32f2xx_hal_cortex.o
 .ARM.attributes
                0x000000b0       0x33 Drivers\STM32F2xx_HAL_Driver\Src\stm32f2xx_hal_dma.o
 .ARM.attributes
                0x000000e3       0x33 Drivers\STM32F2xx_HAL_Driver\Src\stm32f2xx_hal_gpio.o
 .ARM.attributes
                0x00000116       0x33 Drivers\STM32F2xx_HAL_Driver\Src\stm32f2xx_hal_i2c.o
 .ARM.attributes
                0x00000149       0x33 Drivers\STM32F2xx_HAL_Driver\Src\stm32f2xx_hal_rcc.o
 .ARM.attributes
                0x0000017c       0x33 Drivers\STM32F2xx_HAL_Driver\Src\stm32f2xx_hal_tim.o
 .ARM.attributes
                0x000001af       0x33 Drivers\STM32F2xx_HAL_Driver\Src\stm32f2xx_hal_tim_ex.o
 .ARM.attributes
                0x000001e2       0x33 Drivers\STM32F2xx_HAL_Driver\Src\stm32f2xx_hal_uart.o
 .ARM.attributes
                0x00000215       0x33 Src\Character_lcd.o
 .ARM.attributes
                0x00000248       0x33 Src\atten_ctrl.o
 .ARM.attributes
                0x0000027b       0x33 Src\eeprom.o
 .ARM.attributes
                0x000002ae       0x33 Src\main.o
 .ARM.attributes
                0x000002e1       0x33 Src\sth30_crc.o
 .ARM.attributes
                0x00000314       0x33 Src\stm32f2xx_hal_msp.o
 .ARM.attributes
                0x00000347       0x33 Src\stm32f2xx_it.o
 .ARM.attributes
                0x0000037a       0x33 Src\syscalls.o
 .ARM.attributes
                0x000003ad       0x33 Src\system_stm32f2xx.o
 .ARM.attributes
                0x000003e0       0x33 Src\uart.o
 .ARM.attributes
                0x00000413       0x21 startup\startup_stm32f207xx.o
 .ARM.attributes
                0x00000434       0x2d c:/program files (x86)/atollic/truestudio for stm32 9.3.0/armtools/bin/../lib/gcc/arm-atollic-eabi/6.3.1/../../../../arm-atollic-eabi/lib/armv7-m\libc_nano.a(lib_a-errno.o)
 .ARM.attributes
                0x00000461       0x2d c:/program files (x86)/atollic/truestudio for stm32 9.3.0/armtools/bin/../lib/gcc/arm-atollic-eabi/6.3.1/../../../../arm-atollic-eabi/lib/armv7-m\libc_nano.a(lib_a-impure.o)
 .ARM.attributes
                0x0000048e       0x2d c:/program files (x86)/atollic/truestudio for stm32 9.3.0/armtools/bin/../lib/gcc/arm-atollic-eabi/6.3.1/../../../../arm-atollic-eabi/lib/armv7-m\libc_nano.a(lib_a-init.o)
 .ARM.attributes
                0x000004bb       0x2d c:/program files (x86)/atollic/truestudio for stm32 9.3.0/armtools/bin/../lib/gcc/arm-atollic-eabi/6.3.1/../../../../arm-atollic-eabi/lib/armv7-m\libc_nano.a(lib_a-memcpy-stub.o)
 .ARM.attributes
                0x000004e8       0x2d c:/program files (x86)/atollic/truestudio for stm32 9.3.0/armtools/bin/../lib/gcc/arm-atollic-eabi/6.3.1/../../../../arm-atollic-eabi/lib/armv7-m\libc_nano.a(lib_a-memset.o)
 .ARM.attributes
                0x00000515       0x2d c:/program files (x86)/atollic/truestudio for stm32 9.3.0/armtools/bin/../lib/gcc/arm-atollic-eabi/6.3.1/../../../../arm-atollic-eabi/lib/armv7-m\libc_nano.a(lib_a-nano-vfprintf_float.o)
 .ARM.attributes
                0x00000542       0x2d c:/program files (x86)/atollic/truestudio for stm32 9.3.0/armtools/bin/../lib/gcc/arm-atollic-eabi/6.3.1/../../../../arm-atollic-eabi/lib/armv7-m\libc_nano.a(lib_a-nano-vfprintf_i.o)
 .ARM.attributes
                0x0000056f       0x2d c:/program files (x86)/atollic/truestudio for stm32 9.3.0/armtools/bin/../lib/gcc/arm-atollic-eabi/6.3.1/../../../../arm-atollic-eabi/lib/armv7-m\libc_nano.a(lib_a-printf.o)
 .ARM.attributes
                0x0000059c       0x2d c:/program files (x86)/atollic/truestudio for stm32 9.3.0/armtools/bin/../lib/gcc/arm-atollic-eabi/6.3.1/../../../../arm-atollic-eabi/lib/armv7-m\libc_nano.a(lib_a-puts.o)
 .ARM.attributes
                0x000005c9       0x2d c:/program files (x86)/atollic/truestudio for stm32 9.3.0/armtools/bin/../lib/gcc/arm-atollic-eabi/6.3.1/../../../../arm-atollic-eabi/lib/armv7-m\libc_nano.a(lib_a-setbuf.o)
 .ARM.attributes
                0x000005f6       0x2d c:/program files (x86)/atollic/truestudio for stm32 9.3.0/armtools/bin/../lib/gcc/arm-atollic-eabi/6.3.1/../../../../arm-atollic-eabi/lib/armv7-m\libc_nano.a(lib_a-setvbuf.o)
 .ARM.attributes
                0x00000623       0x2d c:/program files (x86)/atollic/truestudio for stm32 9.3.0/armtools/bin/../lib/gcc/arm-atollic-eabi/6.3.1/../../../../arm-atollic-eabi/lib/armv7-m\libc_nano.a(lib_a-sprintf.o)
 .ARM.attributes
                0x00000650       0x2d c:/program files (x86)/atollic/truestudio for stm32 9.3.0/armtools/bin/../lib/gcc/arm-atollic-eabi/6.3.1/../../../../arm-atollic-eabi/lib/armv7-m\libc_nano.a(lib_a-strcpy.o)
 .ARM.attributes
                0x0000067d       0x17 c:/program files (x86)/atollic/truestudio for stm32 9.3.0/armtools/bin/../lib/gcc/arm-atollic-eabi/6.3.1/../../../../arm-atollic-eabi/lib/armv7-m\libc_nano.a(lib_a-strlen.o)
 .ARM.attributes
                0x00000694       0x2d c:/program files (x86)/atollic/truestudio for stm32 9.3.0/armtools/bin/../lib/gcc/arm-atollic-eabi/6.3.1/../../../../arm-atollic-eabi/lib/armv7-m\libc_nano.a(lib_a-wbuf.o)
 .ARM.attributes
                0x000006c1       0x2d c:/program files (x86)/atollic/truestudio for stm32 9.3.0/armtools/bin/../lib/gcc/arm-atollic-eabi/6.3.1/../../../../arm-atollic-eabi/lib/armv7-m\libc_nano.a(lib_a-wsetup.o)
 .ARM.attributes
                0x000006ee       0x2d c:/program files (x86)/atollic/truestudio for stm32 9.3.0/armtools/bin/../lib/gcc/arm-atollic-eabi/6.3.1/../../../../arm-atollic-eabi/lib/armv7-m\libc_nano.a(lib_a-dtoa.o)
 .ARM.attributes
                0x0000071b       0x2d c:/program files (x86)/atollic/truestudio for stm32 9.3.0/armtools/bin/../lib/gcc/arm-atollic-eabi/6.3.1/../../../../arm-atollic-eabi/lib/armv7-m\libc_nano.a(lib_a-fflush.o)
 .ARM.attributes
                0x00000748       0x2d c:/program files (x86)/atollic/truestudio for stm32 9.3.0/armtools/bin/../lib/gcc/arm-atollic-eabi/6.3.1/../../../../arm-atollic-eabi/lib/armv7-m\libc_nano.a(lib_a-findfp.o)
 .ARM.attributes
                0x00000775       0x2d c:/program files (x86)/atollic/truestudio for stm32 9.3.0/armtools/bin/../lib/gcc/arm-atollic-eabi/6.3.1/../../../../arm-atollic-eabi/lib/armv7-m\libc_nano.a(lib_a-fwalk.o)
 .ARM.attributes
                0x000007a2       0x2d c:/program files (x86)/atollic/truestudio for stm32 9.3.0/armtools/bin/../lib/gcc/arm-atollic-eabi/6.3.1/../../../../arm-atollic-eabi/lib/armv7-m\libc_nano.a(lib_a-localeconv.o)
 .ARM.attributes
                0x000007cf       0x2d c:/program files (x86)/atollic/truestudio for stm32 9.3.0/armtools/bin/../lib/gcc/arm-atollic-eabi/6.3.1/../../../../arm-atollic-eabi/lib/armv7-m\libc_nano.a(lib_a-makebuf.o)
 .ARM.attributes
                0x000007fc       0x2d c:/program files (x86)/atollic/truestudio for stm32 9.3.0/armtools/bin/../lib/gcc/arm-atollic-eabi/6.3.1/../../../../arm-atollic-eabi/lib/armv7-m\libc_nano.a(lib_a-malloc.o)
 .ARM.attributes
                0x00000829       0x2d c:/program files (x86)/atollic/truestudio for stm32 9.3.0/armtools/bin/../lib/gcc/arm-atollic-eabi/6.3.1/../../../../arm-atollic-eabi/lib/armv7-m\libc_nano.a(lib_a-memchr-stub.o)
 .ARM.attributes
                0x00000856       0x2d c:/program files (x86)/atollic/truestudio for stm32 9.3.0/armtools/bin/../lib/gcc/arm-atollic-eabi/6.3.1/../../../../arm-atollic-eabi/lib/armv7-m\libc_nano.a(lib_a-mprec.o)
 .ARM.attributes
                0x00000883       0x2d c:/program files (x86)/atollic/truestudio for stm32 9.3.0/armtools/bin/../lib/gcc/arm-atollic-eabi/6.3.1/../../../../arm-atollic-eabi/lib/armv7-m\libc_nano.a(lib_a-nano-callocr.o)
 .ARM.attributes
                0x000008b0       0x2d c:/program files (x86)/atollic/truestudio for stm32 9.3.0/armtools/bin/../lib/gcc/arm-atollic-eabi/6.3.1/../../../../arm-atollic-eabi/lib/armv7-m\libc_nano.a(lib_a-nano-freer.o)
 .ARM.attributes
                0x000008dd       0x2d c:/program files (x86)/atollic/truestudio for stm32 9.3.0/armtools/bin/../lib/gcc/arm-atollic-eabi/6.3.1/../../../../arm-atollic-eabi/lib/armv7-m\libc_nano.a(lib_a-nano-mallocr.o)
 .ARM.attributes
                0x0000090a       0x2d c:/program files (x86)/atollic/truestudio for stm32 9.3.0/armtools/bin/../lib/gcc/arm-atollic-eabi/6.3.1/../../../../arm-atollic-eabi/lib/armv7-m\libc_nano.a(lib_a-nano-svfprintf.o)
 .ARM.attributes
                0x00000937       0x2d c:/program files (x86)/atollic/truestudio for stm32 9.3.0/armtools/bin/../lib/gcc/arm-atollic-eabi/6.3.1/../../../../arm-atollic-eabi/lib/armv7-m\libc_nano.a(lib_a-nano-vfprintf.o)
 .ARM.attributes
                0x00000964       0x2d c:/program files (x86)/atollic/truestudio for stm32 9.3.0/armtools/bin/../lib/gcc/arm-atollic-eabi/6.3.1/../../../../arm-atollic-eabi/lib/armv7-m\libc_nano.a(lib_a-sbrkr.o)
 .ARM.attributes
                0x00000991       0x2d c:/program files (x86)/atollic/truestudio for stm32 9.3.0/armtools/bin/../lib/gcc/arm-atollic-eabi/6.3.1/../../../../arm-atollic-eabi/lib/armv7-m\libc_nano.a(lib_a-stdio.o)
 .ARM.attributes
                0x000009be       0x2d c:/program files (x86)/atollic/truestudio for stm32 9.3.0/armtools/bin/../lib/gcc/arm-atollic-eabi/6.3.1/../../../../arm-atollic-eabi/lib/armv7-m\libc_nano.a(lib_a-writer.o)
 .ARM.attributes
                0x000009eb       0x2d c:/program files (x86)/atollic/truestudio for stm32 9.3.0/armtools/bin/../lib/gcc/arm-atollic-eabi/6.3.1/../../../../arm-atollic-eabi/lib/armv7-m\libc_nano.a(lib_a-closer.o)
 .ARM.attributes
                0x00000a18       0x2d c:/program files (x86)/atollic/truestudio for stm32 9.3.0/armtools/bin/../lib/gcc/arm-atollic-eabi/6.3.1/../../../../arm-atollic-eabi/lib/armv7-m\libc_nano.a(lib_a-fstatr.o)
 .ARM.attributes
                0x00000a45       0x2d c:/program files (x86)/atollic/truestudio for stm32 9.3.0/armtools/bin/../lib/gcc/arm-atollic-eabi/6.3.1/../../../../arm-atollic-eabi/lib/armv7-m\libc_nano.a(lib_a-isattyr.o)
 .ARM.attributes
                0x00000a72       0x2d c:/program files (x86)/atollic/truestudio for stm32 9.3.0/armtools/bin/../lib/gcc/arm-atollic-eabi/6.3.1/../../../../arm-atollic-eabi/lib/armv7-m\libc_nano.a(lib_a-locale.o)
 .ARM.attributes
                0x00000a9f       0x2d c:/program files (x86)/atollic/truestudio for stm32 9.3.0/armtools/bin/../lib/gcc/arm-atollic-eabi/6.3.1/../../../../arm-atollic-eabi/lib/armv7-m\libc_nano.a(lib_a-lseekr.o)
 .ARM.attributes
                0x00000acc       0x2d c:/program files (x86)/atollic/truestudio for stm32 9.3.0/armtools/bin/../lib/gcc/arm-atollic-eabi/6.3.1/../../../../arm-atollic-eabi/lib/armv7-m\libc_nano.a(lib_a-mbtowc_r.o)
 .ARM.attributes
                0x00000af9       0x2d c:/program files (x86)/atollic/truestudio for stm32 9.3.0/armtools/bin/../lib/gcc/arm-atollic-eabi/6.3.1/../../../../arm-atollic-eabi/lib/armv7-m\libc_nano.a(lib_a-memmove.o)
 .ARM.attributes
                0x00000b26       0x2d c:/program files (x86)/atollic/truestudio for stm32 9.3.0/armtools/bin/../lib/gcc/arm-atollic-eabi/6.3.1/../../../../arm-atollic-eabi/lib/armv7-m\libc_nano.a(lib_a-mlock.o)
 .ARM.attributes
                0x00000b53       0x2d c:/program files (x86)/atollic/truestudio for stm32 9.3.0/armtools/bin/../lib/gcc/arm-atollic-eabi/6.3.1/../../../../arm-atollic-eabi/lib/armv7-m\libc_nano.a(lib_a-nano-reallocr.o)
 .ARM.attributes
                0x00000b80       0x2d c:/program files (x86)/atollic/truestudio for stm32 9.3.0/armtools/bin/../lib/gcc/arm-atollic-eabi/6.3.1/../../../../arm-atollic-eabi/lib/armv7-m\libc_nano.a(lib_a-readr.o)
 .ARM.attributes
                0x00000bad       0x2d c:/program files (x86)/atollic/truestudio for stm32 9.3.0/armtools/bin/../lib/gcc/arm-atollic-eabi/6.3.1/../../../../arm-atollic-eabi/lib/armv7-m\libc_nano.a(lib_a-reent.o)
 .ARM.attributes
                0x00000bda       0x2d c:/program files (x86)/atollic/truestudio for stm32 9.3.0/armtools/bin/../lib/gcc/arm-atollic-eabi/6.3.1/../../../../arm-atollic-eabi/lib/armv7-m\libc_nano.a(lib_a-wctomb_r.o)
 .ARM.attributes
                0x00000c07       0x2d c:/program files (x86)/atollic/truestudio for stm32 9.3.0/armtools/bin/../lib/gcc/arm-atollic-eabi/6.3.1/../../../../arm-atollic-eabi/lib/armv7-m\libc_nano.a(lib_a-ctype_.o)
 .ARM.attributes
                0x00000c34       0x2d c:/program files (x86)/atollic/truestudio for stm32 9.3.0/armtools/bin/../lib/gcc/arm-atollic-eabi/6.3.1/../../../../arm-atollic-eabi/lib/armv7-m\libc_nano.a(lib_a-nano-msizer.o)
 .ARM.attributes
                0x00000c61       0x1d c:/program files (x86)/atollic/truestudio for stm32 9.3.0/armtools/bin/../lib/gcc/arm-atollic-eabi/6.3.1/armv7-m\libgcc.a(_arm_addsubdf3.o)
 .ARM.attributes
                0x00000c7e       0x1d c:/program files (x86)/atollic/truestudio for stm32 9.3.0/armtools/bin/../lib/gcc/arm-atollic-eabi/6.3.1/armv7-m\libgcc.a(_arm_muldivdf3.o)
 .ARM.attributes
                0x00000c9b       0x1d c:/program files (x86)/atollic/truestudio for stm32 9.3.0/armtools/bin/../lib/gcc/arm-atollic-eabi/6.3.1/armv7-m\libgcc.a(_arm_cmpdf2.o)
 .ARM.attributes
                0x00000cb8       0x1d c:/program files (x86)/atollic/truestudio for stm32 9.3.0/armtools/bin/../lib/gcc/arm-atollic-eabi/6.3.1/armv7-m\libgcc.a(_arm_unorddf2.o)
 .ARM.attributes
                0x00000cd5       0x1d c:/program files (x86)/atollic/truestudio for stm32 9.3.0/armtools/bin/../lib/gcc/arm-atollic-eabi/6.3.1/armv7-m\libgcc.a(_arm_fixdfsi.o)
 .ARM.attributes
                0x00000cf2       0x1d c:/program files (x86)/atollic/truestudio for stm32 9.3.0/armtools/bin/../lib/gcc/arm-atollic-eabi/6.3.1/armv7-m\libgcc.a(_arm_addsubsf3.o)
 .ARM.attributes
                0x00000d0f       0x1d c:/program files (x86)/atollic/truestudio for stm32 9.3.0/armtools/bin/../lib/gcc/arm-atollic-eabi/6.3.1/armv7-m\libgcc.a(_arm_cmpsf2.o)
 .ARM.attributes
                0x00000d2c       0x1d c:/program files (x86)/atollic/truestudio for stm32 9.3.0/armtools/bin/../lib/gcc/arm-atollic-eabi/6.3.1/armv7-m\libgcc.a(_arm_fixunssfsi.o)
 .ARM.attributes
                0x00000d49       0x1d c:/program files (x86)/atollic/truestudio for stm32 9.3.0/armtools/bin/../lib/gcc/arm-atollic-eabi/6.3.1/armv7-m\libgcc.a(_aeabi_uldivmod.o)
 .ARM.attributes
                0x00000d66       0x2d c:/program files (x86)/atollic/truestudio for stm32 9.3.0/armtools/bin/../lib/gcc/arm-atollic-eabi/6.3.1/armv7-m\libgcc.a(_udivmoddi4.o)
 .ARM.attributes
                0x00000d93       0x1d c:/program files (x86)/atollic/truestudio for stm32 9.3.0/armtools/bin/../lib/gcc/arm-atollic-eabi/6.3.1/armv7-m\libgcc.a(_dvmd_tls.o)
 .ARM.attributes
                0x00000db0       0x1d c:/program files (x86)/atollic/truestudio for stm32 9.3.0/armtools/bin/../lib/gcc/arm-atollic-eabi/6.3.1/armv7-m/crtn.o
OUTPUT(STM32F207_ChannelCtrlProject.elf elf32-littlearm)

.debug_info     0x00000000    0x22faa
 .debug_info    0x00000000      0xa7d Drivers\STM32F2xx_HAL_Driver\Src\stm32f2xx_hal.o
 .debug_info    0x00000a7d      0xf88 Drivers\STM32F2xx_HAL_Driver\Src\stm32f2xx_hal_cortex.o
 .debug_info    0x00001a05      0xa9d Drivers\STM32F2xx_HAL_Driver\Src\stm32f2xx_hal_dma.o
 .debug_info    0x000024a2      0x78e Drivers\STM32F2xx_HAL_Driver\Src\stm32f2xx_hal_gpio.o
 .debug_info    0x00002c30     0x3382 Drivers\STM32F2xx_HAL_Driver\Src\stm32f2xx_hal_i2c.o
 .debug_info    0x00005fb2      0xd4d Drivers\STM32F2xx_HAL_Driver\Src\stm32f2xx_hal_rcc.o
 .debug_info    0x00006cff     0x351f Drivers\STM32F2xx_HAL_Driver\Src\stm32f2xx_hal_tim.o
 .debug_info    0x0000a21e     0x134f Drivers\STM32F2xx_HAL_Driver\Src\stm32f2xx_hal_tim_ex.o
 .debug_info    0x0000b56d     0x1696 Drivers\STM32F2xx_HAL_Driver\Src\stm32f2xx_hal_uart.o
 .debug_info    0x0000cc03     0x3cfe Src\Character_lcd.o
 .debug_info    0x00010901     0x47d2 Src\atten_ctrl.o
 .debug_info    0x000150d3     0x24a5 Src\eeprom.o
 .debug_info    0x00017578     0x38fb Src\main.o
 .debug_info    0x0001ae73      0xa0e Src\sth30_crc.o
 .debug_info    0x0001b881     0x25b1 Src\stm32f2xx_hal_msp.o
 .debug_info    0x0001de32     0x1f29 Src\stm32f2xx_it.o
 .debug_info    0x0001fd5b      0xfe1 Src\syscalls.o
 .debug_info    0x00020d3c      0x55b Src\system_stm32f2xx.o
 .debug_info    0x00021297     0x1c9d Src\uart.o
 .debug_info    0x00022f34       0x76 startup\startup_stm32f207xx.o

.debug_abbrev   0x00000000     0x37ca
 .debug_abbrev  0x00000000      0x285 Drivers\STM32F2xx_HAL_Driver\Src\stm32f2xx_hal.o
 .debug_abbrev  0x00000285      0x31d Drivers\STM32F2xx_HAL_Driver\Src\stm32f2xx_hal_cortex.o
 .debug_abbrev  0x000005a2      0x2e8 Drivers\STM32F2xx_HAL_Driver\Src\stm32f2xx_hal_dma.o
 .debug_abbrev  0x0000088a      0x1e6 Drivers\STM32F2xx_HAL_Driver\Src\stm32f2xx_hal_gpio.o
 .debug_abbrev  0x00000a70      0x38a Drivers\STM32F2xx_HAL_Driver\Src\stm32f2xx_hal_i2c.o
 .debug_abbrev  0x00000dfa      0x2f8 Drivers\STM32F2xx_HAL_Driver\Src\stm32f2xx_hal_rcc.o
 .debug_abbrev  0x000010f2      0x335 Drivers\STM32F2xx_HAL_Driver\Src\stm32f2xx_hal_tim.o
 .debug_abbrev  0x00001427      0x29c Drivers\STM32F2xx_HAL_Driver\Src\stm32f2xx_hal_tim_ex.o
 .debug_abbrev  0x000016c3      0x304 Drivers\STM32F2xx_HAL_Driver\Src\stm32f2xx_hal_uart.o
 .debug_abbrev  0x000019c7      0x4a7 Src\Character_lcd.o
 .debug_abbrev  0x00001e6e      0x41e Src\atten_ctrl.o
 .debug_abbrev  0x0000228c      0x254 Src\eeprom.o
 .debug_abbrev  0x000024e0      0x505 Src\main.o
 .debug_abbrev  0x000029e5      0x201 Src\sth30_crc.o
 .debug_abbrev  0x00002be6      0x2bd Src\stm32f2xx_hal_msp.o
 .debug_abbrev  0x00002ea3      0x28e Src\stm32f2xx_it.o
 .debug_abbrev  0x00003131      0x2d9 Src\syscalls.o
 .debug_abbrev  0x0000340a      0x126 Src\system_stm32f2xx.o
 .debug_abbrev  0x00003530      0x288 Src\uart.o
 .debug_abbrev  0x000037b8       0x12 startup\startup_stm32f207xx.o

.debug_loc      0x00000000     0xdc5a
 .debug_loc     0x00000000      0x133 Drivers\STM32F2xx_HAL_Driver\Src\stm32f2xx_hal.o
 .debug_loc     0x00000133      0x4a8 Drivers\STM32F2xx_HAL_Driver\Src\stm32f2xx_hal_cortex.o
 .debug_loc     0x000005db      0x735 Drivers\STM32F2xx_HAL_Driver\Src\stm32f2xx_hal_dma.o
 .debug_loc     0x00000d10      0x2d3 Drivers\STM32F2xx_HAL_Driver\Src\stm32f2xx_hal_gpio.o
 .debug_loc     0x00000fe3     0x2fa9 Drivers\STM32F2xx_HAL_Driver\Src\stm32f2xx_hal_i2c.o
 .debug_loc     0x00003f8c      0x50c Drivers\STM32F2xx_HAL_Driver\Src\stm32f2xx_hal_rcc.o
 .debug_loc     0x00004498     0x301c Drivers\STM32F2xx_HAL_Driver\Src\stm32f2xx_hal_tim.o
 .debug_loc     0x000074b4      0xa7c Drivers\STM32F2xx_HAL_Driver\Src\stm32f2xx_hal_tim_ex.o
 .debug_loc     0x00007f30     0x1374 Drivers\STM32F2xx_HAL_Driver\Src\stm32f2xx_hal_uart.o
 .debug_loc     0x000092a4      0x5fa Src\Character_lcd.o
 .debug_loc     0x0000989e     0x36b1 Src\atten_ctrl.o
 .debug_loc     0x0000cf4f      0x15e Src\eeprom.o
 .debug_loc     0x0000d0ad      0x29c Src\main.o
 .debug_loc     0x0000d349      0x222 Src\sth30_crc.o
 .debug_loc     0x0000d56b       0xe7 Src\stm32f2xx_hal_msp.o
 .debug_loc     0x0000d652      0x3ef Src\syscalls.o
 .debug_loc     0x0000da41      0x11c Src\system_stm32f2xx.o
 .debug_loc     0x0000db5d       0xfd Src\uart.o

.debug_aranges  0x00000000      0xeb0
 .debug_aranges
                0x00000000       0xe8 Drivers\STM32F2xx_HAL_Driver\Src\stm32f2xx_hal.o
 .debug_aranges
                0x000000e8       0xa8 Drivers\STM32F2xx_HAL_Driver\Src\stm32f2xx_hal_cortex.o
 .debug_aranges
                0x00000190       0x80 Drivers\STM32F2xx_HAL_Driver\Src\stm32f2xx_hal_dma.o
 .debug_aranges
                0x00000210       0x58 Drivers\STM32F2xx_HAL_Driver\Src\stm32f2xx_hal_gpio.o
 .debug_aranges
                0x00000268      0x1b0 Drivers\STM32F2xx_HAL_Driver\Src\stm32f2xx_hal_i2c.o
 .debug_aranges
                0x00000418       0x88 Drivers\STM32F2xx_HAL_Driver\Src\stm32f2xx_hal_rcc.o
 .debug_aranges
                0x000004a0      0x278 Drivers\STM32F2xx_HAL_Driver\Src\stm32f2xx_hal_tim.o
 .debug_aranges
                0x00000718       0xf8 Drivers\STM32F2xx_HAL_Driver\Src\stm32f2xx_hal_tim_ex.o
 .debug_aranges
                0x00000810      0x170 Drivers\STM32F2xx_HAL_Driver\Src\stm32f2xx_hal_uart.o
 .debug_aranges
                0x00000980      0x120 Src\Character_lcd.o
 .debug_aranges
                0x00000aa0      0x118 Src\atten_ctrl.o
 .debug_aranges
                0x00000bb8       0x30 Src\eeprom.o
 .debug_aranges
                0x00000be8       0x90 Src\main.o
 .debug_aranges
                0x00000c78       0x30 Src\sth30_crc.o
 .debug_aranges
                0x00000ca8       0x50 Src\stm32f2xx_hal_msp.o
 .debug_aranges
                0x00000cf8       0x78 Src\stm32f2xx_it.o
 .debug_aranges
                0x00000d70       0xb0 Src\syscalls.o
 .debug_aranges
                0x00000e20       0x28 Src\system_stm32f2xx.o
 .debug_aranges
                0x00000e48       0x40 Src\uart.o
 .debug_aranges
                0x00000e88       0x28 startup\startup_stm32f207xx.o

.debug_ranges   0x00000000     0x1650
 .debug_ranges  0x00000000       0xd8 Drivers\STM32F2xx_HAL_Driver\Src\stm32f2xx_hal.o
 .debug_ranges  0x000000d8      0x140 Drivers\STM32F2xx_HAL_Driver\Src\stm32f2xx_hal_cortex.o
 .debug_ranges  0x00000218       0xd8 Drivers\STM32F2xx_HAL_Driver\Src\stm32f2xx_hal_dma.o
 .debug_ranges  0x000002f0       0x78 Drivers\STM32F2xx_HAL_Driver\Src\stm32f2xx_hal_gpio.o
 .debug_ranges  0x00000368      0x4b8 Drivers\STM32F2xx_HAL_Driver\Src\stm32f2xx_hal_i2c.o
 .debug_ranges  0x00000820      0x178 Drivers\STM32F2xx_HAL_Driver\Src\stm32f2xx_hal_rcc.o
 .debug_ranges  0x00000998      0x348 Drivers\STM32F2xx_HAL_Driver\Src\stm32f2xx_hal_tim.o
 .debug_ranges  0x00000ce0       0xe8 Drivers\STM32F2xx_HAL_Driver\Src\stm32f2xx_hal_tim_ex.o
 .debug_ranges  0x00000dc8      0x190 Drivers\STM32F2xx_HAL_Driver\Src\stm32f2xx_hal_uart.o
 .debug_ranges  0x00000f58      0x150 Src\Character_lcd.o
 .debug_ranges  0x000010a8      0x120 Src\atten_ctrl.o
 .debug_ranges  0x000011c8       0x20 Src\eeprom.o
 .debug_ranges  0x000011e8      0x208 Src\main.o
 .debug_ranges  0x000013f0       0x20 Src\sth30_crc.o
 .debug_ranges  0x00001410       0xd0 Src\stm32f2xx_hal_msp.o
 .debug_ranges  0x000014e0       0x68 Src\stm32f2xx_it.o
 .debug_ranges  0x00001548       0xa0 Src\syscalls.o
 .debug_ranges  0x000015e8       0x18 Src\system_stm32f2xx.o
 .debug_ranges  0x00001600       0x30 Src\uart.o
 .debug_ranges  0x00001630       0x20 startup\startup_stm32f207xx.o

.debug_line     0x00000000     0x9279
 .debug_line    0x00000000      0x446 Drivers\STM32F2xx_HAL_Driver\Src\stm32f2xx_hal.o
 .debug_line    0x00000446      0x478 Drivers\STM32F2xx_HAL_Driver\Src\stm32f2xx_hal_cortex.o
 .debug_line    0x000008be      0x58d Drivers\STM32F2xx_HAL_Driver\Src\stm32f2xx_hal_dma.o
 .debug_line    0x00000e4b      0x3f0 Drivers\STM32F2xx_HAL_Driver\Src\stm32f2xx_hal_gpio.o
 .debug_line    0x0000123b     0x1dd3 Drivers\STM32F2xx_HAL_Driver\Src\stm32f2xx_hal_i2c.o
 .debug_line    0x0000300e      0x5e7 Drivers\STM32F2xx_HAL_Driver\Src\stm32f2xx_hal_rcc.o
 .debug_line    0x000035f5     0x124b Drivers\STM32F2xx_HAL_Driver\Src\stm32f2xx_hal_tim.o
 .debug_line    0x00004840      0x6de Drivers\STM32F2xx_HAL_Driver\Src\stm32f2xx_hal_tim_ex.o
 .debug_line    0x00004f1e      0xbf7 Drivers\STM32F2xx_HAL_Driver\Src\stm32f2xx_hal_uart.o
 .debug_line    0x00005b15      0x9c5 Src\Character_lcd.o
 .debug_line    0x000064da      0xd28 Src\atten_ctrl.o
 .debug_line    0x00007202      0x3d8 Src\eeprom.o
 .debug_line    0x000075da      0x717 Src\main.o
 .debug_line    0x00007cf1      0x241 Src\sth30_crc.o
 .debug_line    0x00007f32      0x4c8 Src\stm32f2xx_hal_msp.o
 .debug_line    0x000083fa      0x461 Src\stm32f2xx_it.o
 .debug_line    0x0000885b      0x3c0 Src\syscalls.o
 .debug_line    0x00008c1b      0x21b Src\system_stm32f2xx.o
 .debug_line    0x00008e36      0x3c4 Src\uart.o
 .debug_line    0x000091fa       0x7f startup\startup_stm32f207xx.o

.debug_str      0x00000000     0x8d9c
 .debug_str     0x00000000      0xb21 Drivers\STM32F2xx_HAL_Driver\Src\stm32f2xx_hal.o
                                0xba3 (size before relaxing)
 .debug_str     0x00000b21      0x4a8 Drivers\STM32F2xx_HAL_Driver\Src\stm32f2xx_hal_cortex.o
                                0xce2 (size before relaxing)
 .debug_str     0x00000fc9      0x522 Drivers\STM32F2xx_HAL_Driver\Src\stm32f2xx_hal_dma.o
                                0x828 (size before relaxing)
 .debug_str     0x000014eb      0x1d6 Drivers\STM32F2xx_HAL_Driver\Src\stm32f2xx_hal_gpio.o
                                0x591 (size before relaxing)
 .debug_str     0x000016c1      0xaf9 Drivers\STM32F2xx_HAL_Driver\Src\stm32f2xx_hal_i2c.o
                               0x10af (size before relaxing)
 .debug_str     0x000021ba      0x2d1 Drivers\STM32F2xx_HAL_Driver\Src\stm32f2xx_hal_rcc.o
                                0x78a (size before relaxing)
 .debug_str     0x0000248b      0xff0 Drivers\STM32F2xx_HAL_Driver\Src\stm32f2xx_hal_tim.o
                               0x157f (size before relaxing)
 .debug_str     0x0000347b      0x548 Drivers\STM32F2xx_HAL_Driver\Src\stm32f2xx_hal_tim_ex.o
                                0xd97 (size before relaxing)
 .debug_str     0x000039c3      0x6c0 Drivers\STM32F2xx_HAL_Driver\Src\stm32f2xx_hal_uart.o
                                0xccf (size before relaxing)
 .debug_str     0x00004083     0x2a10 Src\Character_lcd.o
                               0x3419 (size before relaxing)
 .debug_str     0x00006a93     0x1bdb Src\atten_ctrl.o
                               0x46e5 (size before relaxing)
 .debug_str     0x0000866e       0x42 Src\eeprom.o
                               0x212a (size before relaxing)
 .debug_str     0x000086b0      0x24e Src\main.o
                               0x3dc6 (size before relaxing)
 .debug_str     0x000088fe       0x52 Src\sth30_crc.o
                                0x637 (size before relaxing)
 .debug_str     0x00008950       0x25 Src\stm32f2xx_hal_msp.o
                               0x29e6 (size before relaxing)
 .debug_str     0x00008975      0x124 Src\stm32f2xx_it.o
                               0x23d9 (size before relaxing)
 .debug_str     0x00008a99      0x24c Src\syscalls.o
                                0x855 (size before relaxing)
 .debug_str     0x00008ce5       0x45 Src\system_stm32f2xx.o
                                0x406 (size before relaxing)
 .debug_str     0x00008d2a       0x72 Src\uart.o
                               0x211a (size before relaxing)

.comment        0x00000000       0x7c
 .comment       0x00000000       0x7c Drivers\STM32F2xx_HAL_Driver\Src\stm32f2xx_hal.o
                                 0x7d (size before relaxing)
 .comment       0x0000007c       0x7d Drivers\STM32F2xx_HAL_Driver\Src\stm32f2xx_hal_cortex.o
 .comment       0x0000007c       0x7d Drivers\STM32F2xx_HAL_Driver\Src\stm32f2xx_hal_dma.o
 .comment       0x0000007c       0x7d Drivers\STM32F2xx_HAL_Driver\Src\stm32f2xx_hal_gpio.o
 .comment       0x0000007c       0x7d Drivers\STM32F2xx_HAL_Driver\Src\stm32f2xx_hal_i2c.o
 .comment       0x0000007c       0x7d Drivers\STM32F2xx_HAL_Driver\Src\stm32f2xx_hal_rcc.o
 .comment       0x0000007c       0x7d Drivers\STM32F2xx_HAL_Driver\Src\stm32f2xx_hal_tim.o
 .comment       0x0000007c       0x7d Drivers\STM32F2xx_HAL_Driver\Src\stm32f2xx_hal_tim_ex.o
 .comment       0x0000007c       0x7d Drivers\STM32F2xx_HAL_Driver\Src\stm32f2xx_hal_uart.o
 .comment       0x0000007c       0x7d Src\Character_lcd.o
 .comment       0x0000007c       0x7d Src\atten_ctrl.o
 .comment       0x0000007c       0x7d Src\eeprom.o
 .comment       0x0000007c       0x7d Src\main.o
 .comment       0x0000007c       0x7d Src\sth30_crc.o
 .comment       0x0000007c       0x7d Src\stm32f2xx_hal_msp.o
 .comment       0x0000007c       0x7d Src\stm32f2xx_it.o
 .comment       0x0000007c       0x7d Src\syscalls.o
 .comment       0x0000007c       0x7d Src\system_stm32f2xx.o
 .comment       0x0000007c       0x7d Src\uart.o

.debug_frame    0x00000000     0x4008
 .debug_frame   0x00000000      0x1f4 Drivers\STM32F2xx_HAL_Driver\Src\stm32f2xx_hal.o
 .debug_frame   0x000001f4      0x158 Drivers\STM32F2xx_HAL_Driver\Src\stm32f2xx_hal_cortex.o
 .debug_frame   0x0000034c      0x150 Drivers\STM32F2xx_HAL_Driver\Src\stm32f2xx_hal_dma.o
 .debug_frame   0x0000049c       0xd4 Drivers\STM32F2xx_HAL_Driver\Src\stm32f2xx_hal_gpio.o
 .debug_frame   0x00000570      0x704 Drivers\STM32F2xx_HAL_Driver\Src\stm32f2xx_hal_i2c.o
 .debug_frame   0x00000c74      0x150 Drivers\STM32F2xx_HAL_Driver\Src\stm32f2xx_hal_rcc.o
 .debug_frame   0x00000dc4      0x928 Drivers\STM32F2xx_HAL_Driver\Src\stm32f2xx_hal_tim.o
 .debug_frame   0x000016ec      0x360 Drivers\STM32F2xx_HAL_Driver\Src\stm32f2xx_hal_tim_ex.o
 .debug_frame   0x00001a4c      0x498 Drivers\STM32F2xx_HAL_Driver\Src\stm32f2xx_hal_uart.o
 .debug_frame   0x00001ee4      0x3c4 Src\Character_lcd.o
 .debug_frame   0x000022a8      0x4f8 Src\atten_ctrl.o
 .debug_frame   0x000027a0       0x68 Src\eeprom.o
 .debug_frame   0x00002808      0x144 Src\main.o
 .debug_frame   0x0000294c       0x5c Src\sth30_crc.o
 .debug_frame   0x000029a8       0xdc Src\stm32f2xx_hal_msp.o
 .debug_frame   0x00002a84      0x10c Src\stm32f2xx_it.o
 .debug_frame   0x00002b90      0x1a8 Src\syscalls.o
 .debug_frame   0x00002d38       0x38 Src\system_stm32f2xx.o
 .debug_frame   0x00002d70       0x78 Src\uart.o
 .debug_frame   0x00002de8       0x20 c:/program files (x86)/atollic/truestudio for stm32 9.3.0/armtools/bin/../lib/gcc/arm-atollic-eabi/6.3.1/../../../../arm-atollic-eabi/lib/armv7-m\libc_nano.a(lib_a-errno.o)
 .debug_frame   0x00002e08       0x2c c:/program files (x86)/atollic/truestudio for stm32 9.3.0/armtools/bin/../lib/gcc/arm-atollic-eabi/6.3.1/../../../../arm-atollic-eabi/lib/armv7-m\libc_nano.a(lib_a-init.o)
 .debug_frame   0x00002e34       0x28 c:/program files (x86)/atollic/truestudio for stm32 9.3.0/armtools/bin/../lib/gcc/arm-atollic-eabi/6.3.1/../../../../arm-atollic-eabi/lib/armv7-m\libc_nano.a(lib_a-memcpy-stub.o)
 .debug_frame   0x00002e5c       0x20 c:/program files (x86)/atollic/truestudio for stm32 9.3.0/armtools/bin/../lib/gcc/arm-atollic-eabi/6.3.1/../../../../arm-atollic-eabi/lib/armv7-m\libc_nano.a(lib_a-memset.o)
 .debug_frame   0x00002e7c       0x90 c:/program files (x86)/atollic/truestudio for stm32 9.3.0/armtools/bin/../lib/gcc/arm-atollic-eabi/6.3.1/../../../../arm-atollic-eabi/lib/armv7-m\libc_nano.a(lib_a-nano-vfprintf_float.o)
 .debug_frame   0x00002f0c       0x60 c:/program files (x86)/atollic/truestudio for stm32 9.3.0/armtools/bin/../lib/gcc/arm-atollic-eabi/6.3.1/../../../../arm-atollic-eabi/lib/armv7-m\libc_nano.a(lib_a-nano-vfprintf_i.o)
 .debug_frame   0x00002f6c       0x74 c:/program files (x86)/atollic/truestudio for stm32 9.3.0/armtools/bin/../lib/gcc/arm-atollic-eabi/6.3.1/../../../../arm-atollic-eabi/lib/armv7-m\libc_nano.a(lib_a-printf.o)
 .debug_frame   0x00002fe0       0x3c c:/program files (x86)/atollic/truestudio for stm32 9.3.0/armtools/bin/../lib/gcc/arm-atollic-eabi/6.3.1/../../../../arm-atollic-eabi/lib/armv7-m\libc_nano.a(lib_a-puts.o)
 .debug_frame   0x0000301c       0x20 c:/program files (x86)/atollic/truestudio for stm32 9.3.0/armtools/bin/../lib/gcc/arm-atollic-eabi/6.3.1/../../../../arm-atollic-eabi/lib/armv7-m\libc_nano.a(lib_a-setbuf.o)
 .debug_frame   0x0000303c       0x38 c:/program files (x86)/atollic/truestudio for stm32 9.3.0/armtools/bin/../lib/gcc/arm-atollic-eabi/6.3.1/../../../../arm-atollic-eabi/lib/armv7-m\libc_nano.a(lib_a-setvbuf.o)
 .debug_frame   0x00003074       0x70 c:/program files (x86)/atollic/truestudio for stm32 9.3.0/armtools/bin/../lib/gcc/arm-atollic-eabi/6.3.1/../../../../arm-atollic-eabi/lib/armv7-m\libc_nano.a(lib_a-sprintf.o)
 .debug_frame   0x000030e4       0x20 c:/program files (x86)/atollic/truestudio for stm32 9.3.0/armtools/bin/../lib/gcc/arm-atollic-eabi/6.3.1/../../../../arm-atollic-eabi/lib/armv7-m\libc_nano.a(lib_a-strcpy.o)
 .debug_frame   0x00003104       0x40 c:/program files (x86)/atollic/truestudio for stm32 9.3.0/armtools/bin/../lib/gcc/arm-atollic-eabi/6.3.1/../../../../arm-atollic-eabi/lib/armv7-m\libc_nano.a(lib_a-wbuf.o)
 .debug_frame   0x00003144       0x2c c:/program files (x86)/atollic/truestudio for stm32 9.3.0/armtools/bin/../lib/gcc/arm-atollic-eabi/6.3.1/../../../../arm-atollic-eabi/lib/armv7-m\libc_nano.a(lib_a-wsetup.o)
 .debug_frame   0x00003170       0x6c c:/program files (x86)/atollic/truestudio for stm32 9.3.0/armtools/bin/../lib/gcc/arm-atollic-eabi/6.3.1/../../../../arm-atollic-eabi/lib/armv7-m\libc_nano.a(lib_a-dtoa.o)
 .debug_frame   0x000031dc       0x68 c:/program files (x86)/atollic/truestudio for stm32 9.3.0/armtools/bin/../lib/gcc/arm-atollic-eabi/6.3.1/../../../../arm-atollic-eabi/lib/armv7-m\libc_nano.a(lib_a-fflush.o)
 .debug_frame   0x00003244      0x11c c:/program files (x86)/atollic/truestudio for stm32 9.3.0/armtools/bin/../lib/gcc/arm-atollic-eabi/6.3.1/../../../../arm-atollic-eabi/lib/armv7-m\libc_nano.a(lib_a-findfp.o)
 .debug_frame   0x00003360       0x54 c:/program files (x86)/atollic/truestudio for stm32 9.3.0/armtools/bin/../lib/gcc/arm-atollic-eabi/6.3.1/../../../../arm-atollic-eabi/lib/armv7-m\libc_nano.a(lib_a-fwalk.o)
 .debug_frame   0x000033b4       0x40 c:/program files (x86)/atollic/truestudio for stm32 9.3.0/armtools/bin/../lib/gcc/arm-atollic-eabi/6.3.1/../../../../arm-atollic-eabi/lib/armv7-m\libc_nano.a(lib_a-localeconv.o)
 .debug_frame   0x000033f4       0x58 c:/program files (x86)/atollic/truestudio for stm32 9.3.0/armtools/bin/../lib/gcc/arm-atollic-eabi/6.3.1/../../../../arm-atollic-eabi/lib/armv7-m\libc_nano.a(lib_a-makebuf.o)
 .debug_frame   0x0000344c       0x30 c:/program files (x86)/atollic/truestudio for stm32 9.3.0/armtools/bin/../lib/gcc/arm-atollic-eabi/6.3.1/../../../../arm-atollic-eabi/lib/armv7-m\libc_nano.a(lib_a-malloc.o)
 .debug_frame   0x0000347c       0x28 c:/program files (x86)/atollic/truestudio for stm32 9.3.0/armtools/bin/../lib/gcc/arm-atollic-eabi/6.3.1/../../../../arm-atollic-eabi/lib/armv7-m\libc_nano.a(lib_a-memchr-stub.o)
 .debug_frame   0x000034a4      0x244 c:/program files (x86)/atollic/truestudio for stm32 9.3.0/armtools/bin/../lib/gcc/arm-atollic-eabi/6.3.1/../../../../arm-atollic-eabi/lib/armv7-m\libc_nano.a(lib_a-mprec.o)
 .debug_frame   0x000036e8       0x2c c:/program files (x86)/atollic/truestudio for stm32 9.3.0/armtools/bin/../lib/gcc/arm-atollic-eabi/6.3.1/../../../../arm-atollic-eabi/lib/armv7-m\libc_nano.a(lib_a-nano-callocr.o)
 .debug_frame   0x00003714       0x38 c:/program files (x86)/atollic/truestudio for stm32 9.3.0/armtools/bin/../lib/gcc/arm-atollic-eabi/6.3.1/../../../../arm-atollic-eabi/lib/armv7-m\libc_nano.a(lib_a-nano-freer.o)
 .debug_frame   0x0000374c       0x2c c:/program files (x86)/atollic/truestudio for stm32 9.3.0/armtools/bin/../lib/gcc/arm-atollic-eabi/6.3.1/../../../../arm-atollic-eabi/lib/armv7-m\libc_nano.a(lib_a-nano-mallocr.o)
 .debug_frame   0x00003778       0x90 c:/program files (x86)/atollic/truestudio for stm32 9.3.0/armtools/bin/../lib/gcc/arm-atollic-eabi/6.3.1/../../../../arm-atollic-eabi/lib/armv7-m\libc_nano.a(lib_a-nano-svfprintf.o)
 .debug_frame   0x00003808       0xac c:/program files (x86)/atollic/truestudio for stm32 9.3.0/armtools/bin/../lib/gcc/arm-atollic-eabi/6.3.1/../../../../arm-atollic-eabi/lib/armv7-m\libc_nano.a(lib_a-nano-vfprintf.o)
 .debug_frame   0x000038b4       0x2c c:/program files (x86)/atollic/truestudio for stm32 9.3.0/armtools/bin/../lib/gcc/arm-atollic-eabi/6.3.1/../../../../arm-atollic-eabi/lib/armv7-m\libc_nano.a(lib_a-sbrkr.o)
 .debug_frame   0x000038e0       0x88 c:/program files (x86)/atollic/truestudio for stm32 9.3.0/armtools/bin/../lib/gcc/arm-atollic-eabi/6.3.1/../../../../arm-atollic-eabi/lib/armv7-m\libc_nano.a(lib_a-stdio.o)
 .debug_frame   0x00003968       0x2c c:/program files (x86)/atollic/truestudio for stm32 9.3.0/armtools/bin/../lib/gcc/arm-atollic-eabi/6.3.1/../../../../arm-atollic-eabi/lib/armv7-m\libc_nano.a(lib_a-writer.o)
 .debug_frame   0x00003994       0x2c c:/program files (x86)/atollic/truestudio for stm32 9.3.0/armtools/bin/../lib/gcc/arm-atollic-eabi/6.3.1/../../../../arm-atollic-eabi/lib/armv7-m\libc_nano.a(lib_a-closer.o)
 .debug_frame   0x000039c0       0x2c c:/program files (x86)/atollic/truestudio for stm32 9.3.0/armtools/bin/../lib/gcc/arm-atollic-eabi/6.3.1/../../../../arm-atollic-eabi/lib/armv7-m\libc_nano.a(lib_a-fstatr.o)
 .debug_frame   0x000039ec       0x2c c:/program files (x86)/atollic/truestudio for stm32 9.3.0/armtools/bin/../lib/gcc/arm-atollic-eabi/6.3.1/../../../../arm-atollic-eabi/lib/armv7-m\libc_nano.a(lib_a-isattyr.o)
 .debug_frame   0x00003a18       0x68 c:/program files (x86)/atollic/truestudio for stm32 9.3.0/armtools/bin/../lib/gcc/arm-atollic-eabi/6.3.1/../../../../arm-atollic-eabi/lib/armv7-m\libc_nano.a(lib_a-locale.o)
 .debug_frame   0x00003a80       0x2c c:/program files (x86)/atollic/truestudio for stm32 9.3.0/armtools/bin/../lib/gcc/arm-atollic-eabi/6.3.1/../../../../arm-atollic-eabi/lib/armv7-m\libc_nano.a(lib_a-lseekr.o)
 .debug_frame   0x00003aac       0x48 c:/program files (x86)/atollic/truestudio for stm32 9.3.0/armtools/bin/../lib/gcc/arm-atollic-eabi/6.3.1/../../../../arm-atollic-eabi/lib/armv7-m\libc_nano.a(lib_a-mbtowc_r.o)
 .debug_frame   0x00003af4       0x28 c:/program files (x86)/atollic/truestudio for stm32 9.3.0/armtools/bin/../lib/gcc/arm-atollic-eabi/6.3.1/../../../../arm-atollic-eabi/lib/armv7-m\libc_nano.a(lib_a-memmove.o)
 .debug_frame   0x00003b1c       0x30 c:/program files (x86)/atollic/truestudio for stm32 9.3.0/armtools/bin/../lib/gcc/arm-atollic-eabi/6.3.1/../../../../arm-atollic-eabi/lib/armv7-m\libc_nano.a(lib_a-mlock.o)
 .debug_frame   0x00003b4c       0x3c c:/program files (x86)/atollic/truestudio for stm32 9.3.0/armtools/bin/../lib/gcc/arm-atollic-eabi/6.3.1/../../../../arm-atollic-eabi/lib/armv7-m\libc_nano.a(lib_a-nano-reallocr.o)
 .debug_frame   0x00003b88       0x2c c:/program files (x86)/atollic/truestudio for stm32 9.3.0/armtools/bin/../lib/gcc/arm-atollic-eabi/6.3.1/../../../../arm-atollic-eabi/lib/armv7-m\libc_nano.a(lib_a-readr.o)
 .debug_frame   0x00003bb4       0x5c c:/program files (x86)/atollic/truestudio for stm32 9.3.0/armtools/bin/../lib/gcc/arm-atollic-eabi/6.3.1/../../../../arm-atollic-eabi/lib/armv7-m\libc_nano.a(lib_a-reent.o)
 .debug_frame   0x00003c10       0x3c c:/program files (x86)/atollic/truestudio for stm32 9.3.0/armtools/bin/../lib/gcc/arm-atollic-eabi/6.3.1/../../../../arm-atollic-eabi/lib/armv7-m\libc_nano.a(lib_a-wctomb_r.o)
 .debug_frame   0x00003c4c       0x20 c:/program files (x86)/atollic/truestudio for stm32 9.3.0/armtools/bin/../lib/gcc/arm-atollic-eabi/6.3.1/../../../../arm-atollic-eabi/lib/armv7-m\libc_nano.a(lib_a-nano-msizer.o)
 .debug_frame   0x00003c6c       0xac c:/program files (x86)/atollic/truestudio for stm32 9.3.0/armtools/bin/../lib/gcc/arm-atollic-eabi/6.3.1/armv7-m\libgcc.a(_arm_addsubdf3.o)
 .debug_frame   0x00003d18       0x50 c:/program files (x86)/atollic/truestudio for stm32 9.3.0/armtools/bin/../lib/gcc/arm-atollic-eabi/6.3.1/armv7-m\libgcc.a(_arm_muldivdf3.o)
 .debug_frame   0x00003d68       0xc4 c:/program files (x86)/atollic/truestudio for stm32 9.3.0/armtools/bin/../lib/gcc/arm-atollic-eabi/6.3.1/armv7-m\libgcc.a(_arm_cmpdf2.o)
 .debug_frame   0x00003e2c       0x20 c:/program files (x86)/atollic/truestudio for stm32 9.3.0/armtools/bin/../lib/gcc/arm-atollic-eabi/6.3.1/armv7-m\libgcc.a(_arm_unorddf2.o)
 .debug_frame   0x00003e4c       0x24 c:/program files (x86)/atollic/truestudio for stm32 9.3.0/armtools/bin/../lib/gcc/arm-atollic-eabi/6.3.1/armv7-m\libgcc.a(_arm_fixdfsi.o)
 .debug_frame   0x00003e70       0x4c c:/program files (x86)/atollic/truestudio for stm32 9.3.0/armtools/bin/../lib/gcc/arm-atollic-eabi/6.3.1/armv7-m\libgcc.a(_arm_addsubsf3.o)
 .debug_frame   0x00003ebc       0xc8 c:/program files (x86)/atollic/truestudio for stm32 9.3.0/armtools/bin/../lib/gcc/arm-atollic-eabi/6.3.1/armv7-m\libgcc.a(_arm_cmpsf2.o)
 .debug_frame   0x00003f84       0x24 c:/program files (x86)/atollic/truestudio for stm32 9.3.0/armtools/bin/../lib/gcc/arm-atollic-eabi/6.3.1/armv7-m\libgcc.a(_arm_fixunssfsi.o)
 .debug_frame   0x00003fa8       0x2c c:/program files (x86)/atollic/truestudio for stm32 9.3.0/armtools/bin/../lib/gcc/arm-atollic-eabi/6.3.1/armv7-m\libgcc.a(_aeabi_uldivmod.o)
 .debug_frame   0x00003fd4       0x34 c:/program files (x86)/atollic/truestudio for stm32 9.3.0/armtools/bin/../lib/gcc/arm-atollic-eabi/6.3.1/armv7-m\libgcc.a(_udivmoddi4.o)
